:020000040800F2
:10000000E83402201D030008257D0008AD6A0008C1
:10001000497C0008E53A0008C9BD0008000000005E
:1000200000000000000000000000000015A900080A
:100030008D580008000000003B31000819850008B9
:1000400037030008370300083703000837030008A8
:100050003703000837030008370300083703000898
:100060003703000837030008370300083703000888
:100070003703000837030008370300083703000878
:10008000370300083703000837030008E93D00087C
:10009000793C000837030008370300089D58000822
:1000A0003703000837030008370300083703000848
:1000B00037030008C9B10008E9B100083703000898
:1000C0003703000837030008370300083703000828
:1000D0003703000841B50008ADB6000825B8000890
:1000E0003703000837030008370300083703000808
:1000F00037030008370300083703000837030008F8
:1001000037030008370300083703000837030008E7
:1001100055B30008370300083703000829B2000868
:1001200037030008370300083703000837030008C7
:10013000370300083703000837030008254100088B
:10014000FD3F0008370300083703000837030008A5
:1001500037030008370300083703000811BA000806
:100160003703000837030008370300083703000887
:100170003703000837030008370300083703000877
:10018000370300083703000800F002F800F0B6F863
:100190000AA090E8000C82448344AAF10107DA45E2
:1001A00001D100F0ABF8AFF2090EBAE80F0013F07E
:1001B000010F18BFFB1A43F00103184774570100E1
:1001C0009457010010F8013B0A4413F0030408BFE0
:1001D00010F8014B1D1108BF10F8015B641E05D01B
:1001E00010F8016B641E01F8016BF9D1002D15D0D8
:1001F00010F8014B03F00C030C2BA1EB04040ABF15
:1002000010F8013BA4EB8314A4EB032405F10103D4
:1002100014F8016B5B1E01F8016BF9D5914238BFF0
:1002200010F8013BD1D3704700230024002500269D
:10023000103A28BF78C1FBD8520728BF30C148BF49
:100240000B6070476E2900F05285702900F0918193
:10025000662914F0BB87652914F0B887672914F064
:10026000B587612914F0B48703681B0A28BF41F0E1
:100270008001692900F00281642900F0FF8075295E
:1002800000F0FC806F2901F04680782900F05D8144
:10029000E92900F0E187E42900F0DE87F52900F084
:1002A000DB87EF2901F04380F82900F05C810368C7
:1002B000DB0928BF41F08001632900F062877329C0
:1002C00000F06787E32901F0C585F32901F0CA85AD
:1002D000002070471FB514F06CFF01F0A1FB040073
:1002E0000020002114F0AEF8401C606000200021C6
:1002F00014F0BEF8E0601FBD10B510BD02F020F88C
:100300001146FFF7E7FF11F0D3FA02F069FA03B4E0
:10031000FFF7F2FF03BC0EF0D9FB0000094880474D
:1003200009480047FEE7FEE7FEE7FEE7FEE7FEE7D7
:10033000FEE7FEE7FEE7FEE704480549034A054BF2
:100340007047000061B1000889010008E82502201B
:10035000E8340220E825022072B6704762B6704782
:10036000EFF3108072B6704780F31088704730BF8B
:10037000704720BF7047B0FA80F0704790FAA0F045
:10038000B0FA80F0704790FAA0F070471CB50C46A8
:10039000064B7B4469460090204600F0D0FE0446A0
:1003A0000020694600F0DEFE20461CBDCF0D000097
:1003B0000FB41CB5084B06AA7B446946009005980B
:1003C00000F0BDFE04460020694600F0CBFE20464A
:1003D0001CBC5DF814FB0000A90D000070B50446BC
:1003E00085690068C10601D5302600E02026C007D7
:1003F00007D070BDD4E9012130469047206A401CE7
:1004000020626D1EF6D570BD70B504468569007812
:10041000C00707D170BDD4E9012120209047206A90
:10042000401C20626D1EF6D570BD70B50C460546A9
:10043000012A05D02878800600D5EA69002302E069
:10044000012305E05B1C934202D2E05C0028F9D155
:10045000A869E618C01AA861286A184428622846C4
:10046000FFF7BCFF04E0D5E9012114F8010B904728
:10047000B442F8D32846FFF7C7FF70BD2DE9F0411D
:100480000646002410687529314616A510D000F0E4
:10049000C3FB002802DA404213A507E031688A074F
:1004A00001D512A502E0490704D511A5012401E0F8
:1004B00000F0BBFB00210A2206F1240709E0B0FB93
:1004C000F2FCB0FBF2F302FB1C003030785418460B
:1004D000491C0028F3D123462A463046BDE8F041A6
:1004E00000F0ACBB000000002D0000002B0000005D
:1004F00020000000F0B40D460188090502D5214C0A
:100500007C4402E01F4C7C440E34002100F12406A0
:1005100008E002F00F071209E75D42EA03721B09C7
:100520007754491C52EA0307F3D1027800231207DB
:1005300004D5702D06D009B1022311342246F0BC37
:1005400000F07CBB01231034F8E770B504460D467B
:100550002146106800F069FB024629462046BDE8A6
:1005600070400023C6E7D21D22F00703D3E9002321
:10057000C0E70368126843F0200303600823C361E7
:100580000023B7E7704E01002DE9F05F894604466D
:100590004FF0000ADFF874B1FB44C0F820A02046F9
:1005A000E1688847002874D0252806D0D4E90121C5
:1005B0009047206A401C2062F1E700265F462046F3
:1005C000E16888472028054607DB312D05D27819D8
:1005D00010F8200C08B10643F1E7B00701D526F06A
:1005E0000406C4F81CA00027C4F818A02A2D09D0BE
:1005F00028460EF064FA38B304EB8708303DC8F89B
:10060000185019E059F8041B204604EB8702916149
:10061000E1688847012F054618D1E069002820DAF3
:1006200026F020061DE0D8F8180000EB800005EB4E
:1006300040003038C8F818002046E1688847054671
:100640000EF03DFA0028EED1012F0AD02E2D08D150
:100650002046E16888477F1C0546022F46F02006A9
:10066000C4DBA069002803DA404246F00106A0611D
:10067000F00701D026F010066C2D0BD0682D09D0A4
:100680004C2D39D06A2D35D0742D35D07A2D33D0FC
:1006900016E038E0E1682F4620468847B842054614
:1006A00009D16C2F26D04FF48060E16806432046C4
:1006B0008847054604E06C2F1AD04FF4807006433B
:1006C0000DB3A5F14100192802D8203546F4006683
:1006D0004A462946204626604E46FFF7B3FD80B1C4
:1006E00001280BD0F61D26F0070000F1080956E797
:1006F0004020E4E78020D8E70020D6E706F104098F
:100700004DE7284652E7206ABDE8F09F004E010001
:100710000FB400B58DB010A9099000910B904FF067
:10072000FF300A9000200C90064878440690064856
:1007300078446A4607900F9909A801F093F80DB024
:100740005DF814FB571100006F1100002DE9FF5FE9
:100750001D464FF0FF3B91464FF000085F46D5E93C
:100760000146A96901987F1C8847296A8246884703
:100770000028F6D1BAF1FF3F0CD0002E24F4C0645B
:1007800019DD600614D5BAF12B0F09D0BAF12D0F7F
:100790000ED103E0584604B0BDE8F09F44F48064F5
:1007A000A96901987F1C8847761E8246002E02DDCB
:1007B000BAF1300F03D0B9F1000F26D032E0A969A9
:1007C000761E01987F1C44F400748847002E8246F0
:1007D00005DDBAF1780F06D0BAF1580F03D0B9F1A0
:1007E000000F10D01EE0B9F1000F02D0B9F1100FC8
:1007F00018D1A969761E01987F1C24F400748847DB
:100800008246102002E0082000E00A20814609E02C
:10081000A96908FB0908761E01987F1C44F400743E
:1008200088478246002E05DD4946504600F08AFD85
:100830000028EDDAE96901988847A00502D46FF035
:100840000100A8E7E00725D1600613D5600502D5B1
:10085000C8F1000000E0404629680A1D2A600968C6
:10086000220501D5087015E0220701D5088011E0A6
:1008700008600FE02868011D29600068210502D585
:1008800080F8008006E0210702D5A0F8008001E092
:10089000C0F8008038467EE770B5064600F0A0F943
:1008A0000468054630460A22002101F05AF82C60FF
:1008B00070BD2DE9F05F93460F4680460446002642
:1008C00000F08EF9D0F80090824614F8015B2DB14B
:1008D00000F07EF90068405DC007F6D12B2D02D0F4
:1008E0002D2D1AD0641E0021CAF800105A46394630
:1008F000204600F0E7FF014627B13868A04201D149
:10090000C7F80080DAF80000022809D0CAF8009081
:10091000700505D54842BDE8F09F46F48066E2E7E1
:100920000846F8E7014A01F055B80000E42C002021
:1009300040EA0103024630B59B0710D14FF0013465
:1009400000E008C208C91D1B9D4315EAC41FF8D06A
:1009500013F0FF0102F8011B0DD01B0AF8E711F894
:10096000013B002B02F8013B05D011F8013B002BA5
:1009700002F8013BF3D130BD2DE9F0410E460546AA
:10098000002400E0641C285D00F039F90746305D62
:1009900000F035F9381A02D1295D0029F2D1BDE8FD
:1009A000F08110B5431C02E010F8011B71B1810702
:1009B000FAD14FF0013202C88C1A8C4314EAC211EA
:1009C000F9D0C01A0A0603D0C01E10BDC01A10BD4F
:1009D0000A0401D0801E10BD0902FCD0401E10BDCB
:1009E00040EA010370B59B072ED14FF00136042A6F
:1009F0002AD308C810C99D1B9D43121F15EAC615AE
:100A000017D0D8B2E1B2401A50EA056110D198B2BD
:100A1000A1B2401A50EA05410AD123F07F4024F0E8
:100A20007F41401A50EA052102D1180EA0EB146054
:100A300070BDA342DBD018BA21BA884201D9012087
:100A400070BD4FF0FF3070BD0AB9002070BD10F8C6
:100A5000013B11F8014B63B1A3420AD1521E08D0E9
:100A600010F8013B11F8014B1BB1A34201D1521EFA
:100A7000EDD1181B70BD421E12F8013F002BFBD1B7
:100A800011F8013B002B02F8013BF9D17047032A12
:100A900040F2308010F0030C00F0158011F8013B9B
:100AA000BCF1020F624498BF11F801CB00F8013B82
:100AB00038BF11F8013BA2F1040298BF00F801CB46
:100AC00038BF00F8013B11F0030300F02580083A1D
:100AD000C0F0088051F8043B083A51F804CBA0E874
:100AE0000810F5E7121D5CBF51F8043B40F8043BC9
:100AF000AFF30080D20724BF11F8013B11F801CBFE
:100B000048BF11F8012B24BF00F8013B00F801CBCE
:100B100048BF00F8012B704710B5203AC0F00B8099
:100B2000B1E81850203AA0E81850B1E81850A0E8F1
:100B30001850BFF4F5AF5FEA027C24BFB1E818504B
:100B4000A0E8185044BF18C918C0BDE810405FEABB
:100B5000827C24BF51F8043B40F8043B08BF704737
:100B6000D20728BF31F8023B48BF11F8012B28BF3C
:100B700020F8023B48BF00F8012B70474FF00002FD
:100B800000B5134694469646203922BFA0E80C5083
:100B9000A0E80C50B1F12001BFF4F7AF090728BF5E
:100BA000A0E80C5048BF0CC05DF804EB890028BFDA
:100BB00040F8042B08BF704748BF20F8022B11F003
:100BC000804F18BF00F8012B70477047704770477F
:100BD00010B500F025FF001D10BD00BF69380100F1
:100BE000004870478825022010B5FFF7F9FF00681C
:100BF00010BD10B50446FFF7F3FF046010BD10B53B
:100C00000446FFF7E5FF0068005DC00602D504F169
:100C1000200010BD204610BD09684A0501D540B22C
:100C20007047C905FCD500B2704709684A0501D56F
:100C3000C0B27047C905FCD580B270472DE9F047B6
:100C40000D4699469246044600F12408016888063C
:100C500004D5E06921F01001216000E00120A842E4
:100C600001DD471B00E00027A1697A1902EB0900AA
:100C7000081AA0612078C00602D42046FFF7AEFB18
:100C8000002608E0D4E901211AF806009047206AFE
:100C9000401C761C20624E45F4DB2078C0060AD545
:100CA0002046FFF79BFB06E0D4E901213020904766
:100CB000206A401C2062381EA7F10107F4DC07E01F
:100CC000D4E9012118F805009047206A401C2062F1
:100CD000281EA5F10105F3DC2046FFF795FB2078DF
:100CE000000602D50220BDE8F0870120FBE711686D
:100CF0000268006A530501D508700AE0D30501D5E2
:100D0000088006E0130603D5C217C1E9000200E01F
:100D100008600120704770472DE9FF4F0C461E46C2
:100D20004FF0FF378BB0D2E90001DDF860800A9008
:100D30008A46C1F30A5505B93D46002108464FF0E1
:100D40000000BAF1000F00F4400005DA00EB80006B
:100D50004FF4400101EA50004FEA9059B9F1010FF8
:100D600000DDB9460A9850EA4A000ED044F6105009
:100D7000A5F2FF3545432F14B8F1000F1ED0754280
:100D8000291E1EDDC9F100021CE0B8F1010F4FF071
:100D9000000001D0302103E0F24305E02154401C63
:100DA000B042FBDB30460022002121540B99C1F8F0
:100DB0000880C1E900200FB0BDE8F08FBD1B6D1C9D
:100DC000DEE74A4600DA694206A801F009FA06ABF6
:100DD00093E8070003AB83E8070050460A9901F047
:100DE0005CFD8DE80700A0F500501F3800900398C7
:100DF000002D0ADD42F21F014A460844002303A9E0
:100E00000390684602F008F809E0A0F500504A4651
:100E10001F38002303A90390684602F027F88DE8E5
:100E200007000004000C03D04FF0FF30410800E041
:100E30001046B8F1000F03D00022009215461EE0C4
:100E4000751E05D400F0F0FD303262556D1EF9D5E7
:100E5000B3460122084302D000227F1C04E0207820
:100E6000302801D100227F1E002A099784D01DE07E
:100E7000112D07DA00F0D8FD303262556D1C50EAB2
:100E80000102F5D1084302D00098C8B10EE000215C
:100E9000681E05E0235C625C63542254401E491CBA
:100EA0008142F7DBAB46A81B401E0990002004F8E6
:100EB0000B000B98099AC0F80880C0E9002B7AE76C
:100EC00011264FF0000857E72DE9F04F88460446F9
:100ED000D21D22F0070191B0D1E90001CDE90A014C
:100EE0000BF012FD02460B98C00F01D02D2007E039
:100EF0002068810701D52B2002E0202101EAC000F3
:100F0000032A099001D0072A05DB03464146204603
:100F100000F056FF0BE12078800601D5E06900E083
:100F20000620B8F1650F814606D0B8F1660F18D0DB
:100F3000B8F1670F70D131E00020B9F1110F0090C6
:100F400001DB112301E009F101030AAA01A90CA8A0
:100F5000FFF7E2FEDDE90C70002609F1010583468A
:100F600047E001204B4600904FF000470AAA01A934
:100F70000CA8FFF7D1FEDDE90DB00C995D46002607
:100F800010B909F101000D18B9EB050003D4C0F147
:100F9000FF3609F10105A5EB09002BE0B9F1010FBE
:100FA00001DA4FF001090020B9F1110F0090484615
:100FB00001DD112300E003460AAA01A90CA8FFF7EE
:100FC000ABFEDDE90C704D46002683462078000715
:100FD0000AD4AB4500DA5D4601A8012D04DD4119B4
:100FE00011F8011C302907D04F4502DA17F1040F20
:100FF00004DA012082460FE06D1EEEE7002F02DCCE
:10100000ED1B3E4403E0781CA84200DD7D1CB81BAC
:1010100000F1010A4FF000472078000703D4AA45E9
:1010200001DB4FF0FF3A0021B7F1004F0DF143080B
:101030008DF8431024D002202B23002F01DA7F42A9
:101040002D230A21021EA0F1010000DC5FB197FBF5
:10105000F1FC97FBF1F201FB1C7C17460CF1300C04
:1010600008F801CDEEE7A8F1010003702188090519
:1010700001D5452100E06521A0F1010800F8011C1F
:1010800009980FA9A1EB0807FF1D00B10120411924
:1010900001EBEA70A1693844081A401EA06120786B
:1010A000C00602D42046FFF799F9099828B1D4E97F
:1010B00001219047206A401C20622078C00622D57A
:1010C0002046FFF78BF91EE0002E04DBB34502DD5E
:1010D00001A8805D00E03020D4E901219047206A1A
:1010E000401C2062761CAAF101005FEA000A0AD1C6
:1010F00000F096FCC0680168405CD4E9012190478B
:10110000206A401C2062281EA5F10105DCDC07E0F6
:10111000D4E9012118F8010B9047206A401C206295
:10112000381EA7F10107F3DC2046FFF76DF9032015
:1011300011B041E601694A1C02610878704700B5A8
:101140008FB0CDE901310021059105497944CDE900
:10115000031011466846FFF717FA0FB000BD0000F4
:10116000E5FFFFFF0A6802F8010B0A60704710B53F
:10117000436913B1AFF3008001E0FFF756F9012096
:1011800010BD127800F124010A7000224A70012279
:10119000EDE711684FF0FF32E9E700002DE9FF5F4E
:1011A00015468A460446DFF8AC80F8440027D8E9A3
:1011B00000103E46CDE9001010E03AF816106A46DD
:1011C00002A801F07FF8411C07D02178890603D5D9
:1011D000E269391891420DD80744761C20788006C0
:1011E00002D5E069B84205DDAE42E6DB3AF816000A
:1011F0000028E2D1A069C01BA0612046FFF7EEF8ED
:10120000D8E90010CDE90010002017E03AF81810D6
:101210006A4602A801F056F8B0F1FF3F81460BD0B4
:1012200000250DF1080B05E0D4E901211BF80500AC
:1012300090476D1C4D45F7D308F10100B042804640
:10124000E4DB206A384420622046FFF7DDF8BDE881
:10125000FF9F0000224301002DE9F0418046D21D8E
:1012600022F007020025D2E90002F52915A614D0C4
:10127000011E72F1000106DA0023D0EB030063EBDC
:10128000020211A608E0D8F800108B0701D50FA6BE
:1012900002E0490701D50EA601251146002408F1F8
:1012A000240704E000F0C0FB30323A55641C50EAD9
:1012B0000102F7D12B46324621464046BDE8F041B7
:1012C000FFF7BCBC000000002D0000002B00000058
:1012D0002000000030B4002100F1240408E002F0F6
:1012E0000705D208303542EA4372DB086554491CD1
:1012F00052EA0305F3D10468002310A2250707D59D
:10130000A40600D421B1C46901230DA2641EC461E6
:1013100030BCFFF793BC10B5044621461068FFF7B8
:1013200084FC02462046BDE810400023D2E7D21DCF
:1013300022F00701D1E90023CCE700000000000003
:10134000300000003A2800D2303820F02002412A34
:1013500001D3A2F13700884201D34FF0FF3070472C
:101360002DE9FF4F06468BB00878FF2806D0491CB0
:101370002D2805D000244FF0000908E000200CE0E3
:101380000124F8E709EB8903491C00EB43090878BD
:10139000FF28F7D114B1C9F100008146107800256B
:1013A0002C46AA4629462D2801D02B2804D1521CB0
:1013B0002D2813D0002082468B461078FF280FD0AE
:1013C0004FF0000C0A21521CA5FB017804FB01819F
:1013D00005FB0C11C5194BEB0104EEE70120EAE710
:1013E000002108464FF00000BAF1000F02D000EBD8
:1013F00080004008C0F38157012F01DD4FF0FF3717
:101400000E9955EA040009EB01080BD04FF00209D0
:1014100018F5FA7F16DA4FEACA70002F706008DDFF
:10142000012007E04FEACA70C6E900B00FB0BDE87E
:10143000F08F00203060FFF7D3FBC0F80090182138
:10144000084616E0B8F5FA7F18DD002F02DAF748F3
:10145000784401E0F6487844D0E90010C6E900106D
:1014600040EACA707060FFF7BBFBC0F8009014211F
:1014700008460FB0BDE8F04F13F0A5BE00210846A6
:101480004FF00000B8F10001099002DAC7F1000244
:1014900000E03A4601DAC8F1000106A800F0A0FE1B
:1014A00006AB93E8070003AB83E8070044F23E0075
:1014B0005BEA04010090584604D144F21E012C4618
:1014C0005D460091210C0904014306D100992404D2
:1014D00044EA15442D041039009104F07F41014382
:1014E00006D10099240244EA15642D0208390091BE
:1014F00004F07041014306D10099240144EA1574B7
:101500002D01091F009104F04041014306D10099CB
:10151000A40044EA9574AD00891E009104F00041D6
:10152000084304D100986D196441401E00904FF0AB
:1015300001033A466846B8F1000FCDE9014503A919
:1015400002DD01F0A8FC01E001F07BFCBAF1000F24
:1015500004460D4601D084F00044002108464FF0B7
:101560000000099940F2FF77484010F00C0F07D1B6
:1015700024F00040284303D0C4F30A50B84212D1EB
:10158000FFF72EFBC0F80090C4F30A50B8420AD10E
:10159000A8487844D0E90010C6E9001004F00041E2
:1015A0000843706042E7C6E900543FE72DE9FF4F6A
:1015B0001F464FF0000A4FF0FF38454691B0D7E97B
:1015C0000146CDF83CA000F02BFAC0680168405CF1
:1015D0001090B96912986D1C8847396A814688470E
:1015E0000028F6D1B9F1FF3F0AD0002E24F4D064D0
:1015F00011DDB9F12B0F08D0B9F12D0F0BD102E09D
:10160000404615B013E744F48064B96912986D1C24
:101610008847761E8146600504A901D52D2000E08B
:101620002B20002E01F1010B0DF130088DF8100078
:101630003FDDB9F1690F08D0B9F1490F05D0B9F113
:101640006E0F02D0B9F14E0F1CD13B4601A8009598
:1016500080E85002DDE912126FF0020013F01EFE66
:10166000C11CCED10EE0B96912986D1C8847814625
:101670001398761E44F4007405600F98401C002EE9
:101680000F9016DDB9F1300FEDD0B9F1780F02D01F
:10169000B9F1580F0DD10F9801280AD13B46CDE979
:1016A0000054DDE91212001F029613F0F5FDC11C73
:1016B000A7D1109989453ED144F0800406E01399E2
:1016C000681CAAF1010A44F400740860B9696D1C31
:1016D0001298761E884730288146F0D02BE010996A
:1016E000894505D1200603D4761E44F0800418E015
:1016F00048460DF0E4F908B3761E0DF123018B4541
:1017000044F4007408D2A9F130000BF8010B200654
:1017100007D5AAF1010003E0200602D40AF1010076
:101720008246A00502D51399681C0860B969129811
:101730006D1C88478146002ED1DC53E0002E51DD20
:10174000B9F1650F02D0B9F1450F4BD1A00549D5CC
:10175000B9696D1C1298761E24F440748847002ED7
:1017600081460CDD2B2804D0B9F12D0F07D144F4AC
:101770008074B96912986D1C8847761E8146E00511
:1017800001D52D2100E02B2108F8011BCDF80080A8
:1017900021E0761E0DF13901884544F400740CD225
:1017A000A9F1300010F0FF0088F8000002D1009984
:1017B000884509D908F1010806E0E00501D51E4871
:1017C00001E042F20F708246B96912986D1C884799
:1017D000814613980560002E04DD48460DF06FF930
:1017E0000028D6D1F96912988847FF2053468BF814
:1017F000000088F8000000200A900B9004AA0CA9B1
:101800000AA8FFF7ADFDA00502D46FF00100F8E6CD
:1018100014F0240F12D0E0071CD13868DDE90A1259
:10182000031D3B600068C0E9001213E0044501009D
:10183000F6440100BA430100F1D8FFFF0AA9684647
:101840000DF02AF9E00705D13868009A011D3960CA
:10185000006802602846D4E60268114413780160EB
:1018600018467047D160054979445161044979446B
:10187000116200211161114600F0F8BAEDFFFFFF7F
:1018800041020000426842B1016811F8013B23B1F6
:10189000521EC0E90012184670470121C160881E1F
:1018A000704742685AB1C368016843B983688B4284
:1018B00005D0491E521CC0E90012002070474FF0AD
:1018C000FF3070472DE9F05F824615468B460027B2
:1018D0000AF10104B9460078302801D09DB113E027
:1018E00014F8010B0127782803D0582801D045B1FE
:1018F0000AE00DB1102D07D1002714F8010B1025B7
:1019000002E0082500E00A250026B0460EE005FBAF
:10191000080005FB06F101271FFA80F801EB1046CD
:10192000B6F5803F00D3B94614F8010B2946FFF7FE
:1019300009FD0028EBDABBF1000F05D00FB1641EE2
:1019400000E05446CBF80040B9F1000F06D0FFF795
:1019500047F902210160C81EBDE8F09F48EA064031
:10196000FAE72DE9F04791460F46804604460026E7
:1019700014F8015B2DB1FFF72BF90068405DC0073B
:10198000F6D12B2D02D02D2D18D0641E4A46394693
:101990002046FFF797FF27B13968A14201D1C7F868
:1019A00000804FF0020471050BD54042002803DD92
:1019B000FFF716F90460A007BDE8F08746F48066DB
:1019C000E4E70028F8DAFFF70BF904606FF0004055
:1019D000F2E700002DE9F04115460E46040002D161
:1019E0002C6804B90BA4204600F09CFC0444207829
:1019F00070B127463146384600F084FC0444207814
:101A000010B1002004F8010B38462C60BDE8F081CD
:101A10000027F9E7000000000048704788250220F1
:101A200000487047A825022030B5B0F10A024FEAFD
:101A3000900E71F100034EEA817EB0EB0E0061EB77
:101A400091014FEA101E4EEA017E10EB0E0041EBB1
:101A500011114FEA102E4EEA016E10EB0E0041EB11
:101A600011214FEA104E4EEA014E10EB0E0041EBF1
:101A70001141401841F100014FEAD00040EA4170A5
:101A80004FEAD10110EB80054FEA810444EA9074DB
:101A900044EB01046D1944EB0404521BA3414FF0C5
:101AA000000348BF0A3200D530BD401C41F100019F
:101AB00030BD10B50446FFF78BF80068005D00F0FC
:101AC000010010BD2DE9F04F04460D46D21D22F055
:101AD000070089B0D0E90097484639460AF014FF5C
:101AE0000246F80F01D02D2307E02068810701D5B9
:101AF0002B2302E0202101EAC0038DF820300BB136
:101B0000012000E00020032A824601D0072A04DBDE
:101B10002946204600F054F93FE12078800601D4A0
:101B20000D2500E0E569C7F30A560D2D49DA0021BD
:101B30004FEA175B08464FF00000002F00F440000A
:101B400007DA00EB80004FF4400100EBD07001EAAF
:101B500060008115012901DD4FF0FF3100224FEABD
:101B6000850CBCF1180F06D31346ACF118004FF0EA
:101B70008052C24003E04FF4801323FA0CF30CF1BF
:101B80000C0CBCF1200F04D3ACF1200C09FA0CF0C2
:101B900001E007FA0CF000294FF0004801DD18B908
:101BA0000FE00ED140450CD319EB02095F4121B97A
:101BB000404502D19F4329EA0209BBEB175F00D0E1
:101BC000761C2088000502D57B48784402E07A48DC
:101BD0007844193808AA302302F80A30037C0AF145
:101BE0000101002E0AF1020A53546A4602DC4FF04A
:101BF000300101E04FF031014FF001088DF8001085
:101C000002D0A6F2FF3603E059EA470100D06B4E3E
:101C1000002D02DC2178090704D54FF002082E219F
:101C20008DF80110C44600210BE0C7F303433F01C8
:101C3000C35C491C6D1E02F80830052908F1010833
:101C400001DA002DF1DC00210CE000EB1973491CD6
:101C50001B786D1E082902F808304FEA091908F1AF
:101C6000010801DA002DF0DC21688B0602D516E0B0
:101C7000A8F10108E04505DD02EB080313F8013C7B
:101C8000302BF5D0B8F1000F09DD02EB080313F893
:101C9000013C2E2B03D1090701D4A8F10108002D26
:101CA00005DD3E2102F808106D1E08F10108407C98
:101CB000002E02F8080008F1010804DA2D2076420F
:101CC00002F8080002E02B2002F808000A214FF475
:101CD0007A70864208F101080BDB96FBF0F3303393
:101CE00002F8083096FBF0F308F1010800FB1366D8
:101CF00001E0642E0CDB642096FBF0F3303302F835
:101D0000083096FBF0F308F1010800FB136601E0D0
:101D10000A2E06DB96FBF1F0303002F8080008F1DD
:101D2000010896FBF1F001FB1060303002F808006A
:101D3000A16908F1010808EB050202EB0A00081A84
:101D4000A0612078C00602D42046FEF747FB216A36
:101D500008AE01EB0A00206204E0D4E9012116F884
:101D6000010B9047BAF1010AF7D22078C00602D5DC
:101D70002046FEF733FB6E4609E016F8010B3E28BD
:101D80000FD0D4E901219047206A401C2062B8F1AD
:101D90000108F2D22046FEF737FB09B00320BDE868
:101DA000F08F206A2844206203E0D4E9012130202A
:101DB00090476D1EEBD3F8E7A53A010002FCFFFF48
:101DC0002DE9F0411F46044603260168072A01F465
:101DD000006004DB08B116A505E016A503E008B114
:101DE00015A500E015A521F010002060A069C01E17
:101DF000A0610FB1401EA0612046FEF7EFFA4FB17F
:101E0000D4E9012138469047206A401C2062C01C5A
:101E1000206206E0206AFAE7D4E9012115F8010BF7
:101E20009047761EF8D22046FEF7EEFABDE8F08124
:101E30004E414E006E616E00494E4600696E66006E
:101E400010B5436913B1AFF3008001E0FFF7A6F9C5
:101E5000012010BD128800F1240182840022C28476
:101E60000122EDE711684FF0FF32E9E72DE9F34F6A
:101E70004FF0000A0C4656468DB001200C9001F13F
:101E80000C000B9062690B9801219047051E2DD024
:101E9000252D2CD0216A8847C0B162690B98012199
:101EA0009047216A88470028F7D16269411E0B9844
:101EB000904700E0761CA1690D988847216A884701
:101EC0000028F7D1E1690D988847DBE7A1690D98F3
:101ED0008847A842074601D1761CD3E7E1690D98EF
:101EE00088477F1C02D1BAF1000F6FD06BE16269A5
:101EF0000B9800273D46394690472A2804D162694D
:101F00000B98012190470125DFF8D08262690B9878
:101F100001219047A0F130010A290AD24745E5DCAA
:101F200007EB870100EB4107303FDFD445F0100598
:101F3000ECE7E90601D46FF000476C280AD04C2882
:101F400014D0682815D06A280DD074281CD07A289F
:101F50001AD01DE062690B98012190476C2802D0CD
:101F600045F0040514E045F002050DE045F02005BC
:101F70000AE062690B9801219047682802D045F079
:101F8000080505E045F4006562690B98012190475A
:101F9000C4E9015765283DD019DC58287AD00CDCFB
:101FA000452837D004DC252826D041289ED131E0B1
:101FB00046282FD0472899D12CE05B2877D061287C
:101FC00028D063287CD0642823D15AE0F6E06F281B
:101FD00048D008DC66281DD067281BD0692821D08E
:101FE0006E2816D127E0702845D0732868D0752850
:101FF00047D078280DD14DE0A1690D988847252854
:1020000005463FF469AFE1690D9888476D1C3FF4C0
:102010006AAFD8E00D9923466A466FF0010013F0CD
:1020200039F9C5E045F0400023464FF000026060FA
:10203000A80736D43EE0E8077FF447AF2068011DCB
:1020400021600068290501D506701BE7290701D525
:10205000068017E7A90703D5F117C0E9006111E76A
:1020600006600FE745F0400023464FF0080260602D
:10207000A80716D41EE040F60E0125EA01006060B4
:1020800016E045F0400023464FF00A026060A807C2
:1020900007D40FE045F040006060A80708D523464C
:1020A00010220D996FF00100AFF3008080E007E08F
:1020B000102223460D996FF00100FEF747FB77E0F1
:1020C0004FF0000963284F46C8464B46CB4602D026
:1020D0005B2806D038E0E80601D40120A060012783
:1020E00032E06269D4F80CB00B98012190475E2869
:1020F00007D14FF0010949466269D4F80CB00B983A
:102100009047216939B900210A4603AB43F82120E1
:10211000491C0829FADBD8B3216949B308F1010841
:1021200062690B98012190475D28F4D1B9F1000F45
:1021300009D0002003A951F82020D24341F82020E3
:10214000401C0828F7DB03AB2069002820794FEA00
:1021500040701ED05B462246CDF80080CDE9019745
:102160000D9900286FF0010020DAAFF300801FE026
:10217000C11703AA00EBD1614B1121F01F0102EB43
:102180008302411A13680120884003431360C7E7A4
:1021900019E00D99224600286FF00100009702DA3D
:1021A000AFF3008004E0AFF3008001E0AFF3008004
:1021B00000280ADA401C06D10C9820B14FF0FF30FD
:1021C0000FB0BDE8F08F5046FAE7E90701D10AF1F8
:1021D000010A064400200C9054E60000CCCCCC0C44
:1021E0002DE9F047814616468AB0354878440DC837
:1021F0008DE80D0032487844801C03AC0DC884E89B
:102200000D0041F69B300844372190FBF1F290FB22
:10221000F1F5A5F1800501FB12041B3C02D56442D7
:10222000012000E00020DFF898A080460027FA4453
:10223000AAF1BE0A0EE0E0070AD03246684607EB74
:10224000470101230AEB810100F010FE8DE8070031
:1022500064107F1C002CEED1194F7F44AE3F19E073
:10226000E80715D007EB04100DF1180A90E80E00EE
:102270008AE80E00C068F04201D1981908903246F1
:10228000012306A903A800F0F1FD03AB83E80700D2
:102290006D10641C002DE3D14FF0010332466946F6
:1022A000B8F1000F03A802D000F0B6FD01E000F085
:1022B000DDFDC9E90001C9F808200AB0BDE8F087D2
:1022C0001435010070B516460C460546FEF780FC35
:1022D000036893F80101012806D0FF2C0FD8185D80
:1022E00068B101202C7070BDD3F807013246214639
:1022F00003F2071303442846BDE8704018474FF027
:10230000FF3070BD30B503461D781DB10A4603E0AD
:10231000AC4201D1181A30BD12F8014B002CF7D194
:102320005B1CF1E730B503461D783DB10A4612F853
:10233000014B1CB1AC42FAD15B1CF5E7181A30BD59
:102340007546FFF769FBAE4605006946534620F027
:102350000700854618B020B5FDF7EEFFBDE8204028
:102360004FF000064FF000074FF000084FF0000B51
:1023700021F00701AC46ACE8C009ACE8C009ACE804
:10238000C009ACE8C0098D46704700002DE9FF4F39
:102390001F464FF03C0987B04FF00042DDE91410B2
:1023A00001F10108DDF858A002EA40500390002036
:1023B00005908346054604460490B969461E089870
:1023C0008847AAF1010A0290BAF1000F3BDD02989A
:1023D0002E2815D01021FEF7B5FF00282EDB4FF078
:1023E000010B0599014317D0B9F1000F0BDB4A46E9
:1023F000C11700F03FFA05430C43A9F1040905E0B9
:10240000012004900BE008B145F001050120059082
:10241000049820B9361D02E0049800B1361FB9694E
:10242000089808F101088847BBF1000FAAF1010ADA
:102430000290C9D00999C1F80080C5E702987028B8
:1024400008D0502806D0F96908988847BBF1000FDA
:1024500014D04FE0002002900120BBF1000F049047
:1024600009D0B969089808F101088847AAF101095B
:10247000B9F1000F07DCF969089888476FF001008F
:102480000BB0BDE8F08F2B2804D02D280CD14FF0D5
:10249000FF300490B969089808F101088847A9F14C
:1024A0000109B9F1000FE6DD411CE4D00A21FEF775
:1024B00049FF0028DFDB029908F1010801EB8101E7
:1024C00000EB41000290B969089888470A21FEF79D
:1024D00039FF099AA9F10109B9F1000FC2F800808A
:1024E00001DD0028E7DAF96908988847049902981D
:1024F00000FB016655EA040004D004F040410900E5
:1025000002D006E0039898E0A40044EA9574AD0078
:10251000B61E04F00041080002D16D196441761E18
:10252000159810F0240F03D04FF00B095C4803E01E
:102530004FF028096FF07D008246564507DAAAEB76
:1025400006018944B9F1410F01DD4FF04109012035
:102550000021A9F1010200F08DF9024628400B4646
:102560002140084301D0012100E00021501E0291CA
:1025700043F1FF3128402140084301D0012000E011
:1025800000200299834651EA0B014FD000210846F2
:102590004FF00000039900F4400039B100EB8000D7
:1025A0004FF4400100EBD07001EA60008015012873
:1025B00002DD4FF0FF3000E013D0401C36D002980F
:1025C00060B3BBF1000F0CD14A460120002100F09E
:1025D00051F928402140084301D0012000E00020AB
:1025E000E0B101204A46002100F044F903464019B9
:1025F0000A4661412D1A8C4111D3B9F1400F09DD12
:10260000159810F0240F02D0AAF1340603E0AAF1C5
:10261000170600E0761C00254FF0004406E05B1E24
:1026200042F1FF3220EA030521EA0204CAF1010067
:10263000B04206DA1B49039808430190002000903D
:102640000EE0039AC4F3D321E80A0A43164940EA8C
:1026500044500A433146CDE9000268460CF025FAA1
:10266000159810F0240F0BD01598C00715D13868B5
:10267000DDE90012031D3B600068C0E900120CE0B8
:1026800002A869460CF008FA1598C00705D1386809
:10269000029A011D3960006802604046F0E60000C1
:1026A00002FCFFFF0000F07F0000F03F2DE9FF4F2C
:1026B00092461D4685B04FF00041DDE9124BDDE941
:1026C00014727F1E01EA4B50414940F0FF4940EA35
:1026D0000108002122F020004928049102D04E2850
:1026E00028D04CE03BA0012607C88DE80700A96967
:1026F0000698641C88477F1E014606D41DF8060014
:1027000018B121F0200181420BD0E9690698884771
:10271000032E34D0082E32D06FF0010009B0BDE88E
:10272000F08F761C032E01D0082EE0D1601CCAF871
:102730000000DCE7A9690698641C88477F1E2AD43C
:1027400020F02000412826D1A9690698641C8847FA
:102750007F1E20D420F020004E281CD1A9690698A5
:10276000641C88477F1E48F4002849F48009CAF891
:10277000004001D4282806D0E969069888475FEA16
:10278000CB7012D022E0A9690698641C88477F1E8E
:1027900001D4002803DAE96906988847BCE72928AC
:1027A000F1D1641CCAF80040E9E71BF0240F07D000
:1027B00028680499031D2B600068C0E9001805E033
:1027C0002868021D2A600068C0F800902046A5E72E
:1027D0000000F07F494E46494E4954590000000020
:1027E00010B50446AFF300802046BDE81040FDF769
:1027F0008EBD00004FF0013C50F8042B51F8043B13
:102800009A4221D1A2EB0C03934313EACC1317D1C4
:1028100050F8042B51F8043B9A4215D1A2EB0C035B
:10282000934313EACC130BD150F8042B51F8043B1B
:102830009A4209D1A2EB0C03934313EACC13DBD0E9
:102840004FF00000704700BFD01A01BAB1FA81F111
:1028500001F0180122FA01F0CB40C1F12001DBB2F6
:10286000C0B2C01A2CFA01F3D11A914311EAC31174
:10287000E6D17047B2F120030AD5C2F1200301FA74
:1028800002F120FA03F300FA02F041EA0301704773
:1028900000FA03F14FF0000070475FEA400C08BFF8
:1028A00091F0000F4FEA8C234FEAC12243EA5151C5
:1028B0004FEA1C5018BF00F5F0404FEA300018BF37
:1028C00041F000415FEA6C5C00F02980BCF1FF3F01
:1028D00008BF40F080407047130C06BF12044FF051
:1028E000100C4FF0000C130E04BF12020CF1080C78
:1028F000130F04BF12010CF1040C930F04BF9200DC
:102900000CF1020CD30F04BF52000CF1010C114664
:102910004FF00002A0F11F00A0EB0C00704711F077
:10292000004F08BF704731F000413FF4D5AF0B0CAA
:1029300006BF09044FF0100C4FF0000C0B0E04BF43
:1029400009020CF1080C0B0F04BF09010CF1040C77
:102950008B0F04BF89000CF1020CCB0F04BF4900A0
:102960000CF1010CCCF12003A0EB0C0022FA03F3D4
:1029700002FA0CF241EA030100F10100704720F075
:102980007F4C80EA030023F07F47ACEB070303F59D
:102990007C5300F0004003F1FF032DE980494FEA2A
:1029A000154B09B44FEA144325EA0B4E24EA0348B9
:1029B0000FF2042606EB132749083E785FEA32023D
:1029C00003FB0667C7F5000707FB06F64FEA543717
:1029D0004FEAD64606F1020607FB066CCCF1005C16
:1029E0004FEA1C472CEA074C07FB06F40CFB06F5E4
:1029F00004EB15464FEA961634BF00204FF0004016
:102A00004FEAD13706FB07FC4FEA1C4C0CFB0BF7D7
:102A1000D21B03FB0CF761EB07010CFB0EF7B0EBCD
:102A2000074072EB17420CFB08F734BFA2EB0742DA
:102A3000B2EB074261EB17414FEA0C444FEA9107B2
:102A400006FB07FC4FEA1C4C0CFB0BF7B0EBC74036
:102A500072EB573203FB0CF734BFA2EBC742B2EB69
:102A6000C74261EB57310CFB0EF7B0EBC70072EBBE
:102A700057720CFB08F734BFA2EBC702B2EBC702D8
:102A800061EB5771039F4FEA816141EA921104EBB8
:102A9000CC044FEAD1374FEA826206FB07FC42EAD8
:102AA00090124FEA80604FEA1C4C0CFB0BF7D21BD4
:102AB00003FB0CF761EB07010CFB0EF7B0EB0740D3
:102AC00072EB17420CFB08F734BFA2EB0742B2EBE4
:102AD000074261EB17414FEA8C554FEA910704EB2F
:102AE0009C2406FB07FC4FEA1C4C0CFB0BF7B0EBDD
:102AF000C74072EB573203FB0CF734BFA2EBC7425F
:102B0000B2EBC74261EB57310CFB0EF7B0EBC700DD
:102B100072EB57720CFB08F734BFA2EBC702B2EBA3
:102B2000C70261EB577115EB4C254FEA816141EA11
:102B300092114FEA82624FEAD13742EA901206FBC5
:102B400007FC44F100044FEA80604FEA1C4C0CFB88
:102B50000BF7D21B03FB0CF761EB07010CFB0EF725
:102B6000B0EB074072EB17420CFB08F734BFA2EB47
:102B70000742B2EB074261EB174115EB1C154FEA18
:102B8000813141EA92414FEA823242EA90424FEA71
:102B900080304FEA0C7644F1000448EA03434EEAE1
:102BA0000B484FF0000EB2EB080C71EB030724BF8B
:102BB000624639464EEB0E0E4FF0000B00185241A4
:102BC00049414BEB0B0BB2EB080C71EB03077BF1AC
:102BD000000B24BF624639464EEB0E0E4FF0000B41
:102BE0000018524149414BEB0B0BB2EB080C71EB57
:102BF00003077BF1000B24BF624639464EEB0E0EF5
:102C000051EA020718BF46F0010616EB0E7655F1A1
:102C1000000254F1000103D5BDE88901BDE8008838
:102C2000BDE88901BDE80048B619524141EB0101F8
:102C3000A3F10103704780807F7E7D7C7B7A797869
:102C4000777676757473727171706F6E6E6D6C6C71
:102C50006B6A6A6968686766666564646363626113
:102C60006160605F5F5E5E5D5D5C5C5B5B5A5A5994
:102C70005958585757565655555554545353525200
:102C80005251515050504F4F4F4E4E4D4D4D4C4C58
:102C90004C4B4B4B4A4A4A494949484848474747A1
:102CA00047464646454545444444444343434342DE
:102CB000424242414141000046EA0646A3F57053B4
:102CC0004FEA164646EA42564FEAD22242EA4152BB
:102CD00010B54FEAD121A3F1010300F02FF820F045
:102CE000004000F1020C00F0004701EB00501146DB
:102CF000BCF5006F40EA070000D210BDBAF1000F2A
:102D00000AD01CB503B44FF004004FF004014FF09B
:102D100000000FBCBDE810404FF00001BBF1010FF7
:102D2000B9BF04484FF0FF310348002140EA0700D3
:102D300010BD00BFFFFFEF7F0000F07F002B9C461F
:102D400030D477002BD01CB54FEA370703B44FF0CF
:102D500010004FF01001BAF1000F06D0BCF1000FC7
:102D6000DCBF40F0080040F008014FF000000FBC4D
:102D7000BDE810400BF1010BBBF1010F08BF5FEA8A
:102D8000170722BF12F1010211F101014FF00041BA
:102D900043F1000300F0004043EA00007047F9D31C
:102DA0005708D0E746EA064613F1400F4FEA1646A9
:102DB0001FDD13F1200FDFBF16430A460021203329
:102DC0005B42BED0C3F1200746EA064602FA07F787
:102DD0004FEA164646EA0706C3F1200722FA03F235
:102DE00001FA07F721FA03F14FF0000342EA070264
:102DF000A7E746EA020646EA06464FEA164646EACC
:102E00000106BCBF46EA0646360C4FF000034FF001
:102E100000024FF0000194E72DE9804C9A4693465A
:102E200070B491E8380007C831EA400C48BF34EA72
:102E3000430C03D5FFF7A3FDFFF780FFF0BCBDE80F
:102E4000008C2DE9804C9A46934670B491E8380086
:102E500007C831EA400C48BF34EA430C03D5FFF7FA
:102E60008EFDFFF729FFF0BCBDE8008C2DE9804CFA
:102E70009A46934670B491E8380007C810F0804F26
:102E800008BF13F0804F03D100F01AF8FFF756FF88
:102E9000F0BCBDE8008C2DE9804C9A46934670B496
:102EA00091E8380007C810F0804F08BF13F0804F3A
:102EB00003D100F005F8FFF7FFFEF0BCBDE8008C81
:102EC00020F07F4780EA030023F07F4C07EB0C03E0
:102ED000A3F57C5300F00040A3F1FE0392F0000F35
:102EE00000F0B38095F0000F00F077802DE90149E4
:102EF0004FEA11404FEA144621EA004800FB06FC65
:102F000024EA064708FB06F607FB08F800FB07F76C
:102F100018EB06484CEB164C4FEA124B18EB0748DF
:102F20004FEA15464CEB174022EA0B4E0BFB06FC12
:102F300025EA06470EFB06F607FB0EFE0BFB07F71E
:102F40001EEB064E4CEB164C4FF000061EEB074EE8
:102F50004CEB174B18EB0B0840F1000018EB0E0B75
:102F600058EB000840F100008F1A4FF000013CBF01
:102F7000C943661B14BFB5EB040C00213CBFC94319
:102F8000F61B4FEA17444EEA8E0E27EA04454FEA35
:102F90001C4704FB07622CEA074C05FB07F70CFBF8
:102FA00005F604FB0CFC16EB074642EB174216EB4A
:102FB0000C4642EB1C421BEB060658EB0202414159
:102FC00046EA9E0601D5BDE80189B619524141EB9A
:102FD0000101A3F10103BDE801894FEA14454FEA5D
:102FE000114724EA054621EA074C05FB07F406FBD6
:102FF00007F70CFB06F105FB0CFC11EB074144EB5A
:1030000017444FEA124711EB0C4144EB1C4422EAEF
:10301000074C05FB07F206FB07F70CFB06F605FB62
:103020000CFC16EB074642EB174216EB0C4642EB44
:103030001C456A1854F1000148BF7047B619524147
:1030400041EB0101A3F10103704795F0000F37D068
:103050004FEA11424FEA144721EA024624EA074C9C
:1030600002FB07F106FB07F70CFB06F402FB0CFC66
:1030700014EB074441EB17414FEA154714EB0C449E
:1030800041EB1C4125EA074C02FB07F506FB07F75D
:103090000CFB06F602FB0CFC16EB074645EB17454E
:1030A00016EB0C4645EB1C42121951F1000148BFCA
:1030B0007047B619524141EB0101A3F1010370477A
:1030C0004FEA14454FEA114724EA054621EA074C26
:1030D00005FB07F106FB07F70CFB06F24FF00006B5
:1030E00005FB0CFC12EB074241EB174112EB0C42C3
:1030F00051EB1C4148BF7047921841EB0101A3F10D
:103100000103704721484FF0FF010170002080F358
:1031100009881F48016881F308881E484FF08051D4
:10312000016062B6FEE71B484FF0805101607047B6
:1031300018484FF080510160704772B6EFF3098074
:1031400050B11EF0100F08BF20ED108A734620E921
:10315000F80F11490968086000B5104880475DF80C
:1031600004EB0F480F490A7802700B480E490A68B1
:1031700002601068B0E8F80F9E461EF0100F08BFFE
:10318000B0EC108A80F3098862B6704722ED00E047
:10319000B807002004ED00E0B00700201584000807
:1031A0009A0700209B070020B407002010B503F009
:1031B0000DFD4E48007958BB01204D4908704FF471
:1031C0007A71022003F000FD002048494872084649
:1031D00090F8AD00A8B104F04BFB4448B0F8C8002B
:1031E00000F4807010B904F083FC7DE09FED410A8B
:1031F000414880ED010A9FED3F0A404880ED010AF9
:1032000072E00CF017FB0FF0A7FA0CF0F3FB6BE089
:103210003748007880B13A48806904280CD10020F2
:10322000334908709FED330A364880ED070A9FED59
:10323000310A334880ED070A2C481A300EF032FF6D
:103240002A4890F8260010B110F024FC01E006F0A6
:103250009BFD2649D1F8C8000BF03AFCB8B12348D1
:1032600020300CF08FFB0FF071FA204991ED000A2D
:10327000BDEEC00A10EE100A0EF04CFA00EE100A75
:10328000B8EEC00A194880ED000A0CF00BFA174896
:10329000D0F8C800B0F5007F04D01448D0F8C800BA
:1032A000402803D10FF052FA0CF0C4FA0F4890F8FE
:1032B000DB0048B103F0D0FF0C48B0F8C80000F4C0
:1032C000807008B904F08CF9084890F8DA0058B119
:1032D00004F0CEFA0548B0F8C80000F4807008B9D0
:1032E00004F006FC0FF032FA10BD0000641F02204B
:1032F0003C0300200000000018170120681701207F
:1033000090170120401701200246642A04D10123AE
:10331000324880F8AF3003E00023304880F8AF3007
:10332000752A04D101232D4880F8AE3003E0002334
:103330002A4880F8AE30652A03D0642A01D0752A65
:1033400001D100207047662A03D1612901D10320F1
:10335000F8E7662A03D1632901D10420F2E7662A3F
:1033600003D16D2901D10120ECE7622A03D1612943
:1033700001D10520E6E7622A03D1632901D10620A5
:10338000E0E7622A03D16D2901D10220DAE7662A3B
:1033900003D16C2901D10720D4E7622A03D16C291B
:1033A00001D10920CEE7662A03D1722901D1082074
:1033B000C8E7622A03D1722901D10A20C2E7462A4E
:1033C00003D16D2901D10B20BCE7422A03D16D291D
:1033D00001D10C20B6E70020B4E70000641F0220F2
:1033E00010B502460B460021002000BF04E0545CEB
:1033F0000444A0B24C1CA1B29942F8DB10BD0000FD
:1034000008B52EE01748407F18B10121164806F094
:103410002DFA1448817F807F401E124A90770A2936
:1034200002DA0020114648771048407F18B1012188
:103430000F4806F03DFB0D48817F807F401E0B4A00
:1034400090770A2906DA0020114648772421104691
:10345000FDF794FB09F0E4F96A460821022004F024
:10346000DBFFCFE728160120000E01204C160120BB
:10347000780E012010B58AB004463E480078052831
:1034800017D109A8032100220592CDE90621089051
:1034900010464FF480711922374BCDE90132CDE946
:1034A000031002200023354A35A10090394804F06A
:1034B00003FE09A8032100220592CDE90621089008
:1034C00010464FF40061CC22334BCDE90132CDE9F7
:1034D00003100A200023314A31A10090364804F03D
:1034E000EBFD09A8072100220592CDE906210890ED
:1034F00010464FF40061CC22304BCDE90132CDE9CA
:103500000310042000232E4A2EA10090314804F01D
:10351000D3FD09A8032100220592CDE906210890D8
:1035200010464FF40061CC222B4BCDE90132CDE99E
:10353000031008200023294A29A100902E4804F0F6
:10354000BBFD032000210591CDE907040691084643
:103550004FF40061CC22294BCDE90132CDE90310B3
:1035600005200023264A27A100902B4804F0A4FD43
:103570000AB010BD98010020502D002055360008DB
:10358000417070205461736B2046656564446F67B9
:1035900000000000E82C0020B83100203D36000873
:1035A000417070205461736B2045746865726E655C
:1035B000742053657200000050310020F09200200A
:1035C00001340008417070205461736B2043414EF8
:1035D0000000000088920020205200201D360008C4
:1035E000417070205461736B2045746865726E651C
:1035F0007420436C69000000B851002058B30020CB
:103600006D360008417070205461736B20537065F3
:103610006564204374720000F0B2002008B509E030
:103620000BF074FB0449C1F814016A46082101201B
:1036300004F0F2FEF4E70000641F022008B507F072
:1036400037FD06E00CF0ACFB6A4608210A2004F0C6
:10365000E3FEF7E708B50BF07FFB06E002F03EF96A
:103660006A4600210A2004F0D7FEF7E708B50AE011
:1036700008F07CFB09F02AF908F08CFB6A46082167
:103680000A2004F0C9FEF3E710B52DED048B3B488A
:1036900090F82700012804D100F088F8BDEC048BD5
:1036A00010BD374890ED000AB8EEC00A3548D0ED9D
:1036B000000AB4EE600AF1EE10FA5CD1304890EDE9
:1036C000010AB8EEC00A2F48D0ED010AB4EE600A34
:1036D000F1EE10FA4FD12948817E2B484068401EF8
:1036E000814223DB254890F8200002281ED124487F
:1036F00090ED020A10EE101A084611F0E9FC41ECB8
:10370000190BB0EE490AF0EE690A09F059FCB0EE67
:10371000408AF0EE608A9FED1D0B53EC102B51ECAC
:10372000180B11F0A3F926D20120B7E7144890ED49
:10373000020A10EE101A084611F0CAFC41EC190BEF
:10374000B0EE490AF0EE690A09F03AFCB0EE408AA0
:10375000F0EE608A9FED0F0B53EC102B51EC180B21
:1037600011F084F907D20548C27E0CA1012008F0AF
:10377000FBFA012092E7002090E70000641F02207E
:103780002816012038210220C06D01200000000011
:10379000000024400000000000002E40D5FDB3A32F
:1037A000B5BDB4EF202025640D0A000010B54A48CD
:1037B00090ED060ADFED490AB4EEE00AF1EE10FAE8
:1037C0007CD24748C07E01283ED1454890F8C400CD
:1037D000012805D14348007810B90120424908600A
:1037E00041480068012807D13D48C27E3FA1012021
:1037F00008F0BAFA012010BD394890F8C40060B949
:10380000354890ED060ADFED3E0AB4EEE00AF1EE2F
:1038100010FA02D2012180F82C102F4890F82C00C9
:1038200000284CD02C4890ED060ADFED360AB4EEA5
:10383000E00AF1EE10FA42DD2948C27E32A10120F1
:1038400008F092FA0120D6E72548C07E012816D15B
:10385000234890F8C500012805D13148007810B9F7
:103860000120304908602F480068012827D11C48F2
:10387000C27E2DA1012008F077FA0120BBE716488F
:1038800090ED070AD0ED050AB2EE041A70EEC10AF7
:10389000B4EEE00AF1EE10FA11DB90ED060AD0ED7D
:1038A000070AB4EEE00AF1EE10FA08D20C48C27E24
:1038B00022A1012008F058FA01209CE709E00848FD
:1038C00090F8C40007490870054890F8C5001449ED
:1038D000087000208FE7000094200220000096432B
:1038E000641F0220F11D0020E81D0020D7F3B9E27B
:1038F000B5E7B5BDB4EF202025640D0A0000000037
:10390000000048420000C842CEB4C9A8B5BDB9E223
:10391000B5E7B5BDB4EF202025640D0A0000000016
:10392000F21D0020EC1D0020D3D2B9E2B5E7B5BDF1
:10393000B4EF202025640D0A00000000D5FDB3A3DC
:10394000B5BDB4EF202025640D0A00001FB5684600
:1039500006F060FA019804B010BD00002DE9F041B6
:10396000FFF7F4FF054614480068B5FBF0F4214664
:10397000481EB0F1807F00D31BE0481E4FF0E022CC
:10398000506150170F22002807DA13071F0E0B4B48
:1039900000F00F06361F9F5503E013071E0E084B5D
:1039A0001E5400BF00204FF0E022906107201061FC
:1039B00000BFBDE8F08100003053010818ED00E0C1
:1039C00000E400E038B50025404890F83E0E082895
:1039D0003DD008DC01280FD002280ED0032815D0D6
:1039E000042870D129E00B2830D020285BD0212872
:1039F00049D0272867D13DE065E035480223012200
:103A000000210090084601F0D5FE5CE03048032319
:103A1000012200210090084601F0CCFE2D48D0F88C
:103A2000C8102DA005F076FB04460623002211469F
:103A30000090012001F0BEFE45E02548042301224C
:103A400000210090084601F0B5FE3CE03BE01F4835
:103A5000D0F8400E10B1012802D100E000E000BF14
:103A600000BF1B480823012202210090002001F022
:103A7000A1FE28E0164827230122002100900846D5
:103A800001F098FE1FE0124821230122002100903E
:103A9000084601F08FFE124A51680C4AD2F8400ED7
:103AA0000CF01AF80FE00A482023012200210090B0
:103AB000084601F07FFE0A4A5168044AD2F8400ED7
:103AC0000CF0A4F800BF00BF38BD0000D0020220F7
:103AD00030090220641F02202530347800000000E5
:103AE0001011022000BFFEE730B58BB004460D4632
:103AF0000121084606F05EF90121480606F06AF940
:103B00004FF4C050099002208DF8280000208DF855
:103B10002A0003208DF8290001208DF82B0009A927
:103B2000534801F0EDFE09220B21514801F030FF0E
:103B300009220C214E4801F02BFF00208DF81E00B9
:103B400001208DF81F0000208DF820008DF8210045
:103B50008DF822008DF823008DF81A50052C45D2DF
:103B6000DFE804F003101D2A370000208DF81B0049
:103B700006208DF81C0005208DF81D001E20ADF8D4
:103B8000180040E000208DF81B0006208DF81C0076
:103B900005208DF81D001820ADF8180033E0002036
:103BA0008DF81B0006208DF81C0005208DF81D00E7
:103BB0000F20ADF8180026E000208DF81B0006202D
:103BC0008DF81C0005208DF81D000C20ADF81800A4
:103BD00019E000208DF81B0006208DF81C00052040
:103BE0008DF81D000620ADF818000CE000208DF8BF
:103BF0001B0006208DF81C0005208DF81D000620F6
:103C0000ADF8180000BF00BF06A91A4800F03BFC41
:103C100000208DF812008DF8130001208DF814009B
:103C20000020ADF80800ADF80A00ADF80C00ADF8C2
:103C30000E00ADF8100001208DF8150002A800F06C
:103C400005FB012202210B4800F014FC14208DF822
:103C5000040001208DF8050000208DF806000120E9
:103C60008DF8070001A804F05FF800200BB030BD0C
:103C7000000002400064004030B585B000250024FB
:103C800000BF00BFFCF76CFB044600BF00BF04F0A0
:103C90001DF900BF00BF2046FCF766FB00BF00BF58
:103CA00002212B4800F056FB00284AD06A4600212A
:103CB000274800F072FC40F281110098884202D13E
:103CC000684608F0E3F940F283110098884202D177
:103CD000684608F053FA0098B0F5C17F02D16846F3
:103CE00008F0FEF90098B0F5C27F02D1684608F0EE
:103CF0006FFA40F285110098884202D1684608F0B8
:103D0000B5FA40F281310098884202D1684608F045
:103D1000D7FA40F283310098884202D1684608F011
:103D200005FB40F282410098884202D1684608F0C3
:103D30005DF940F284410098884202D1684608F05B
:103D40007DF900200090019004F0D6F805B030BD58
:103D5000006400402DE9F04786B0074688461646C5
:103D600099464FF0140A0025009712200190002078
:103D70008DF808008DF809008DF80A6000BF05E095
:103D800018F805100DF10B0041556D1CB542F7D325
:103D90001DE06946134800F078FC0446042C0FD05F
:103DA00006E05046411E01F0FF0A012800DA05E056
:103DB00021460C4800F0FCFC0028F2D000BF07E0D0
:103DC0005046411E01F0FF0A012800DA00E0E0E75A
:103DD00000BF05AA0821484604F01EFB002006B0DB
:103DE000BDE8F0870064004010B5002400BF00BFAC
:103DF000FCF7B6FA044600BF00BF04F067F800BF46
:103E000000BF2046FCF7B0FA00BF00BF01211548F3
:103E100000F0C8F90121134800F09CFA012804D1F0
:103E20000121104800F0BEF914E001210D4800F016
:103E300091FA012804D101210A4800F0B3F909E000
:103E40000121084800F086FA012803D10121054824
:103E500000F0A8F900220121024800F00BFB04F059
:103E60004BF810BD0064004030B58BB004460D46E1
:103E70000121022005F09EFF01214FF0C06005F0F6
:103E8000A9FF6020099002208DF8280000208DF8FD
:103E90002A0003208DF8290001208DF82B0009A9A4
:103EA000544801F02DFD09220521524801F070FD12
:103EB000092206214F4801F06BFD00208DF81E00FD
:103EC00001208DF81F0000208DF820008DF82100C2
:103ED0008DF822008DF823008DF81A50052C45D25C
:103EE000DFE804F003101D2A370000208DF81B00C6
:103EF00006208DF81C0005208DF81D001E20ADF851
:103F0000180040E000208DF81B0006208DF81C00F2
:103F100005208DF81D001820ADF8180033E00020B2
:103F20008DF81B0006208DF81C0005208DF81D0063
:103F30000F20ADF8180026E000208DF81B000620A9
:103F40008DF81C0005208DF81D000C20ADF8180020
:103F500019E000208DF81B0006208DF81C000520BC
:103F60008DF81D000620ADF818000CE000208DF83B
:103F70001B0006208DF81C0005208DF81D00062072
:103F8000ADF8180000BF00BF06A91B4800F07BFA7F
:103F90000E208DF8120000208DF8130001208DF8FE
:103FA00014000020ADF80800ADF80A00ADF80C00D0
:103FB000ADF80E00ADF8100001208DF8150002A834
:103FC00000F044F9012202210B4800F053FA40208E
:103FD0008DF8040001208DF8050000208DF8060002
:103FE00001208DF8070001A803F09EFE00200BB011
:103FF00030BD0000000402400068004030B585B0CC
:104000000025002400BF00BFFCF7AAF9044600BF4A
:1040100000BF03F05BFF00BF00BF2046FCF7A4F920
:1040200000BF00BF0221184800F094F920B36A468F
:104030000021154800F0B1FA0098B0F5007F0CD1CE
:104040009DF80C009DF80B1040EA012000EE100ACC
:10405000B8EEC00A0D4880ED430A40F201210098F5
:10406000884208D19DF812109DF8110041EA002104
:104070000648C0F8101100BF00200090019003F026
:104080003BFF05B030BD000000680040641F022007
:104090002DE9F04786B007468846164699464FF008
:1040A000140A002500971220019000208DF80800C6
:1040B0008DF809008DF80A6000BF05E018F80510BA
:1040C0000DF10B0041556D1CB542F7D31DE069465B
:1040D000134800F0DAFA0446042C0FD006E05046EC
:1040E000411E01F0FF0A012800DA05E021460C48D4
:1040F00000F05EFB0028F2D000BF07E05046411EF2
:1041000001F0FF0A012800DA00E0E0E700BF05AA9D
:104110000821484604F080F9002006B0BDE8F08789
:104120000068004010B5002400BF00BFFCF718F97C
:10413000044600BF00BF03F0C9FE00BF00BF204619
:10414000FCF712F900BF00BF0121154800F02AF862
:104150000121134800F0FEF8012804D10121104884
:1041600000F020F814E001210D4800F0F3F80128D8
:1041700004D101210A4800F015F809E0012108489E
:1041800000F0E8F8012803D10121054800F00AF801
:1041900000220121024800F06DF903F0ADFE10BDD0
:1041A00000680040B1F5007F3AD00FDC202928D00C
:1041B00006DC01291CD004291DD0082940D11DE0AE
:1041C000402921D0B1F5807F3AD126E0B1F5004FEA
:1041D00031D006DCB1F5806F25D0B1F5006F2FD15D
:1041E00024E0B1F5803F12D0B1F5003F28D111E0B5
:1041F000154A826025E00822C26022E01022C260D7
:104200001FE0082202611CE01022026119E008226E
:10421000426016E01022426013E00422426010E087
:10422000042242600DE0042242600AE00022826122
:104230000422426005E0002282610422426000E024
:1042400000BF00BF704700000101010010B5002150
:10425000837A012202FA03F13D4A126842F0010218
:104260003B4B1A603A4A1C3212688A43384B1C3363
:104270001A60027BCAB9364A0C3212688A43344B40
:104280000C331A604288C38842EA0343304A403202
:10429000847A42F834300288838842EA03432C4A05
:1042A0004032847A02EBC4025360027B012A19D1A6
:1042B000274A0C3212680A43254B0C331A60428895
:1042C000038842EA0343224A4032847A42F8343077
:1042D000C288838842EA03431D4A4032847A02EB53
:1042E000C4025360C27A3AB9194A121D12688A434D
:1042F000174B1B1D1A6006E0154A121D12680A436F
:10430000134B1B1D1A60028932B9114A143212680C
:104310008A430F4B14331A600289012A06D10C4AD2
:10432000143212680A430A4B14331A60427B012A82
:1043300006D1074A1C3212680A43054B1C331A6027
:10434000034A126822F00102014B1A6010BD0000FE
:104350000066004070B504460D460026606928409E
:10436000002871D0B5F5807F5CD010DC082D35D0E9
:1043700006DC012D20D0022D24D0042D72D127E09F
:10438000102D31D0202D35D0402D6BD138E0B5F532
:10439000004F60D009DCB5F5007F49D0B5F5806FDE
:1043A0004CD0B5F5006F5DD14FE0B5F5803F2DD015
:1043B000B5F5003F56D12FE0A0682D4901F086F9F0
:1043C000064651E0E068032101F080F906464BE023
:1043D000E068082101F07AF9064645E0E06810211E
:1043E00001F074F906463FE02069032101F06EF9FF
:1043F000064639E02069082101F068F9064633E0F5
:104400002069102101F062F906462DE0606808215C
:1044100001F05CF9064627E06068102101F056F9CA
:10442000064621E0A069012101F050F906461BE093
:10443000A069022101F04AF9064615E0A0690421AD
:1044400001F044F906460FE00FE0A069702101F089
:104450003DF9064608E06068042101F037F9064698
:1044600002E0FFE7002600BF00E00026304670BDF6
:10447000010101001AB143690B43436102E0436942
:104480008B434361704730B5024600200023146817
:1044900024F002041460146844F00104146000E085
:1044A0005B1C546804F001041CB94FF6FF74A3426E
:1044B000F6D1546804F001040CB900206CE08C794A
:1044C000012C04D1146844F08004146003E01468E3
:1044D00024F080041460CC79012C04D1146844F0D9
:1044E0004004146003E0146824F0400414600C7A63
:1044F000012C04D1146844F02004146003E0146813
:1045000024F0200414604C7A012C04D1146844F087
:104510001004146003E0146824F0100414608C7A12
:10452000012C04D1146844F00804146003E01468FA
:1045300024F008041460CC7A012C04D1146844F0EF
:104540000404146003E0146824F0040414608C78FC
:10455000A407CD7844EA05640D7944EA05444D7911
:1045600044EA05540D886D1E2C43D461146824F070
:1045700001041460002300E05B1C546804F0010493
:104580001CB14FF6FF74A342F6D1546804F0010445
:104590000CB1002000E0012030BD10B500F5D8734B
:1045A00003EB01131B6803F004031372137A53B96E
:1045B00000F5D87303EB01131B6840F2FF7404EAA3
:1045C0005353136009E000F5D87303EB01131B6824
:1045D0006FF0604404EAD303536000F5D87303EB33
:1045E00001131B6803F00203537200F5D87303EB49
:1045F00001135B6803F00F03937200F5D87303EBAC
:1046000001135B681B0AD37400F5D87303EB011325
:104610009B68D37200F5D87303EB01139B681C0AE7
:10462000147300F5D87303EB01139B681C0C5473CF
:1046300000F5D87303EB01139B681B0E937300F511
:10464000D87303EB0113DB68D37300F5D87303EB66
:104650000113DB681C0A147400F5D87303EB011313
:10466000DB681C0C547400F5D87303EB0113DB6892
:104670001B0E937421B9C36843F02003C36003E0A9
:10468000036943F02003036110BD10B5024600200A
:10469000936803F08063B3F1806F00D110E09368FA
:1046A00003F00063B3F1006F01D1012008E09368CB
:1046B00003F08053B3F1805F01D1022000E00420B9
:1046C000042874D002F5C07303EB00131B6803F0D9
:1046D000010402F5C07303EB00131C600B7A7BB975
:1046E0004B7A0C8843EA445302F5C07404EB00147F
:1046F0002468234302F5C07404EB0014236010E027
:104700000B7A4C6843EAC4034C7A234302F5C07425
:1047100004EB00142468234302F5C07404EB001476
:1047200023608B7A03F00F038B7202F5C07303EBE7
:1047300000135B6823F00F0402F5C07303EB001352
:104740005C6002F5C07303EB00135B688C7A234353
:1047500002F5C07404EB001463608B7B1C064B7B7A
:1047600044EA03440B7B44EA0323CC7A234302F557
:10477000C07404EB0014A3608B7C1C064B7C44EAE1
:1047800003440B7C44EA0323CC7B234302F5C0742F
:1047900004EB0014E36002F5C07303EB00131B6825
:1047A00043F0010402F5C07303EB00131C6010BD5D
:1047B00010B50246002321B1012907D002290FD1EB
:1047C00009E090681D4C00EA04030BE090681C4C63
:1047D00000EA040306E090681A4C00EA040301E0D2
:1047E000002300BF00BF184C181BA34216D007DCE3
:1047F00083B16FF08060184470B1022818D111E0C5
:10480000B0F5007F10D0114C204448B1B0F5003F06
:104810000ED10BE002230DE000230BE0002309E0A2
:10482000002307E0012305E0012303E0012301E069
:10483000002300BF00BFD8B210BD00000300000479
:104840000003000800000310000100080001FFF74A
:1048500010B500F01FF800F019F810BD10B50024D5
:1048600000BF00BFFBF77CFD044600BF00BF102166
:10487000054803F0EBF900BF00BF2046FBF774FDCD
:1048800000BF00BF10BD000058D3002010B5FFF7D7
:10489000E5FF10BD10B500200249086000F00AF8DD
:1048A00010BD00008C07002001490860704700001F
:1048B0008C07002010B5FFF749F804460848006847
:1048C00040F08070064908600020064948600846AC
:1048D000006840F0010008602046FFF7E5FF10BDCA
:1048E000FCED00E0001000E001494868704700005E
:1048F000001000E010B52DED0A0B2DED108B94B0DB
:104900009DED240A10EE101A084610F0E1FB41EC70
:10491000190B9DED250A10EE101A084610F0D8FB71
:1049200041EC1A0B9DED270A10EE101A084610F004
:10493000CFFB41EC1B0B9DED280A10EE101A084628
:1049400010F0C6FB41EC1C0B9DED2A0A10EE101A6C
:10495000084610F0BDFB41EC1D0B9DED2B0A10EE3F
:10496000101A084610F0B4FB41EC1E0B53EC1C2B44
:1049700051EC1A0B10F0C2FA9FED9F1BCDE9040118
:104980009DED040B08F090FB8DED080B53EC1B2BF9
:1049900051EC190B10F0B2FA9FED971BCDE9040111
:1049A0009DED040B08F080FB8DED060B9DED080BD3
:1049B00053EC102B9DED060B51EC100B0FF0ACFDE2
:1049C000CDE90E019DED0E0B09F0FAF98DED0C0B02
:1049D00053EC1E2B51EC1A0B10F090FA9FED861B36
:1049E000CDE904019DED040B08F05EFB8DED080B95
:1049F00053EC1D2B51EC190B10F080FA9FED7E1B30
:104A0000CDE904019DED040B08F04EFB8DED060B86
:104A10009DED080B53EC102B9DED060B51EC100B8C
:104A20000FF07AFDCDE90E019DED0E0B09F0C8F9EE
:104A30008DED0A0B53EC1E2B51EC1C0B10F05EFAA3
:104A40009FED6D1BCDE904019DED040B08F02CFBDF
:104A50008DED080B53EC1D2B51EC1B0B10F04EFA97
:104A60009FED651BCDE904019DED040B08F01CFBD7
:104A70008DED060B9DED080B53EC102B9DED060BF9
:104A800051EC100B0FF048FDCDE90E019DED0E0B22
:104A900009F096F9B0EE40FAF0EE60FA9DED0A0BDF
:104AA00053EC102B9DED0C0B51EC100B0FF034FD63
:104AB00053EC1F2BCDE906019DED060B51EC100BBD
:104AC0000FF02AFD9FED4C0B53EC102BCDE90801A4
:104AD0009DED080B51EC100B0FF0DAFD41EC180BBB
:104AE00053EC1F2B51EC180B10F008FACDE908011C
:104AF0009DED0A0B53EC102B51EC180B10F0FEF946
:104B0000CDE904019DED0C0B53EC102B51EC180B6F
:104B100010F0F4F953EC182BCDE900019DED000BDA
:104B200051EC100B0FF0DEFFCDE902019DED040BFF
:104B300053EC102B9DED020B51EC100B0FF0D2FF3C
:104B4000CDE906019DED080B53EC102B9DED060BF6
:104B500051EC100B0FF0C6FFCDE90E019DED0E0BD1
:104B600009F02EF98DED100B53EC1F2B9FED220B4E
:104B700051EC100B0FF08CFDCDE908019DED100BF1
:104B800053EC102B9DED080B51EC100B0FF0AAFF0E
:104B9000CDE91201B0EE4E5AF0EE6E5AB0EE4D4A2B
:104BA000F0EE6D4AB0EE4C3AF0EE6C3AB0EE4B2AB5
:104BB000F0EE6B2AB0EE4A1AF0EE6A1AB0EE490A2D
:104BC000F0EE690A04F0BAFA044620460FF023FF1B
:104BD000CDE908019DED120B53EC102B9DED080B58
:104BE00051EC100B0FF07EFF41EC100B14B0BDEC3C
:104BF000108B0AB010BD0000000000000000004053
:104C0000F0EE400A9FED3D0AF4EEC00AF1EE10FA14
:104C100005DD9FED3B0A30EEC00AF0EE400A9FED45
:104C2000390AF4EEC00AF1EE10FA05D29FED340A0B
:104C300030EE800AF0EE400AB2EE040AF4EEC00A4A
:104C4000F1EE10FA0CD2BAEE040AF4EEC00AF1EE5C
:104C500010FA05DD9FED2C0A2C4880ED000A48E093
:104C60009FED2B0AF4EEC00AF1EE10FA0CD29FED84
:104C7000290AF4EEC00AF1EE10FA05DD9FED260ACE
:104C8000224880ED000A34E09FED240AF4EEC00AC9
:104C9000F1EE10FA06D29FED1B0AF4EEC00AF1EE17
:104CA00010FA0DDA9FED1E0AF4EEC00AF1EE10FACA
:104CB0000CDD9FED120AF4EEC00AF1EE10FA05D8F1
:104CC0009FED0E0A114880ED000A12E09FED150AD3
:104CD000F4EEC00AF1EE10FA0BD29FED130AF4EED7
:104CE000C00AF1EE10FA04DD9FED100A074880EDCE
:104CF000000A064890ED000A7047000000003443A7
:104D00000000B443000034C300000000A8210020CC
:104D10000000C8420000A0420000B44200002AC3C4
:104D200000002A430000A0C20000C8C20000B4C2B4
:104D300010B52DED0A8BB0EE408AF0EE608A38EEA9
:104D4000680A10EE101A084610F0C2F941EC1A0B6E
:104D5000B0EE4A0AF0EE6A0A08F032F9B0EE409A74
:104D6000F0EE609A9FED2A0B53EC102B51EC190BCF
:104D70000FF0B6FF2DD238EE680A10EE101A084672
:104D800010F0A6F941EC1C0BB0EE4C0AF0EE6C0AE8
:104D900008F016F9B0EE40BAF0EE60BA9FED1E0BC7
:104DA00053EC102B51EC1B0B10F0A8F841EC1A0B34
:104DB000B0EE4A0AF0EE6A0A08F002F9B0EE409A44
:104DC000F0EE609A51EC190B0FF074FB1449086077
:104DD00018E038EE680A10EE101A084610F078F95C
:104DE00041EC1A0BB0EE4A0AF0EE6A0A08F0E8F855
:104DF000B0EE409AF0EE609A51EC190B0FF05AFBAE
:104E000007490860064890ED000ABDEC0A8B10BD0A
:104E10000000000000806640000000000080764036
:104E2000A421002010B52DED0A8B7448D0ED022A84
:104E300090ED012AD0ED001A714890ED021AD0EDE4
:104E4000010A90ED000A06F023FA6E4880ED030A8D
:104E50006D4890ED024AD0ED013A90ED003A684875
:104E6000D0ED022A90ED012AD0ED001A634890EDB2
:104E7000021AD0ED010A90ED000AFFF73BFDB0EEFB
:104E8000409AF0EE609A51EC190B0FF007FB41ECE1
:104E9000180B0FF00FFB5B494860084690ED010AC4
:104EA00010EE101A084610F013F941EC1C0B9FEDA0
:104EB000571BB0EE4C0AF0EE6C0A08F0F5F8B0EEB5
:104EC00040AAF0EE60AA4F4890ED030A10EE101AC7
:104ED000084610F0FDF841EC1C0B9FED4C1BB0EEAA
:104EE0004C0AF0EE6C0A08F0DFF8B0EE40BAF0EED3
:104EF00060BA53EC1A2B51EC1B0B0FF0FFFF41EC87
:104F0000190BB0EE490AF0EE690A08F059FFB0EE4D
:104F1000408AF0EE608A51EC180B0FF0CBFA394959
:104F2000C8613948D0ED022A90ED012AD0ED001A6F
:104F3000324890ED021AD0ED010A90ED000A06F019
:104F4000A7F9304880ED040A90ED010A10EE101A1E
:104F5000084610F0BDF841EC1C0B9FED2C1BB0EE89
:104F60004C0AF0EE6C0A08F09FF8B0EE409AF0EEB2
:104F7000609A244890ED040A10EE101A084610F0CA
:104F8000A7F841EC1C0B9FED211BB0EE4C0AF0EE94
:104F90006C0A08F089F8B0EE40BAF0EE60BA53EC53
:104FA000192B51EC1B0B0FF0A9FF41EC180BB0EEC5
:104FB000480AF0EE680A08F003FFB0EE40AAF0EEEF
:104FC00060AA51EC1A0B0FF075FA0E4988610E4871
:104FD000D0ED022A90ED012AD0ED001A084890ED9C
:104FE000021AD0ED010A90ED000A06F051F90548C9
:104FF00080ED050ABDEC0A8B10BD000044210220A3
:105000002C210220942002203821022000000000E0
:105010000000004070B52DED108B8CB0F0EE409A82
:10502000B0EE60FAB0EE419AF0EE61FA05460E4637
:105030001446BE4890F8230030B101280AD0022857
:1050400012D0032824D119E094ED000AB84880ED6D
:10505000000A1EE094ED000ADFEDB60A30EE600AA9
:10506000B34880ED000A14E094ED000ADFEDB20AC7
:1050700030EE600AAE4880ED000A0AE094ED000AC6
:10508000DFEDAC0A30EE200AA94880ED000A00E00E
:1050900000BF00BF1FEE900A10F01AF841EC180B89
:1050A00019EE100A10F014F853EC182BCDE900019A
:1050B0009DED000B51EC100B0FF014FD41EC1E0B9D
:1050C0009FED9E0B53EC102B0FF0E2FA41EC1C0B02
:1050D000974800680FF0FCFF41EC1D0B53EC1C2BB4
:1050E0000FF01AFA41EC1B0BB0EE4B0AF0EE6B0A14
:1050F00008F002FE8DED020B1FEE100A0FF0E8FF24
:1051000041EC1B0B53EC182B0FF0ECFC41EC1A0B91
:105110009DED020B53EC102B0FF0E4FCCDE90601E2
:1051200019EE100A0FF0D4FF53EC182BCDE9000153
:105130009DED000B51EC100B0FF0D4FC9FED7F0B9D
:1051400053EC102BCDE902019DED020B51EC100B3D
:105150000FF09EFA41EC1C0B754800680FF0B8FF89
:1051600041EC1E0B53EC1C2B0FF0D6F941EC1B0B42
:10517000B0EE4B0AF0EE6B0A07F0BEFEB0EE40DA7E
:10518000F0EE60DA19EE900A0FF0A2FF41EC1B0B73
:1051900053EC182B0FF0A6FC41EC1A0B53EC1D2B13
:1051A0000FF0A0FCCDE904019DED060B53EC102B94
:1051B0009DED040B51EC100B0FF0A0FECDE90A01A0
:1051C00019EE100A0FF084FF41EC1C0B53EC182B66
:1051D0000FF088FC41EC1B0B9FED580B53EC102B90
:1051E0000FF056FA41EC1A0B514800680FF070FFAF
:1051F00053EC1A2BCDE900019DED000B51EC100B87
:105200000FF08AF9CDE902019DED020B07F074FE63
:10521000B0EE40DAF0EE60DA1FEE100A0FF058FF41
:1052200041EC1A0B53EC182B0FF05CFC41EC1E0BFD
:1052300053EC1D2B0FF056FCCDE9060119EE100AB8
:105240000FF046FF41EC1C0B53EC182B0FF04AFCFF
:1052500041EC1E0B9FED390B53EC102B0FF018FA9D
:1052600041EC1B0B324800680FF032FF41EC1D0B84
:1052700053EC1B2B0FF050F941EC1A0BB0EE4A0A1D
:10528000F0EE6A0A08F038FD8DED020B19EE900A77
:105290000FF01EFF41EC1A0B53EC182B0FF022FC01
:1052A000CDE900019DED020B53EC102B9DED000BA1
:1052B00051EC100B0FF016FCCDE904019DED060B2F
:1052C00053EC102B9DED040B51EC100B0FF024F957
:1052D000CDE9080195ED000A10EE101A08460FF00E
:1052E000F7FE41EC1B0B9DED0A0B53EC102B0FF05E
:1052F00013F941EC1A0B0FF0DDF8286096ED000A67
:1053000010EE101A08460FF0E3FE41EC1B0B9DED6A
:10531000080B53EC102B0FF0FFF841EC1A0B0FF0B9
:10532000C9F830600CB0BDEC108B70BD641F02205A
:1053300064230020DA0FC93FDA0F49400000000063
:1053400000000040B0EE401ADFED111AB0EE610A25
:1053500071EE601AB0EE610ADFED0E1AB4EEE10AEA
:10536000F1EE10FA05D8DFED0C1A70EE211AB0EE4E
:10537000610ADFED0A1AB4EEE10AF1EE10FA05DB7C
:10538000DFED051A70EE611AB0EE610A7047000099
:1053900000000000DA0F49C0DA0FC940DA0F4940B7
:1053A00010B52DED060B2DED088B9FED2E0AB0EEFE
:1053B000408A9DED080ADDED0B0AB4EE600AF1EEBD
:1053C00010FA1BD19DED0C0ADDED090AB4EEE00ADE
:1053D000F1EE10FA04DD9FED240AB0EE408A3BE0C6
:1053E0009DED0C0ADDED090AB4EEE00AF1EE10FACB
:1053F00032D29FED1E0AB0EE408A2DE09DED0B0AE1
:10540000DDED080A30EE600A10EE101A08460FF0C3
:105410005FFE41EC1A0B9DED0C0ADDED090A30EE42
:10542000600A10EE101A08460FF052FE41EC1B0BFA
:10543000B0EE4A1AF0EE6A1AB0EE4B0AF0EE6B0AC2
:1054400007F062FCB0EE409AF0EE609A51EC190B56
:105450000FF030F808EE100AB0EE480ABDEC088BE9
:1054600006B010BD00000000DA0FC93FDA0FC9BF57
:10547000244890ED000AB8EEC00A2348D0ED030A94
:1054800030EE200A214880ED000A1E4890ED010A06
:10549000B8EEC00A1C48D0ED010A30EE200A1B48C5
:1054A00080ED010A174890ED040A1948D0ED100A62
:1054B00030EE200A154880ED020A90ED020ADFED79
:1054C000150AB4EEE00AF1EE10FA08DD90ED020ADA
:1054D000DFED110A30EE600A80ED020A11E00B48A0
:1054E00090ED020ADFED0D0AB4EEE00AF1EE10FADB
:1054F00007D290ED020ADFED080A30EE200A80EDB7
:10550000020A70472816012094200220442102201C
:10551000641F0220DA0F4940DA0FC940DA0F49C090
:10552000F8B504460E460020009000255D4800783E
:1055300068B94FF4FA615C48FBF720FB00205B4937
:105540000870012057490870002059490880232C11
:105550000FD101205549087056480088401C554914
:10556000088008460088012806D10020504908809C
:1055700002E000204F4908804C480078052873D28B
:10558000DFE800F00311043E050086E000BF4FF4A1
:10559000FA614548FBF7F2FA0120444908700020FF
:1055A0004349088000BF202C0CD041480088B0F54A
:1055B000FA6F07DA3E4801880088401C3C4A108098
:1055C000394844545A2C0DD13B480088401C3A4974
:1055D000088008460088022803D103203349087058
:1055E0000DE05AE000203449088031480088B0F5C9
:1055F000FA6F03DB02202D49087000E04DE000BF88
:105600002B4909880839284A88186A462BA1FBF7D4
:105610007FF827480088083801B22348FDF7E0FEEC
:1056200005460098854204D041F234210098884212
:105630001BD14FF4FA612348FBF7A0FA1A4921481D
:10564000FBF776F94FF4FA611748FBF797FA1D4814
:10565000FBF7A7F91C49C1F8E800002014490880AD
:1056600004201249087018E015E04FF4FA610E4862
:10567000FBF784FA00200E49088002200B490870CD
:10568000232C07D14FF4FA610748FBF777FA002083
:105690000749088001E000BFFEE700BF034800782B
:1056A000F8BD0000622A002020B00120632A0020FB
:1056B000642A0020682A0020662A002025303478D9
:1056C00000000000007B0120201002200246002084
:1056D00002EA01030BB1012000E000207047000046
:1056E00070B5002502212D4880F83C1E302180F83D
:1056F0003E1E2B4800F030FA0546002413E004EB70
:105700008400284A02EB80012748FBF735F905465B
:105710001DB9224880F83C4E07E0022C01D102203E
:1057200070BD601CC4B2032CE9DB00BF002414E090
:1057300004EB84001D4A02EB80011B482838FBF76C
:105740001BF905461DB9154880F83D4E07E0062CAB
:1057500001D10320E4E7601CC4B2072CE8DB00BFE2
:10576000002416E004EB440000EBC400104A02EBF6
:1057700040010D482830FBF7FFF805461DB90748E2
:1057800080F83E4E07E0302C01D10720C8E7601CAE
:10579000C4B2312CE6DB00BF0020C1E7D0020220FA
:1057A00020B001200025002040B80120A0250020C5
:1057B0002C2600202DE9FE4F82460C4615461E463B
:1057C0000C9F224890F8280000283DD14FF4FA6140
:1057D0001F48FBF7D3F91D48B0F8640030B11B48EF
:1057E000B0F864201BA11D48FAF7E2FD06EB460065
:1057F00000EBC6001A4901EB4000CDE9000705EBBC
:105800008500184901EB800304EB8400134901EB88
:10581000800215A10E48FAF7CBFD0D48FBF7C1F841
:105820000FFA80F949460A48FDF7DAFD80464246FC
:1058300013A102A8FAF7BCFD02A90548FBF71BF962
:105840000120024981F82800BDE8FE8F641F022074
:105850006C1702202530345800000000A0250020DD
:105860002C2600200025002023232C2C25732C2CF3
:1058700025732C2C25732C2C25732C2C0000000058
:10588000253034782C2C5A5A00000000704700BF95
:10589000011EA0F1010290B2FAD1704710B504A127
:1058A000012006F061FA4FF4807000F011F810BD8D
:1058B0003C2A2A2A2A2A2A2A2A2A2A2A2A2A2A2A36
:1058C0002A2ABFAAC6F4B1A3B4E60D0A000000005C
:1058D0000149086070470000143C014010B50748BA
:1058E000006800F07F000549091D096801F07F018B
:1058F000884202D27F2006F051FB10BD002C0040F0
:10590000F0B50A4600210023002400BF3DE0012538
:1059100005FA01F3156805EA03049C4234D10568D1
:105920004F000326BE40B543056015794E00B540D3
:105930000668354305601579012D02D01579022DD1
:1059400016D185684F000326BE40B5438560557962
:105950004E00B540866835438560456801268E4017
:10596000B5434560456896798E40B6B2354345608B
:10597000C5684F000326BE40B543C560D5794E00CB
:10598000B540C6683543C560491C1029BFD3F0BD7A
:10599000F0B5002300244D07ED0E02FA05F3CE10FA
:1059A00000F1200555F826504E07F70E0F26BE4091
:1059B000B543CF1000F1200646F82750CE1000F175
:1059C000200555F8265045EA0304CE1000F12005C5
:1059D00045F82640F0BD0246002013690B400BB18C
:1059E000012000E000207047418370470183704729
:1059F00000B52DED0A0BC5B09DED450ADDED480A59
:105A0000B4EEE00AF1EE10FA04DD4FF0FF304F493A
:105A1000086002E001204D4908609DED471ADDED68
:105A2000460A9DED450A68460AF09AFF302269460B
:105A300030A8FBF771F8DDED4D2A9DED4C2ADDED28
:105A40004B1A9DED4A1ADDED490A9DED480A68465C
:105A50000BF00EF83022694624A8FBF75DF824A964
:105A600030A80AF04BFE8DED3F0ACDED400A8DEDDA
:105A7000411ADDED412A9DED402ADDED3F1A9DEDF5
:105A8000471ADDED460A9DED450A05F001FC304858
:105A900080ED000A2F4890F82000082804D02D48F7
:105AA00090F820000A2810D12848012203682848CD
:105AB00090ED000A3FA924A80BF07AFA8DED420A76
:105AC000CDED430A8DED441A19E0224890F82000EC
:105AD000072804D01F4890F8200009280FD11B4840
:105AE000002203681A4890ED000A3FA924A80BF091
:105AF0005FFA8DED420ACDED430A8DED441A45AAB9
:105B000030A968460BF042FC3022694618A8FBF722
:105B100003F842AA24A968460BF038FC30226946F3
:105B20000CA8FAF7F9FF0CA918A80AF0E7FD8DED0B
:105B30003C0ACDED3D0A8DED3E1A9DED3C0ADDEDB2
:105B40003D0A9DED3E1A4FB000BD000060230020CD
:105B50005C230020641F022070B50446002146F239
:105B6000E000015128A12948FAF7DCFE054647E08C
:105B700046F2E0000059042829D14FF4FA6104F5F7
:105B80009650FAF7FBFF2A4621A104F59650FAF742
:105B90000FFC46F2E001095901EB810204F5FA61BC
:105BA00001EBC2001BA21AA1FAF702FC4FF4FA6142
:105BB00045F610102044FAF7E1FF4FF4FA6204F5BD
:105BC000965145F610102044FAF7A6FF0CE046F275
:105BD000E001095901EB810204F5FA6101EBC20011
:105BE0002A460BA1FAF7E4FB46F2E0000059401CFC
:105BF00046F2E001085104A10020FAF793FE0546A1
:105C0000002DB5D1002070BD2C2C0000007B0120A0
:105C100025730000300000002DE9F0418EB00446ED
:105C20000D461646342101A8FAF7A8FF2846FAF7D0
:105C3000B8FE80464246294601A8FAF728FF002010
:105C40002070314601A8FAF76DFE074611E0217871
:105C5000C1EB0112611C01EB42003A4608A1FAF7C0
:105C6000A7FB2078401C207031460020FAF75AFE2E
:105C70000746002FEBD100200EB0BDE8F0810000F8
:105C800025730000F0EE401AB4EEE01AF1EE10FABF
:105C900004DD30EEA10AF0EE400A08E0B4EEE01AAE
:105CA000F1EE10FA03D230EEE10AF0EE400A30EEE7
:105CB000C10AB0EEC00AB4EEE10AF1EE10FA01D862
:105CC000F0EE410AB0EE600A704700002DE9F041A5
:105CD000054600240026002146F2E400415100BFA1
:105CE0000BE004EB840141F690222A4402EBC10050
:105CF0002821FAF743FF601C84B2B4F5C87FF0DBBB
:105D0000D6A105F59650FAF70DFE804611E006EB98
:105D1000860141F690222A4402EBC1004246D0A1FE
:105D2000FAF746FBCDA10020FAF7FCFD8046701C77
:105D300086B2B8F1000FEAD1CAA1CD48FAF71CFE2D
:105D400078B900240BE004EB4401C1EB4411C94ACB
:105D500002EBC100E821FAF711FF601C84B2B442E3
:105D6000F1DBC548C0F88064BEA1C148FAF704FE63
:105D700000287DD1C14890F8DD00012879D109F0D3
:105D800039FEBF48466000242CE1BB48C0F884645B
:105D900004EB840241F690232B4403EBC20104EB95
:105DA0004402C2EB4412B34B03EBC200B5A2FFF7AF
:105DB00033FF002734E004EB4401C1EB4411AD4A4A
:105DC00002EBC101491CC7EB071201EB42000A229A
:105DD0000021FAF76EFD014604EB4400C0EB4410CD
:105DE000A44A02EBC000D83040F8271004EB44006E
:105DF000C0EB4410114601EBC000D83050F827002A
:105E000000EE100AB8EEC00AC4EBC4019C480C3086
:105E100000EB810000EB870080ED000A781C87B260
:105E2000022FC8DB04EB4401C1EB4411914A02EBA1
:105E3000C101491C04EB4402C2EB44128D4B13F820
:105E40003220521EC2EB021201EB4200FAF724FD8F
:105E5000C4EBC4028A490C3101EB8201886104EB76
:105E60004401C1EB4411834A02EBC101491C01E02A
:105E7000C8E0EFE004EB4402C2EB44127D4B13F8A0
:105E80003220921EC2EB021201EB4200FAF704FD2F
:105E9000C1B2C4EBC4027A480C3000EB820001733B
:105EA00004EB4401C1EB4411724A02EBC101491CED
:105EB00004EB4402C2EB44126E4B13F83220D21EA4
:105EC000C2EB021201EB4200FAF7E6FCC4EBC4029B
:105ED0006B490C3101EB8201086104EB4400C0EB1B
:105EE0004410644901EBC000401C04EB4401C1EBC9
:105EF0004411604A12F83110491FC1EB011100EB47
:105F0000410104EB4400C0EB441002EBC0000988DF
:105F1000A0F8D31004EB4400C0EB4410114601EB91
:105F2000C000401C04EB4401C1EB441112F83110D5
:105F3000091FC1EB011100EB410104EB4400C0EB70
:105F4000441002EBC0000988A0F8D51004EB44000F
:105F5000C0EB4410114601EBC00090F8D50070284A
:105F600008D10121C4EBC40245480C3000EB82008B
:105F700001751BE004EB4400C0EB44103D4901EB0C
:105F8000C00090F8D500712808D10221C4EBC402EA
:105F90003B480C3000EB8200017507E00021C4EBA8
:105FA000C40237480C3000EB8200017504EB440258
:105FB000C2EB44122F4B03EBC20292F8D51004EB54
:105FC0004402C2EB441203EBC20292F8D300FDF785
:105FD0009BF9C4EBC4022A490C3101EB8201C88150
:105FE000601C84B2B442FFF6D0AE0021234880F892
:105FF000DB1080F8DA1080F8DD104FF4127004F036
:106000006BF927E0002423E01FA11948FAF7B4FC3C
:1060100070B904EB840141F690222A4402EBC100DE
:1060200010220021FAF745FC194941F824000DE03F
:1060300004EB840141F690222A4402EBC1000A22BB
:106040000021FAF736FC124941F82400601C84B2A2
:10605000B442D9DB0020BDE8F08100003A3A0000EC
:10606000257300007365746C726F75740000000016
:1060700068B80120D0820120D0120220641F0220C3
:10608000C06D01205F000000736574746970730057
:106090001011022010B52DED068BFE480078002867
:1060A0007ED1FD48D0ED022A90ED012AD0ED001AF4
:1060B000FA4890ED021AD0ED010A90ED000AFFF7C0
:1060C0006FF9F74880ED090A9FEDF60AF64880ED72
:1060D000000A0020F5490870F54890ED020A10EE1C
:1060E000101A08460EF0F4FF41EC190BB0EE490A05
:1060F000F0EE690A06F064FFB0EE408AF0EE608AC6
:106100009FEDEC0B53EC102B51EC180B0EF0AEFC8A
:1061100070D2EA4890ED020A10EE101A08460EF00E
:10612000D7FF41EC190BB0EE490AF0EE690A06F010
:1061300047FFB0EE408AF0EE608A9FEDDE0B53EC35
:10614000102B51EC180B0EF091FCE1D2D44890EDDD
:10615000091AF0EE410ADA4890ED041AB0EE410A4D
:10616000FFF7F0F810EE104A20460EF0B1FF41ECB8
:106170001A0BB0EE4A0AF0EE6A0A06F021FFB0EE02
:10618000409AF0EE609A9FEDCF0B53EC102B51EC40
:10619000190B0EF0A7FC41EC180B0EF08BF900E088
:1061A00061E0C1490863084690ED0C0ADFEDC70ABB
:1061B000B4EEE00AF1EE10FA0DDD90ED0C0ADFED21
:1061C000C40AB4EEE00AF1EE10FA04D29FEDC10A5F
:1061D00080ED0C0A14E0B44890ED0C0ADFEDBE0A25
:1061E000B4EEE00AF1EE10FA05DD9FEDBC0A80ED99
:1061F0000C0A05E036E09FEDAB0AAB4880ED0C0AD7
:106200009FEDB70AB74880ED070A9FEDB50AB6487B
:1062100080ED070AB34890ED080AB8EEC00AD0ED49
:10622000070A30EE600A10EE101A08460EF050FF12
:1062300041EC190BB0EE490AF0EE690A06F0C0FE17
:10624000B0EE408AF0EE608A9FEDA80B53EC102B65
:1062500051EC180B0EF00AFC04D801208D4908708F
:10626000A44908702CE28B4800780128FAD18E48A6
:1062700090F82000032804D08B4890F820000428D0
:1062800032D1874890ED091AF0EE410A9A4890ED14
:10629000021AB0EE410AFFF755F8984880ED000A5F
:1062A0007F4890ED091AF0EE410A934890ED021AEA
:1062B000B0EE410AFFF746F810EE104A20460EF005
:1062C00007FF41EC190BB0EE490AF0EE690A06F03F
:1062D00077FEB0EE408AF0EE608A51EC180B0EF0BB
:1062E000E9F88749086039E06D4890ED091AF0EE49
:1062F000410A814890ED021ADFED821A31EE211A2F
:10630000B0EE410AFFF71EF87C4880ED000A6448B1
:1063100090ED091AF0EE410A774890ED021ADFED90
:10632000791A31EE211AB0EE410AFFF70BF810EEA0
:10633000104A20460EF0CCFE41EC190BB0EE490A93
:10634000F0EE690A06F03CFEB0EE408AF0EE608A9C
:1063500051EC180B0EF0AEF869490860684890EDF2
:10636000000ADFED690AB4EEE00AF1EE10FA07DB8D
:1063700090ED000ADFED640A30EE600A80ED000A5D
:106380005C480078F0B35E4800680EF0A1FE41EC76
:10639000180B9FED5E0B53EC102B0EF0A1FC0AD8EE
:1063A0004148B0F8720000EE100AB8EE400A3E48CC
:1063B00080ED000AF6E0524800680EF089FE41ECDC
:1063C000180B9FED520B53EC102B0EF04FFB27D206
:1063D0004B4890ED000ADFED4F0AB4EEE00AF1EE13
:1063E00010FA1DDD3048B0F8720000EE100AB8EE69
:1063F000400AB0EE402AF3EE0E1A9FED471ADFED89
:10640000450A00E01AE03E4890ED000A0BF062FAFF
:10641000BDEEC00AB8EEC00A234880ED000AC1E014
:10642000374890ED000ADFED3B0AB4EEE00AF1EEEA
:1064300010FA02D800202F490870B3E09FED190A26
:10644000194880ED000A9FED170A264880ED070ADB
:106450009FED140A244880ED070A154890ED020AC2
:1064600010EE101A08460EF033FE41EC190BB0EE98
:10647000490AF0EE690A06F0A3FDB0EE408AF0EE9C
:10648000608A9FED0C0B53EC102B51EC180B0EF0A7
:10649000EDFA43E0901F0020382102202C21022039
:1064A0009420022000000000641F0220B01F002082
:1064B0001817012000000000000014406817012098
:1064C000281601206666666666A64C4000008C426F
:1064D0000000DC420000B4420000204300003443CE
:1064E00089415F4240170120901701200000000001
:1064F0000000F03FB11F002044210220A81F00200F
:10650000A41F0020DA0F4940DA0FC9403333333378
:106510003333E33FCDCCCC3C9A99193F42D26C48FF
:1065200090ED020A10EE101A08460EF0D1FD41EC73
:10653000190BB0EE490AF0EE690A06F041FDB0EE23
:10654000408AF0EE608A1FED250B53EC102B51ECC6
:10655000180B0EF08BFA25D25E4890ED080AB8EEC3
:10656000C00AD0ED070A30EE600A10EE101A084695
:106570000EF0AEFD41EC190BB0EE490AF0EE690ADF
:1065800006F01EFDB0EE408AF0EE608A1FED290B8A
:1065900053EC102B51EC180B0EF068FA02D80120C6
:1065A0004D4908704D4890ED000A4D4880ED000AB5
:1065B0004948007801287ED11FED460A484880ED01
:1065C000000A1FED480A474880ED000A464890ED52
:1065D000020A10EE101A08460EF07AFD41EC190B73
:1065E000B0EE490AF0EE690A06F0EAFCB0EE408A25
:1065F000F0EE608A1FED510B53EC102B51EC180B91
:106600000EF034FA5CD2324890ED020A10EE101A05
:1066100008460EF05DFD41EC190BB0EE490AF0EEB4
:10662000690A06F0CDFCB0EE408AF0EE608A1FEDFC
:106630005F0B53EC102B51EC180B0EF017FA3FD2F6
:106640002848D0F8140129490968401A40F2DC5161
:10665000884235D9234890F82000032804D02148E7
:1066600090F8200004280DD101211E48807E401E94
:10667000C0EBC0021E4800EB8200C18100201D4912
:1066800008701DE0174890F82000052804D0154830
:1066900090F82000062813D102211248807E401E67
:1066A000C0EBC002124800EB8200C18100201149FA
:1066B000087005E0FFE70B48D0F814010B490860AB
:1066C000B7EE080A0CF032FDBDEC068B10BD0000E1
:1066D0006817012040170120B01F0020A81F0020CC
:1066E000AC1F0020641F022018170120B41F0020D7
:1066F000CC6D0120901F002010B52DED068B314888
:1067000090ED000A10EE101A08460EF0E1FC41EC84
:10671000190BB0EE490AF0EE690A06F051FCB0EE32
:10672000408AF0EE608A9FED280B53EC102B51EC61
:10673000180B0EF0D5FA0ED82548B0F91C0000EE63
:10674000100AB8EEC00A224880ED000AB6EE000A30
:106750000CF0ECFC33E01B4890ED000A10EE101A30
:1067600008460EF0B5FC41EC1A0BB0EE4A0AF0EE0A
:106770006A0A06F025FCB0EE409AF0EE609A51EC01
:10678000190B0DF097FE08EE100A1148B0F91C0025
:1067900000EE100AB8EEC00AB0EE402ADFED0D1A86
:1067A0009FED0D1ADFED0D0AB0EE480A0BF092F8DE
:1067B000074880ED000A9FED0A0A0CF0B7FCBDEC1B
:1067C000068B10BD94200220333333333333E33F41
:1067D000641F02200000C8429A99193F000000007F
:1067E000CDCC4C3E10B52DED0A8BA748D0ED022A3A
:1067F00090ED012AD0ED001AA44890ED021AD0EDD8
:10680000010A90ED000A04F043FDB0EE408A9FEDCE
:10681000A00AB4EEC08AF1EE10FA24DD9D4890ED96
:10682000030A10EE101A08460EF052FC41EC1C0B45
:10683000B0EE4C0AF0EE6C0A06F0C2FBB0EE40AAD5
:10684000F0EE60AA18EE100A0EF042FC41EC1B0BB1
:1068500053EC1A2B0EF052FB41EC190B0DF02AFEF3
:106860008C49086123E08B4890ED030A10EE101A62
:1068700008460EF02DFC41EC1C0BB0EE4C0AF0EE7D
:106880006C0A06F09DFBB0EE40AAF0EE60AA18EE8E
:10689000100A0EF01DFC41EC1B0B53EC1A2B0EF0F2
:1068A0002DFB41EC190B0DF005FE7A4908617A4881
:1068B00090F82000784991F8211088420AD1764852
:1068C000B0F91C0000EE100AB8EEC00A724880ED64
:1068D000000ABAE0704890F8210007280ED06E48F0
:1068E00090F82100082809D06B4890F82100092869
:1068F00004D0694890F821000A2841D16548D0EDBC
:10690000040A6548B0F8680000EE100AB8EE400AC4
:10691000F4EEC00AF1EE10FA0ADB5F48B0F91C0091
:1069200000EE100AB8EEC00A5B4880ED000A8CE069
:106930005948B0F91C0000EE900AF8EEE00AB0EEFB
:10694000602A5548B0F91E0000EE900AF8EEE00A01
:10695000F0EE601A5048B0F8680000EE900AF8EEC9
:10696000600AB0EE601A4B48D0ED040AB0EE600A3F
:10697000DFED4A0A0AF0AEFF474880ED000A64E006
:106980004448D0ED040A4448B0F8680000EE100A0C
:10699000B8EE400AF4EEC00AF1EE10FA0ADB3E4807
:1069A000B0F91C0000EE100AB8EEC00A3A4880EDBB
:1069B000000A4AE03748D0ED040A3748B0F86800CA
:1069C00000EE100AB8EE400AF4EEC00AF1EE10FA3A
:1069D00031D8304890ED040ADFED310AB4EEE00A18
:1069E000F1EE10FA27DD2C48B0F91C0000EE900AF9
:1069F000F8EEE00AB0EE602A2748B0F8660000EE34
:106A0000900AF8EE600AF0EE601A2348B0F86800C9
:106A100000EE900AF8EE600AB0EE601A1D48D0ED64
:106A2000040AB0EE600ADFED1E0A0AF053FF1A48AE
:106A300080ED000A09E01848B0F8660000EE100A80
:106A4000B8EE400A144880ED000A124890ED030A9F
:106A5000DFED130AB4EEE00AF1EE10FA04D29FED76
:106A6000110A0D4880ED000A0F4890ED010AB5EEBD
:106A7000C00AF1EE10FA04D09FED080A064880ED36
:106A8000000ABDEC0A8B10BD382102202C21022007
:106A900000401C4694200220641F022000000000D9
:106AA000000096430000C8420C18012070B531A5C3
:106AB00000240BE0285D3A49888000BF38480088F0
:106AC00000F040000028F9D0601CC4B22A2CF1D399
:106AD0004FE07F2005F062FA05F020FA3148007897
:106AE000401C3049087008460078012800DD70BD60
:106AF000002240F225512C4805F078F8002240F29F
:106B00002771294805F072F8002240F225512448E7
:106B100005F06CF8002240F22771214805F066F874
:106B2000002240F22551214805F060F8002240F291
:106B300027711E4805F05AF8002240F225511C48E2
:106B400005F054F8002240F22771194805F04EF87C
:106B500000BFBFF34F8F1748006800F4E06016498C
:106B60000843001D13490860BFF34F8F00BF00BFEB
:106B7000FEE7AEE70D0A456E7465722048617264E7
:106B80004661756C745F48616E646C65722C20534D
:106B9000797374656D2048616C742E0D0A000000D5
:106BA0000010014074070020001401400044004020
:106BB000004800400CED00E00000FA0510B50AF0B6
:106BC0001BFD0AF05BFC10BD7047000010B52C489F
:106BD000407F88B1C82001F0EDF82A4908700846C6
:106BE000007820B10121084602F088FA08E000216F
:106BF000012002F083FA03E00121084602F07EFA48
:106C00002148407F88B1C82001F0D4F81F4908709E
:106C10000846007820B10121032002F06FFA08E055
:106C20000021032002F06AFA03E00121032002F0B0
:106C300065FA174890F8FA0088B1C82001F0BAF850
:106C4000144908700846007820B10121022002F0A2
:106C500055FA08E00021022002F050FA03E0012179
:106C6000022002F04BFA0848407F20B101210420A5
:106C700002F044FA03E00021042002F03FFA10BDC4
:106C80004C160120C021002028160120C12100201F
:106C9000641F0220C221002010287DD2DFE800F00E
:106CA000081C2C3D57658191A0A9B2C2D2E0F2F038
:106CB0004FF41671824A51644FF4FA7191644FF4A3
:106CC000C871D1644FF41671116540F23A215165D3
:106CD00040F226219165F1E04FF47A71784A5164CF
:106CE0004FF4487191644FF41671D1644FF44871B8
:106CF000116551659165E1E09621714A51647821F1
:106D000091646421D1644FF4EB7111654FF4DC712F
:106D100051654FF4D2719165D0E04FF49661684AA5
:106D200051644FF47A7191644FF44871D164114603
:106D3000C96DC1F5FA7111651146C96DC1F5FA71D8
:106D400051651146C96DC1F5FA719165B6E04FF410
:106D500096615B4A51644FF47A7191644FF44871C3
:106D6000D164116551659165A8E040F2DC51544A47
:106D7000516440F24C4191644FF47A71D1641146F0
:106D8000C96DC1F5617111651146C96DC1F56171BA
:106D900051651146C96D00E08FE0C1F561719165E3
:106DA0008CE04FF4FA61464A51644FF4C861916433
:106DB0004FF49661D16440F24C4111655165916583
:106DC0007CE04FF448713E4A51644FF4167191646F
:106DD0004FF4C871D16449001165516591656DE04A
:106DE0000021374A51649164D16411655165916500
:106DF00064E00021324A51649164D16411655165A7
:106E000091655BE04FF461712D4A51644FF42F712D
:106E100091644FF4FA71D1644FF448711165516572
:106E200091654BE04FF44871254A51644FF4167157
:106E300091644FF4C871D1644FF4E17111655165EB
:106E400091653BE04FF448711D4A51644FF416714F
:106E50009164C821D16489001165516591652DE067
:106E60004FF49661164A51644FF47A7191644FF46D
:106E70004871D1644FF47A711165516591651DE0D7
:106E80000EE0FFE74FF416710D4A51644FF4C871DC
:106E90009164C821D16489001165516591650DE047
:106EA0004FF4C871064A51644FF496719164C82139
:106EB000D16411655165916500E000BF00BF704766
:106EC000641F022010B50446202C79D2DFE804F0BC
:106ED000101D2A3744515E6B798693A0ADBAC7D492
:106EE000F1FEEEEDECEBEAE9E8E7E6E5E4E3E2E10A
:106EF0000021162002F002F90021172002F0FEF80E
:106F00000021182002F0FAF8A4E10121162002F075
:106F1000F5F80021172002F0F1F80021182002F006
:106F2000EDF897E10021162002F0E8F80121172082
:106F300002F0E4F80021182002F0E0F88AE10021D4
:106F4000162002F0DBF80021172002F0D7F801210B
:106F5000182002F0D3F87DE10121162002F0CEF8CE
:106F60000121172002F0CAF80021182002F0C6F80B
:106F700070E10021162002F0C1F80121172002F073
:106F8000BDF80021182002F0B9F863E101211620B4
:106F900002F0B4F80021172002F0B0F80021182008
:106FA00002F0ACF856E10021162002F0A7F800210B
:106FB000172002F0A3F80021182002F09FF849E101
:106FC00047E10121162002F099F80121172002F073
:106FD00095F80121182002F091F83BE101211620DB
:106FE00002F08CF80021172002F088F80121182007
:106FF00002F084F82EE10021162002F07FF8012132
:10700000172002F07BF80121182002F077F821E127
:107010000121162002F072F80121172002F06EF80B
:107020000121182002F06AF814E10121162002F073
:1070300065F80121172002F061F80021182002F004
:107040005DF807E10021162002F058F80021172012
:1070500002F054F80121182002F050F8FAE0012162
:10706000162002F04BF80021172002F047F801210A
:10707000182002F043F8EDE00021162002F03EF85F
:107080000121172002F03AF80121182002F036F809
:10709000E0E0D1E0C3E0B5E0A7E099E08BE07DE07F
:1070A0006FE061E053E045E037E029E01BE00DE0F0
:1070B000FFE70121162002F021F80121172002F03C
:1070C0001DF80121182002F019F8C3E00121162053
:1070D00002F014F80121172002F010F80021182006
:1070E00002F00CF8B6E00021162002F007F80021AB
:1070F000172002F003F80121182001F0FFFFA9E09A
:107100000121162001F0FAFF0021172001F0F6FFFF
:107110000121182001F0F2FF9CE00021162001F06F
:10712000EDFF0121172001F0E9FF0121182001F0F6
:10713000E5FF8FE00121162001F0E0FF012117207B
:1071400001F0DCFF0121182001F0D8FF82E00121CD
:10715000162001F0D3FF0121172001F0CFFF0021FD
:10716000182001F0CBFF75E00021162001F0C6FFCA
:107170000021172001F0C2FF0121182001F0BEFFFD
:1071800068E00121162001F0B9FF0121172001F06C
:10719000B5FF0121182001F0B1FF5BE000211620AE
:1071A00001F0ACFF0121172001F0A8FF01211820F8
:1071B00001F0A4FF4EE00121162001F09FFF002105
:1071C000172001F09BFF0121182001F097FF41E0FB
:1071D0000021162001F092FF0021172001F08EFF00
:1071E0000121182001F08AFF34E00121162001F06E
:1071F00085FF0121172001F081FF0021182001F0F7
:107200007DFF27E00021162001F078FF01211720E3
:1072100001F074FF0021182001F070FF1AE0012135
:10722000162001F06BFF0021172001F067FF0021FD
:10723000182001F063FF0DE00021162001F05EFF31
:107240000021172001F05AFF0021182001F056FFFD
:1072500000E000BF00BF10BD10B52DED0A8BD54872
:1072600000680DF035FF41EC180BD34890ED020A91
:1072700010EE101A08460DF02BFF41EC1A0BB0EE81
:107280004A0AF0EE6A0A05F09BFEB0EE409AF0EE74
:10729000609A53EC182B51EC190B0DF0E7FB35D22B
:1072A000C44800680DF014FF41EC180BC24890ED83
:1072B000030A10EE101A08460DF00AFF41EC1A0BF3
:1072C000B0EE4A0AF0EE6A0A05F07AFEB0EE409A95
:1072D000F0EE609A53EC182B51EC190B0DF0C6FB35
:1072E00014D2B6480078012810D1202002F0F4FF13
:1072F0004FF4007003F0AEFD0121B14880F8DD10BD
:10730000002180F8DB1080F8AC104FE10020AB4981
:107310000870AC480078012843D1A74890ED020AD4
:10732000A948D0ED000AB4EEE00AF1EE10FA03DD50
:107330000120A349087416E09F4890ED020AA24874
:10734000D0ED000AF1EE600AB4EEE00AF1EE10FAB8
:1073500003D202209A49087405E000209849087475
:10736000022098490870944890ED040A10EE101A13
:1073700008460DF0ADFE41EC1A0B9FED940B53EC5B
:10738000102B0DF0AFFB41EC190B0DF093F808EE4C
:10739000100AB0EE480AFDF733FC874880ED060A74
:1073A00004E188480078022868D1032084490874E1
:1073B0009FED880A084680ED0C0A7F4890ED040A8C
:1073C00010EE101A08460DF083FE41EC1C0B9FEDE9
:1073D0007F0B53EC102B0DF085FB41EC1B0B0DF0DC
:1073E00069F808EE100A744890ED060AF0EE400ABB
:1073F000B0EE480AFDF79CFCDFED760A30EE600A3D
:1074000010EE104A20460DF063FE41EC1A0BB0EE70
:107410004A0AF0EE6A0A05F0D3FDB0EE409AF0EEAB
:10742000609A9FED6D0B53EC102B51EC190B0DF086
:107430001DFBB5D20020624908745F4890ED040A34
:1074400010EE101A08460DF043FE41EC1A0B9FEDAA
:107450005F0B53EC102B0DF045FB41EC190B0DF0BD
:1074600029F808EE100AB0EE480AFDF7C9FB5248A9
:1074700080ED060A03205349087097E051480078D0
:10748000032826D14C4890ED020A4F48D0ED000A5F
:10749000B4EEE00AF1EE10FA03DD01204849087469
:1074A00084E0454890ED020A4748D0ED000AF1EE2D
:1074B000600AB4EEE00AF1EE10FA03D2022040496D
:1074C000087473E000203E49087404203D490870A8
:1074D0006CE03C480078042868D1394908749FED75
:1074E0003D0A084680ED0C0A334890ED040A10EE80
:1074F000101A08460DF0ECFD41EC1C0B9FED330B10
:1075000053EC102B0DF0EEFA41EC1B0B0CF0D2FFFC
:1075100008EE100A284890ED060AF0EE400AB0EE98
:10752000480AFDF705FCDFED2B0A30EE600A10EE8D
:10753000104A20460DF0CCFD41EC1A0BB0EE4A0A81
:10754000F0EE6A0A05F03CFDB0EE409AF0EE609A6B
:107550009FED210B53EC102B51EC190B0DF086FA1B
:1075600024D2002016490874134890ED040A10EE46
:10757000101A08460DF0ACFD41EC1A0B9FED130BF1
:1075800053EC102B0DF0AEFA41EC190B0CF092FFFE
:1075900008EE100AB0EE480AFDF732FB064880ED0F
:1075A000060A01200549087006490870BDEC0A8BDF
:1075B00010BD0000682100204C160120AD210020E4
:1075C000641F0220AC2100206C21002066666666E4
:1075D00066A64C400000B442000000000000F03FEE
:1075E00010B52DED0A8B944890ED040A10EE101A98
:1075F00008460DF06DFD41EC1C0B9FED900B53EC1C
:10760000102B0DF06FFA41EC1B0B0CF053FF08EE42
:10761000100A894890ED060AF0EE400AB0EE480ADA
:10762000FDF786FBDFED870A30EE600A10EE104AA8
:1076300020460DF04DFD41EC1A0BB0EE4A0AF0EE7B
:107640006A0A05F0BDFCB0EE409AF0EE609A51EC8B
:10765000190B0CF02FFF7C490860084690ED000ADA
:107660007A4880ED000A7A48007C05280ED2DFE8CF
:1076700000F0030E192481009FED760A764880ED14
:10768000000A9FED740A754880ED000ACFE0B3EE62
:107690000E0A714880ED000AB3EE0E0A6F4880EDC5
:1076A000000AC4E0BBEE0E0A6B4880ED000ABBEE98
:1076B0000E0A6A4880ED000AB9E0634890ED000ABE
:1076C000DFED670AB4EEE00AF1EE10FA15DD60486E
:1076D000B0F87200404200EE100AB8EEC00A5E48F0
:1076E00080ED000A5A48B0F8720000EE100AB8EEB9
:1076F000400A5A4880ED000A3BE0534800680DF00C
:10770000E7FC41EC180B9FED570B53EC102B0DF0E1
:10771000E7FA24D24E48B0F8720000EE100AB8EE34
:10772000400AB0EE402AF3EE041AB3EE0E1AF6EE5B
:10773000000A454890ED000A0AF0CCF84B4880ED6D
:10774000000A90ED000AB1EE400A434880ED000ABD
:10775000464890ED000A414880ED000A09E09FED9F
:107760003D0A3D4880ED000A9FED3A0A3B4880ED16
:10777000000A5CE0344890ED000ADFED390AB4EE0F
:10778000E00AF1EE10FA15DD3148B0F8720000EEB3
:10779000100AB8EE400A304880ED000A2C48B0F8D4
:1077A0007200404200EE100AB8EEC00A2B4880ED8D
:1077B000000A3BE0244800680DF08AFC41EC180BFD
:1077C0009FED280B53EC102B0DF08AFA24D22048A1
:1077D000B0F8720000EE100AB8EE400AB0EE402A8F
:1077E000F3EE041AB3EE0E1AF6EE000A164890ED08
:1077F000000A0AF06FF81D4880ED000A90ED000ABB
:10780000154880ED000A194890ED000AB1EE400AD3
:10781000124880ED000A09E09FED0E0A0E4880ED47
:10782000000A9FED0C0A0D4880ED000A00BF00BF62
:10783000BDEC0A8B10BD00004C1601206666666622
:1078400066A64C400000B442B02100207C210020FC
:10785000641F022000000000E8160120001701202C
:1078600000003442000000000000E03FB42100208E
:1078700010B52DED068B934800680DF029FC41EC06
:10788000180B914890ED020A10EE101A08460DF000
:107890001FFC41EC1A0BB0EE4A0AF0EE6A0A05F042
:1078A0008FFBB0EE409AF0EE609A53EC182B51EC3F
:1078B000190B0DF0DBF837D2824800680DF008FC98
:1078C00041EC180B804890ED030A10EE101A0846A0
:1078D0000DF0FEFB41EC1A0BB0EE4A0AF0EE6A0A1C
:1078E00005F06EFBB0EE409AF0EE609A53EC182B68
:1078F00051EC190B0DF0BAF816D274480078012833
:1079000012D1802002F0E8FC4FF4007003F0A2FADC
:1079100001216F4880F8DD10002180F8DA1080F82E
:10792000AD1080F8AF10CAE00020684908706948BF
:107930000078012843D1644890ED020A6648D0EDF2
:10794000000AB4EEE00AF1EE10FA03DD012060490E
:10795000487416E05C4890ED020A5F48D0ED000ADA
:10796000F1EE600AB4EEE00AF1EE10FA03D2022062
:107970005749487405E0002055494874022055498C
:107980000870514890ED040A10EE101A08460DF0E8
:107990009FFB41EC1A0B9FED510B53EC102B0DF09C
:1079A000A1F841EC190B0CF085FD08EE100AB0EEC1
:1079B000480AFDF725F9444880ED060A7FE045486E
:1079C0000078022826D10320414948749FED450ADA
:1079D000454880ED070A90ED081AB8EEC11AF0EE9E
:1079E000410A90ED071AB0EE410AFDF7A1F9F0EE59
:1079F000000AB4EEE00AF1EE10FA01D8012000E02E
:107A0000002000285BD00020314948740320314910
:107A1000087054E02F480078032826D12A4890EDBA
:107A2000030A2D48D0ED000AB4EEE00AF1EE10FA98
:107A300003DD02202649487441E0234890ED030A03
:107A40002548D0ED000AF1EE600AB4EEE00AF1EE4E
:107A500010FA03D201201E49487430E000201C496E
:107A6000487404201B49087029E01A48007804284B
:107A700025D1174948749FED1D0A1B4880ED070A60
:107A800090ED081AB8EEC11AF0EE410A90ED071A0F
:107A9000B0EE410AFDF74CF9F0EE000AB4EEE00A50
:107AA000F1EE10FA01D8012000E0002038B10020EA
:107AB0000749487401200549087006490870BDEC63
:107AC000068B10BD74210020281601207121002092
:107AD000641F0220702100207821002066666666FF
:107AE00066A64C400000B442401701200000000090
:107AF00010B52DED0A8B494890ED040A10EE101ACE
:107B000008460DF0E5FA41EC1C0B9FED450B53ECDC
:107B1000102B0CF0E7FF41EC1B0B0CF0CBFC08EE3C
:107B2000100A3E4890ED060AF0EE400AB0EE480A10
:107B3000FDF7FEF8DFED3C0A30EE600A10EE104A69
:107B400020460DF0C5FA41EC1A0BB0EE4A0AF0EEF1
:107B50006A0A05F035FAB0EE409AF0EE609A51EC00
:107B6000190B0CF0A7FC314908603148407C05280E
:107B70004FD2DFE800F0030E192439009FED2D0AE3
:107B80002D4880ED010A9FED2B0A2C4880ED010A5B
:107B90003FE0B3EE0E0A284880ED010AB3EE0E0A6C
:107BA000264880ED010A34E0BBEE0E0A224880ED43
:107BB000010ABBEE0E0A214880ED010A29E09FED83
:107BC0001D0A1D4880ED010A9FED1A0A1B4880ED31
:107BD000010A9FED150A1A4880ED070A9FED120A67
:107BE000184880ED070A14E09FED120A124880ED54
:107BF000010A9FED100A114880ED010A9FED0D0A60
:107C00000F4880ED070A9FED0B0A0E4880ED070A2A
:107C100000BF00BFBDEC0A8B10BD0000281601207C
:107C20006666666666A64C400000B442B821002035
:107C3000641F0220000000001817012068170120AF
:107C4000401701209017012000BFFEE730B5054620
:107C50000C4622460021284600F001F830BD2DE9EF
:107C6000F04103460C4617460FB9BDE8F08103B951
:107C7000FBE70025002202E02D022543521C042AC6
:107C8000FAD3384603F0030C1946BCF1000F08D0B4
:107C9000624603E001F8014B401E521C08B1042A61
:107CA000F8D30E4601E020C6001F0428FBD231465F
:107CB00002E001F8014B401E0028FAD100BFD4E7D2
:107CC00070B504460D461448D0F8140113490968EC
:107CD000401AB0F5FA7F1DD90F48D0F814010F49AA
:107CE00008600D48C07A50B10D4844718571002379
:107CF0000822014640F20A60FCF7CAF90AE0084887
:107D000044710020064988710023082240F20A606D
:107D1000FCF7BEF970BD0000641F0220A013002014
:107D2000981300207047000070B5002100230F2237
:107D3000C4781CB3174C246804F4E064C4F5E06410
:107D4000C4F30721C1F10404E3B20A4144789C4022
:107D5000E1B28478144021430C07210E0E4C0578C3
:107D60006155047804F01F050124AC4005786D11BD
:107D7000AD0005F1E025C5F8004109E0047804F004
:107D80001F050124AC40054D0678761145F82640C4
:107D900070BD00000CED00E000E400E080E100E0D8
:107DA00002490143024A1160704700000000FA05D1
:107DB0000CED00E001460B48D0F814010A4A1268A5
:107DC000801A88420AD90748D0F81401064A106080
:107DD0000648007880F00100044A107003480078DB
:107DE00070470000641F0220D8160020DC16002017
:107DF0007047704770B5044600F054F800201E49E3
:107E000008701E4908701E4908701E4908601E4906
:107E100008601E4908701E4908701E4908701E48F7
:107E2000006858B11D48056845B11B48066803E065
:107E3000761E002028602D1D002EF9D10020184943
:107E4000087000F001FD00F02FFD204600F0DCFD81
:107E5000208800B170BD204600F096FB208800B15C
:107E6000F8E7204601F0EEF8208800B1F2E7FFF7CE
:107E7000BFFF00BFEEE70000980700209907002031
:107E80009D070020B0070020B40700209A070020BB
:107E90009B0700209C07002000530108FC520108AA
:107EA000A6070020064800680649096800EB810023
:107EB000054908600846006820F007000860704720
:107EC000FC52010800530108B80700200848007858
:107ED000012800D0704707480078FA2800DBF9E74E
:107EE00004480078401C0349087000BFF2E7000016
:107EF000990700209807002010B500242948007831
:107F0000012800D010BD00BFF8F72AFA044600BFD0
:107F10002548007828B900BF2046F8F725FA00BFA9
:107F2000F0E721480078401E1F4908700846007895
:107F3000002805DD00BF2046F8F716FA00BFE1E78C
:107F40001A480078002805DD00BF2046F8F70CFA33
:107F500000BFD7E700F064FC1549087008460078B8
:107F600000EB4000134951F820001349086008460F
:107F7000006812490968884205D100BF2046F8F719
:107F8000F3F900BFBEE70E480068401C0C490860CA
:107F9000FBF7CEF800BF2046F8F7E6F900BF00BFB8
:107FA000B0E7000099070020980700209D070020F7
:107FB0009B07002050DC0020B4070020B007002001
:107FC000A007002010B500241A480078002800DD22
:107FD00010BD19480078002800DDF9E700BFF8F768
:107FE000BFF9044600BF00F01BFC144908700846A6
:107FF000007800EB4000124951F820001149086058
:108000000846006810490968884205D100BF20462B
:10801000F8F7AAF900BFDBE70C480068401C0B49E1
:108020000860FBF780F800BF2046F8F79DF900BF15
:1080300000BFCDE7980700209D0700209B07002088
:1080400050DC0020B4070020B0070020A00700206B
:1080500010B5044612480078E8B900F0E1FB114978
:10806000087008460078104908700E48007800EB48
:1080700040000E4951F820000D490860084600688C
:108080000C490860012006490870FBF73BF843F6ED
:108090009920208002E045F68A60208010BD000013
:1080A000990700209B0700209A07002050DC002041
:1080B000B4070020B00700202DE9FF4F85B004462B
:1080C00091469A46DDF854B0199E139D0020029007
:1080D00012980F2809D13F48844206D046F27321F6
:1080E0001A98018009B0BDE8F08F204600F098FC96
:1080F00000211A98018006F0010088B106F0020004
:1081000070B1A8460020049007E00020C8F80000E5
:1081100008F104080498401C049004985845F4D3CE
:10812000149805EB80000390CDE900B62A4651462D
:108130004846039B00F006F98046C4F82890C4F82E
:108140002CA006982062129884F83700C4F80080AA
:108150000398A06017986065189860606562C4F81D
:1081600038B0A687002706E0002104F15C0040F843
:108170002710781CC7B2002FF6D0204600F030F848
:1081800000BF00BFF8F7ECF8029000BF00BF94F802
:10819000370000F065FB204600F0CEFB0E4800885B
:1081A000401C0D4908800D480078012807D000BF09
:1081B00000BF0298F8F7D8F800BF00BF92E700BFF1
:1081C00000BF0298F8F7D0F800BF00BFFFF7FAFE33
:1081D00000BF87E7E8DB0020A40700209907002004
:1081E000704770472DE9F0470746884614461D46FC
:1081F0004FF000090CB10020206000BF00BFF8F76D
:10820000AFF8814600BF00BF43480068406CD0B162
:1082100041480068406C401E3F49096848643E4838
:108220000068466C1CB13C480068006C206000BFD0
:1082300000BF4846F8F798F800BF00BF002028802C
:108240003046BDE8F08708F4004058B100BF00BFD9
:108250004846F8F789F800BF00BF46F2B010288002
:108260000020EEE72D48007800280BDD00BF00BF9E
:108270004846F8F779F800BF00BF46F663502880FB
:108280000020DEE73B4607220021084600F0B4F953
:1082900000BF00BF4846F8F767F800BF00BFFFF710
:1082A00091FE00BF00BFF8F75BF8814600BF00BF3A
:1082B0001948006890F8350020B101280AD0032839
:1082C00018D110E01CB114480068006C2060002038
:1082D000288013E01CB110480068006C206046F252
:1082E000A91028800AE00CB10020206047F2D920B4
:1082F000288003E046F62E60288000BF00BF0648B5
:108300000068466C00BF00BF4846F8F72DF800BF74
:1083100000BF304695E70000B00700209D07002011
:108320002DE9F04105460E4614464FF0000823465D
:1083300042463146284600F0C9FB07463846BDE8AC
:10834000F0810000F0B50446DDE9055602EB85003A
:1083500020F007004FF0807C071F3846C7F800C0A8
:10836000071F38463C60DFF8A8C0071F3846C7F82B
:1083700000C04FF0123C071F3846C7F800C04FF04E
:10838000033C071F3846C7F800C04FF0023C071FE8
:108390003846C7F800C0071F38463B60071F3846FD
:1083A00039604FF0113C071F3846C7F800C04FF046
:1083B000103C071F3846C7F800C04FF0093C071FA4
:1083C0003846C7F800C04FF0083C071F3846C7F8CA
:1083D00000C04FF0073C071F3846C7F800C04FF0F9
:1083E000063C071F3846C7F800C04FF0053C071F82
:1083F0003846C7F800C04FF0043C071F3846C7F89E
:1084000000C06FF0020C071F3846C7F800C0F0BD6F
:10841000A98A0008704700002DE9F04105460E4684
:108420001446002726480078002804DD46F66350ED
:108430002080BDE8F08136B1022E05D0042E0AD08E
:10844000082E09D101E000BF00BF1DB947F27E2010
:108450002080EEE704E003E045F625602080E8E7B1
:1084600000BF00BF00BFF7F77BFF074600BF00BF9C
:1084700001201449096881F836002346324629460E
:108480001048006800F018FC208838B100BF00BF19
:108490003846F7F769FF00BF00BFCAE70948006820
:1084A00000F068FA00BF00BF3846F7F75DFF00BF75
:1084B00000BFFFF787FD0020208000BFB9E7000064
:1084C0009D070020B007002070B50446002600BFBD
:1084D00000BFF7F745FF064600BF00BF0648056826
:1084E00000BF00BF3046F7F73FFF00BF00BF0020CE
:1084F0002080284670BD0000A807002008B500F0C5
:1085000009F86A4600210248FFF70AFF08BD00008B
:1085100010DD00207047000010B5002400BF00BF30
:10852000F7F71EFF044600BF00BF08480078401C54
:108530000649087000BF00BF2046F7F715FF00BFCF
:1085400000BFFFF7DBFFFFF7D7FC10BD9807002047
:10855000002400BF14E000BF00BFF7F701FF04468E
:1085600000BF00BF07480068401C0649086000BF04
:1085700000BF2046F7F7F8FE00BF00BFFFF739FC49
:10858000E9E700009407002010B58AB004460020F7
:108590000E4908600B2000210591CDE907040691E2
:1085A00008460B4909680B4A12680B4B1B68CDE95A
:1085B0000132CDE903100F200023084A08A10090E2
:1085C0000C48FFF779FD0AB010BD000094070020A9
:1085D000D8520108D4520108D05201085185000830
:1085E00075432F4F532D4949492049646C652054E8
:1085F00061736B00E8DB00202DE9F04105460C4675
:1086000016461F461248006880F834600020104962
:10861000096881F8350039460D48006800F0D8F93E
:108620006CB104F10808EC60012229460848006892
:1086300000F010F82946404600F01FF806E0002040
:1086400003490968C887024909680863BDE8F081E1
:10865000B007002010B5C287016300230AE00024A0
:108660004C600C600C614C610C83CC6188602031E3
:108670005C1CA3B29342F2DB10BDF0B58E6896F895
:10868000375007893FB90127078100274F600F60E6
:108690000160416023E007897F1C0781026806E0D2
:1086A000946894F83770AF4200DD02E05268002A07
:1086B000F6D100BF32B900274F6043680B605960A4
:1086C00041600CE017682FB9116000270F604A6005
:1086D000016004E013680B604A6059601160F0BDEE
:1086E0002DE9F0410446256BE68F0AE0D5F80C80B1
:1086F00008F108072946384600F00AF82035701EB0
:1087000086B2002EF2DC0020E0872063BDE8F08115
:1087100010B50489012C03D100240460446011E0E9
:108720000C6824B94A680024146002600AE04C68AE
:1087300024B90B6800245C60436003E00B684A685E
:108740005A6013600489641E048100244C600C602C
:1087500010BD2DE9F84306460C4617469846089D7D
:1087600094F83600082842D2DFE800F00405080932
:108770000607242500BF00BF00BF39E000BF94F802
:108780003400032807D143463A4621463046009537
:1087900000F031F800E0256416B12046FFF7A0FF95
:1087A000204600F073F900203434A070607004F8A3
:1087B00034091DE000BF94F83400032807D1434674
:1087C0003A4621463046009500F015F800E0256451
:1087D000204600F04FFB16B12046FFF781FF042032
:1087E0003434A0700020607004F8340900E000BF49
:1087F00000BFBDE8F883F0B50446059E086BCD8F39
:108800000AE0C768A74204D1046142610383C661DC
:1088100004E020306F1EBDB2002DF2DC00BFF0BDC1
:1088200070B50025074C03E005F12000C5B2241DFA
:1088300020680028F8D02068F7F79DFD2844C5B2CD
:10884000284670BD90070020002004E00021034A64
:1088500042F82010401C0028F8D0704790070020F4
:1088600030B5420900F01F030121C3F11F04A140EC
:10887000034C54F822400C43014D45F8224030BDD2
:108880009007002030B5420900F01F030121C3F119
:108890001F04A140034C54F822408C43014D45F87D
:1088A000224030BD9007002000210AE001EB410288
:1088B000054B03EB820000220281026042604A1CE9
:1088C000D1B21029F2D3704750DC002010B5044615
:1088D00094F83700FFF7C4FF94F83700054909788A
:1088E000884203D1204600F027F802E0204600F03D
:1088F00003F810BD9A07002010B590F8373003EB4D
:1089000043030C4C04EB83010B893BB901230B811E
:108910000023C36003610860486009E00B895B1CA9
:108920000B810B68C360002303610A681061086053
:1089300010BD000050DC002010B590F8373003EB7C
:1089400043030B4C04EB83010B893BB901230B81DF
:108950000023C36003610860486008E00B895B1C6A
:108960000B810023C3604A680261D060486010BD7B
:1089700050DC00202DE9F041054695F8370000EB6A
:108980004000124901EB80042F69EE6887B946B9AF
:10899000002020812060606095F83700FFF772FFAB
:1089A0000EE02089401E208100203061266007E013
:1089B0002089401E2081FE600EB9676000E03761AB
:1089C00000202861E860BDE8F081000050DC002054
:1089D00038B504460D4685B16B460222294620462D
:1089E00000F06AF9BDF8000018B9032084F83600D9
:1089F00006E0022084F8360002E0022084F8360007
:108A00002046FFF7B7FF38BD0021034A1180034A13
:108A10001160018070470000A4070020A00700201B
:108A20000022026082604260C26002614261826133
:108A3000C26114A20262002242628262C2620264C5
:108A4000002106E0002300F15C0242F821304A1CBC
:108A5000D1B20029F6D000223430026142600263B4
:108A6000C26202814FF00042426100228261C26113
:108A7000026242620270427082701022C270343808
:108A8000704700003F5461736B00000010B504464E
:108A9000204600F0EFF994F8360000F0040010B919
:108AA0002046FFF713FF10BD08B506480068FFF722
:108AB00098FB00BF6A46002103480068FFF7ACFC42
:108AC000F8E70000B0070020305301082DE9F84313
:108AD0000446884617461D464FF0000900BF00BFF8
:108AE000F7F73EFC814600BF00BF0CB96748046839
:108AF00027640020288094F83600082876D2DFE822
:108B000000F0040550510607525300BF00BF00BFDC
:108B10000420012804D0022813D0042833D122E0F5
:108B2000606CFF280CD100BF00BF4846F7F71CFC63
:108B300000BF00BF46F6C55028800020BDE8F8837E
:108B400022E04FF6FF71606C88420BD100BF00BF7E
:108B50004846F7F709FC00BF00BF46F6C55028801D
:108B60000020EBE710E0606C401C58B900BF00BF6C
:108B70004846F7F7F9FB00BF00BF46F6C55028800E
:108B80000020DBE700E000BF00BF606C401C6064B9
:108B9000666C00BF00BF4846F7F7E6FB00BF00BFAA
:108BA00071E000BF00BF00BF94F83400072815D162
:108BB00000231A46214618460097FFF7CAFD666C47
:108BC00000BF00BF4846F7F7CFFB00BF00BF08F467
:108BD000004000284AD1FFF7F5F947E004200128BA
:108BE00005D0022813D0042833D122E03FE0606C86
:108BF000FF280BD100BF00BF4846F7F7B5FB00BF09
:108C000000BF46F6C5502880002097E722E04FF6C7
:108C1000FF71606C88420BD100BF00BF4846F7F778
:108C2000A3FB00BF00BF46F6C5502880002085E7A3
:108C300010E0606C401C58B900BF00BF4846F7F711
:108C400093FB00BF00BF46F6C5502880002075E7A3
:108C500000E000BF00BF606C401C6064666C00BF39
:108C600000BF4846F7F780FB00BF00BF0BE000BF26
:108C700000BF4846F7F778FB00BF00BF46F62D60FF
:108C80002880002600BF00BF304657E7B00700200D
:108C9000002108E0064A02EBC10000220260828047
:108CA000C2804A1C91B2034A12889142F2DB70479B
:108CB00068DB0020485301082DE9F04F0C461646AA
:108CC0001D46042E1ED1DFF8A091D9F80090A4EB28
:108CD0000909A9F1010313F5803F0DD94FF00009EF
:108CE000C0F84C90C0F85090C0F81C9047F27E2914
:108CF000A5F80090BDE8F08FC46403F10109C0F845
:108D000050903FE084B3082E25D1D0F8489009EB6D
:108D10000407DFF85491D9F80090A7EB0909A9F1ED
:108D20000103A34201D2C76406E0DFF83C91D9F801
:108D30000090A144C0F84C90DFF82CA1D0F84C90E2
:108D4000DAF800A0A9EB0A09C0F85090D0F84C90CE
:108D5000C0F8489016E0DFF81091D9F80090A144CF
:108D6000C0F84C9004650DE0FFE74FF00009C0F833
:108D70004C90C0F85090C0F81C9047F27E29A5F89E
:108D80000090B7E7DFF8E4A0BAF800A0D0F84C9064
:108D9000B9FBFAFB0AFB1B991FFA89F8DFF8D090A0
:108DA00009EBC802B2F80490B9F1000F0BD14FF0F3
:108DB0000009C0F81490C0F8189010604FF0010935
:108DC000A2F804903EE0116834E0DFF89CA0D1F8EE
:108DD0004C90DAF800A0A9EB0A09C1F85090D0F83D
:108DE0005090D1F850A0D1450ED9D1F81490B9F1D6
:108DF000000F01D049691DE04FF00009C0F8149040
:108E000081614861002115E0D1F81890B9F1000F97
:108E100007D14FF00009C0F81890416188611060D7
:108E200007E0D1F818C0C0F818C04161CCF81400B0
:108E3000886100210029C8D1B2F8049009F1010924
:108E4000A2F80490B2F80690B2F804A0D14503DA73
:108E5000B2F80490A2F80690C2614FF00009A5F89C
:108E6000009000BF46E70000A80700204853010813
:108E700068DB002010B5C269BAB10024046514682B
:108E8000844205D14169116039B100248C6104E04C
:108E9000816943694B6103B1996100244461846134
:108EA000C461C4649488641E948010BD2DE9F05F91
:108EB0004FF0000B00BF00BFF7F752FA834600BF28
:108EC00000BF4FF0000A50480068401C4E4908603F
:108ED000084600684D490988B0FBF1F201FB120019
:108EE0001FFA80F94A4800EBC9073C68002678E081
:108EF000002C75D0D4F8148094F8360008286BD272
:108F0000DFE800F00408051B0638074B00BF00BF70
:108F100000BF62E03C49E06C0968401A20653A49AC
:108F2000E06C0968884206D1002084F836002046AB
:108F3000FFF7ACFD00E001264FE03349E06C096823
:108F4000401A20653049E06C0968884210D1002041
:108F500020642046FFF7C4FB2046FFF797FD002062
:108F60003434A07003206070002004F8340900E05D
:108F7000012632E02449E06C0968401A2065224944
:108F8000E06C0968884206D1042084F83600204647
:108F9000FFF770FF00E001261FE01B49E06C096845
:108FA000401A20651849E06C0968884210D10020F9
:108FB00020642046FFF794FB2046FFF75BFF042068
:108FC0003434A07003206070002004F8340900E0FD
:108FD000012602E004E0FFE700BF00BF444600E0D6
:108FE0000126002E84D0CAF100050A480068A84274
:108FF00001D20848056000BF00BF5846F7F7B4F932
:1090000000BF00BFBDE8F09FA8070020485301083B
:1090100068DB0020AC0700201CB500BF0EE001ABF0
:109020006A4600210846FFF7DDF8BDF8040028B9BC
:1090300003480078012801D1FFF738FFEFE700006F
:109040009907002010B58AB0044600201D49086029
:109050001D490860FFF71CFE1C48006820B947F254
:10906000122020800AB010BD19480068194909680B
:10907000884203D247F213202080F3E71648007895
:109080000F2803D347F211202080EBE70B200021AB
:1090900005910A46CDE9070406910D4800680F497D
:1090A00009680A4B1B68CDE90131CDE903020A4882
:1090B000007800230A4A0BA100900F48FEF7FCFF3E
:1090C00000BFCFE7A8070020AC07002038530108F5
:1090D000405301082C530108345301083C53010844
:1090E0001990000875432F4F532D49494920546961
:1090F000636B205461736B0010DD002030B50546B2
:109100000C461CB1284601F0BBF802E0284601F0ED
:1091100013FF30BD0FB438B5002400BF05A8009080
:109120000548009A0499F7F731F9044600200090A9
:10913000014838BC5DF814FB3418012030B52DED22
:10914000108B87B0B0EE40AAF0EE60AAB0EE41BA44
:10915000F0EE61BAB0EE428AF0EE628AB0EE439A67
:10916000F0EE639AB0EE44CAF0EE64CAB0EE45DAAF
:10917000F0EE65DA53EC182B51EC1A0B0BF0BEFE37
:1091800041EC1F0B0BF096F9054653EC192B51ECF3
:109190001B0B0BF0B3FE41EC1F0B0BF08BF90446DD
:1091A00028460BF095FF41EC1F0B53EC192B51ECAB
:1091B0001D0B0BF0A3FE53EC1F2BCDE900019DED21
:1091C000000B51EC100B0BF08DFCCDE90401204697
:1091D0000BF07EFF41EC1F0B53EC182B51EC1C0BDA
:1091E0000BF08CFE53EC1F2BCDE900019DED000B25
:1091F00051EC100B0BF076FCCDE902019DED040B58
:1092000053EC102B9DED020B51EC100B0BF076FE86
:1092100041EC1E0B9FED0D0B53EC102B51EC1E0B74
:109220000BF05EFD05D24FF0FF3007B0BDEC108BA8
:1092300030BD9FED060B53EC102B51EC1E0B0BF0C9
:1092400015FC01D20120F0E70020EEE7000000004D
:10925000000000002DE9F0472DED0E8B88B004468C
:109260000025002600279FED9B0AB0EE408A9FED67
:10927000990AF0EE408A9FED970A10EE108A9FED52
:10928000950AB0EE409A9FED930AF0EE409A9FED5A
:10929000910A10EE10AA904890ED010AB5EEC00AAE
:1092A000F1EE10FA08D18D4890ED010AB5EEC00A32
:1092B000F1EE10FA00D100E001278949086A0BF0AD
:1092C000AAFB41EC1E0B9FED870B53EC102B0BF010
:1092D000DFF941EC1D0BB0EE4D0AF0EE6D0A03F024
:1092E0000BFEB0EE40BAF0EE60BA7B4890ED020A99
:1092F000DFED7E0A80EE201A11EE109A48460BF040
:10930000E7FE41EC1C0B53EC1B2B0BF0EBFB41EC91
:109310001A0B0BF0CFF808EE100A7549086A0BF02B
:109320007AFB41EC1E0B9FED6F0B53EC102B0BF0F7
:10933000AFF941EC1D0BB0EE4D0AF0EE6D0A03F0F3
:10934000DBFDB0EE40BAF0EE60BA644890ED020A80
:10935000DFED660A80EE201A11EE109A48460BF0F7
:10936000B7FE41EC1C0B53EC1B2B0BF0BBFB41EC91
:109370001A0B0BF09FF808EE900A38EE280AF0EE70
:10938000000A80EE201A11EE108A5549086A0BF087
:1093900042FB41EC1E0B9FED530B53EC102B0BF0DB
:1093A00077F941EC1D0BB0EE4D0AF0EE6D0A04F0BA
:1093B000A3FCB0EE40BAF0EE60BA474890ED020A66
:1093C000DFED4A0A80EE201A11EE109A48460BF0A3
:1093D0007FFE41EC1C0B53EC1B2B0BF083FB41EC91
:1093E0001A0B0BF067F809EE100A4149086A0BF0F6
:1093F00012FB41EC1E0B9FED3B0B53EC102B0BF0C3
:1094000047F941EC1D0BB0EE4D0AF0EE6D0A04F089
:1094100073FCB0EE40BAF0EE60BA304890ED020A4C
:10942000DFED320A80EE201A11EE109A48460BF05A
:109430004FFE41EC1C0B53EC1B2B0BF053FB41EC90
:109440001A0B0BF037F809EE900A39EE290AF0EE04
:10945000000A80EE201A11EE10AA50460BF038FEDA
:1094600041EC1A0B40460BF033FE41EC1B0B002085
:109470000122CDE904209FED1F0BCDE906708DED93
:10948000020B8DED00AB53EC1B2B1CA12046F6F715
:109490008FFF22490870012504E0605D3044C6B2A8
:1094A000681C05B21D480078401EA842F5DC1B4927
:1094B0000978601832461AA1F6F77AFF1749097839
:1094C0000844164908700846007808B0BDEC0E8BB9
:1094D000BDE8F08700000000181701206817012080
:1094E000401701206666666666A64C4000007A4416
:1094F000901701207B14AE47E17A943F24252E3348
:10950000662C252E33662C252E33662C25642C25BF
:10951000642C25642C25642A00000000481A0020D1
:1095200025303258230D0A0010B504461048008833
:10953000642802DD00200E4908802078242802D10A
:1095400000200B4908802178094802880088401CC7
:10955000074B1880074881542078232807D11846E4
:109560000188044800F008F800200149088010BD77
:109570006C1A0020701601202DE9F0412DED0A8BA8
:1095800094B004460E4601259FED9C0A8DED130A0A
:109590009FED9A0A8DED120A9FED980A8DED110A42
:1095A0009FED960A8DED100A9FED940A8DED0F0A3E
:1095B0009FED920A8DED0E0A4FF0000800200D90ED
:1095C0000C90012221468EA0F7F70AFA00287AD1E2
:1095D00000270B900BA88B498B4A8C4BCDE90632A8
:1095E000CDE908100EA810A90FAA0DABCDE90232E3
:1095F000CDE904100CA811A912AB13AACDE90010F3
:1096000083A1601CF7F784F80BE0605D3844C7B2B3
:10961000681CC5B2B54204DD14B0BDEC0A8BBDE8D0
:10962000F081605D2A28F0D19DF82C0087427AD124
:109630009DED130ADFED800A20EE200A7F4880EDC1
:10964000400A9DED120ADFED7C0A20EE200A80ED33
:10965000410A9DED110ADFED7A0AB4EEE00AF1EE5F
:1096600010FA07D89DED110ADFED760A30EE200AD8
:109670008DED110A9DED110ADFED730AB4EEE00ADB
:10968000F1EE10FA07DB9DED110ADFED6E0A30EE08
:10969000600A8DED110A9DED110A684880ED420ABD
:1096A0000C98C1B2654880F8FA100D98C1B26348B1
:1096B00080F8FB109DED0F0A80ED3F0A53480068CB
:1096C00010B1012101E097E000215C4880F89F1073
:1096D0004D48006808B1012100E00021574880F89A
:1096E000A0104848006808B1012100E0002153485B
:1096F00080F8A110554890ED000AB5EEC00AF1EED1
:1097000010FA58D0524890ED000ADDED120A9FED94
:109710004A1A10EE810A10EE101A08460BF0D8FC17
:1097200041EC1C0B00E066E09FED4A1BB0EE4C0ADA
:10973000F0EE6C0A03F0B8FCB0EE40AAF0EE60AABE
:10974000424890ED000ADDED130A9FED3B1A10EE42
:10975000810A10EE101A08460BF0BAFC41EC1C0B03
:109760009FED3C1BB0EE4C0AF0EE6C0A03F09CFC43
:10977000B0EE40BAF0EE60BA53EC1A2B51EC1B0B72
:109780000AF0CAFE41EC190BB0EE490AF0EE690A84
:1097900004F016FBB0EE408AF0EE608A9FED2F0BCE
:1097A00053EC102B51EC180B0BF09AFA03D24FF438
:1097B000805001F04FFB9DED100A2A4880ED010A10
:1097C0009DED0E0A80ED000A2748407F012809D14F
:1097D000254890ED040A2348D0ED010A30EE600AD6
:1097E00080ED020A1F4890ED010AD0ED020A30EE2A
:1097F000200A80ED010A00BF00BF0DE70000000055
:1098000024000000681A0020641A0020601A00205A
:1098100025662C25662C25662C25642C25642C2594
:10982000662C25662C25662C25642C25642C256445
:109830002A2530325823000000007A44641F022099
:10984000DA0F49C0DA0FC940DA0F4940581A002030
:109850005C1A002000000000000000400000000032
:1098600000406F40E01701202816012030B52DED93
:10987000068B91B004460D469FED760A8DED100AD9
:109880009FED740A8DED0F0A9FED720A8DED0E0AA1
:1098900000200D900C900B900A90099009A80AA93D
:1098A0000BAA0CABCDE90432CDE906100DA80EA928
:1098B0000FAA10ABCDE90032CDE90210664B674A22
:1098C00067A12046F6F724FF6448006842F20F7152
:1098D000884206D0614800686A4908605E480068AE
:1098E00048600B9801287DD19DED100ADFED660AD6
:1098F00030EE600A10EE101A08460BF0E9FB41EC5E
:10990000190B9FED620B53EC102B0BF0EBF841ECB5
:10991000180B0AF0CFFD5B49C8609DED0F0ADFED23
:109920005D0A30EE600A10EE101A08460BF0D0FB0C
:1099300041EC190B9FED550B53EC102B0BF0D2F8AB
:1099400041EC180B0AF0B6FD4E49886008464068A5
:1099500042F2BC5188420DD14A4800684E498842C3
:1099600008D1484890ED020AF3EE040A30EE200ACE
:1099700080ED020A4348406842F2BC5188420DD152
:109980004048006810F5E15F08D13E4890ED020ABA
:10999000F1EE040A30EE200A80ED020A3F4890ED15
:1099A0001F0ADDED0E0A30EE200A10EE101A0846EE
:1099B0000BF08EFB41EC190B9FED390B53EC102B88
:1099C0000AF066FE41EC180B0AF074FD2D4908619F
:1099D0000B980877344801680068401C324A1060D0
:1099E000142900E031E030DD0020114608600E98B7
:1099F0000BF06EFB41EC180B224890ED030A10EEC1
:109A0000101A08460BF064FB41EC190B1D4890ED51
:109A1000020A10EE101A08460BF05AFB41EC1A0B22
:109A20001848407F099A0B99CDE9061208908DEDF0
:109A3000048B8DED029B8DED00AB07480368074852
:109A40001A490268012002F08FF911B0BDEC068BB3
:109A500030BD00000000000088180020841800209D
:109A60003C256458592564402825667825662925B3
:109A7000664025784025784025642D25642D256491
:109A80003E000000281601200000C8433333333362
:109A90003333CB3F0000964390E8FFFF641F022062
:109AA0006666666666A64C40801800206857010806
:109AB00030B52DED088B91B004460D469FED710A2F
:109AC0008DED100A9FED6F0A8DED0F0A9FED6D0A67
:109AD0008DED0E0A00200D900C900B900A900990CD
:109AE00009A80AA90BAA0CABCDE90432CDE90610EE
:109AF0000DA80EA90FAA10ABCDE90032CDE90210D6
:109B0000614B624A62A12046F6F702FE0B980128DB
:109B10007ED19DED100A674880ED000A9DED0F0A89
:109B2000654880ED000A5948006864490860564855
:109B3000006848606249D1F888000AF06CFF41EC87
:109B4000190B9DED100ADFED5F0A30EE600AB1EEF1
:109B5000400A10EE101A08460BF0BAFA41EC1B0B43
:109B60009FED590B53EC102B0AF0BCFF41EC1A0B84
:109B700053EC192B0BF0C2F941EC180B0AF09AFCCC
:109B80004E49C8604E49D1F884000AF044FF41ECC8
:109B9000190B9DED0F0ADFED4E0A30EE600AB1EEB3
:109BA000400A10EE101A08460BF092FA41EC1B0B1B
:109BB0009FED450B53EC102B0AF094FF41EC1A0B70
:109BC00053EC192B0BF09AF941EC180B0AF072FCCC
:109BD0003A4988603A4890ED200ADDED0E0A30EEF1
:109BE000200AF7EE000A30EE600A10EE101A08465E
:109BF0000BF06EFA41EC190B9FED360B53EC102B6A
:109C00000AF046FD41EC180B0AF054FC2B4900E029
:109C100034E008610B980877304801680068401C00
:109C20002E4A1060322929DD0020114608600E9866
:109C30000BF04EFA41EC180B204890ED030A10EEA1
:109C4000101A08460BF044FA41EC190B1B4890ED32
:109C5000020A10EE101A08460BF03AFA41EC1A0B01
:109C60000B9806908DED048B8DED029B8DED00AB76
:109C700006481B490268012002F076F811B0BDECDD
:109C8000088B30BD000000009418002090180020C0
:109C90003C25645859256440282566782566292581
:109CA000664025784025784025642D25642D25645F
:109CB0003E000000781800207C1800204C1601207F
:109CC000641F02200000C843333333333333CB3FA8
:109CD000000096436666666666A64C408C180020B7
:109CE0001C57010830B591B0402201A9022000F0B4
:109CF000D9F90546A5B1002404E001A90819FFF728
:109D000013FC641CAC42F8D3002017490860002102
:109D1000164880F8F8104FF4005000F0DDFA20E00B
:109D200011480068401C1049086008460068B0F5FA
:109D3000FA7F16DB01210D4880F8F810480301F086
:109D400089F80B4801680068401C094A1060B1F5A9
:109D5000FA7F06DD00201146086006A1012002F00E
:109D600003F811B030BD0000701A0020641F0220FB
:109D7000741A0020BCA4B9E2B6A8CEBBB6AACAA782
:109D80002121210D0A00000010B5FBF771FB0449E9
:109D900091F8200004F0E8FF024807F0C3FD10BD71
:109DA000641F02207C20022008B5016800919DED0F
:109DB000000A08BD29B1064A12680243044B1A6022
:109DC00004E0034A12688243014B1A6070470000A6
:109DD0003038024029B1064A12680243044B1A6027
:109DE00004E0034A12688243014B1A607047000086
:109DF0004038024029B1064A12680243044B1A60F7
:109E000004E0034A12688243014B1A607047000065
:109E100044380240F0B5002100220024022500262B
:109E20000223324F3F6807F00C0121B1042905D00D
:109E3000082937D105E02E4F076036E02D4F076027
:109E400033E02A4F3F1F3F68C7F38056274F3F1F1D
:109E50003F6807F03F036EB1264FB7FBF3F7DFF81B
:109E60008CC0ACF1040CDCF800C0CCF3881C07FB00
:109E70000CF40CE01E4FB7FBF3F7DFF870C0ACF149
:109E8000040CDCF800C0CCF3881C07FB0CF4174F63
:109E90003F1F3F68C7F301477F1C7D00B4FBF5F708
:109EA000076002E0124F076000BF00BF0F4F3F681E
:109EB00007F0F0010909104F7A5C0768D740476046
:109EC0000A4F3F6807F4E051890A0B4F7A5C4768F4
:109ED000D7408760054F3F6807F46041490B064F44
:109EE0007A5C4768D740C760F0BD00000838024080
:109EF0000024F40000127A00CC05002030B503469F
:109F00000020054C234404E033F8015B0D54401C51
:109F10005B1C9042F8DB30BD00F8070870B50546C1
:109F20000024012D04D0022D05D0032D09D105E018
:109F300000F0A2FF08E000F0AFFF05E000F0BEFF78
:109F400002E000F099FF00BF00BF0220FBF79FFC7A
:109F50004FF480713648FBF73EFD012802D144F0F2
:109F6000010401E024F0010480213148FBF733FDB6
:109F7000012802D144F0020401E024F0020440214F
:109F80002B48FBF728FD012802D144F0040401E02E
:109F900024F0040420212648FBF71DFD012802D1EE
:109FA00044F0080401E024F0080410212048FBF7E5
:109FB00012FD012802D144F0100401E024F0100445
:109FC00008211B48FBF707FD012802D144F02004BB
:109FD00001E024F0200404211548FBF7FCFC0128D3
:109FE00002D144F0400401E024F040044FF4004169
:109FF0001048FBF7F0FC012802D144F0800401E096
:10A0000024F08004012D04D0022D05D0032D09D1A8
:10A0100005E000F029FF08E000F036FF05E000F061
:10A0200043FF02E000F020FF00BF00BF204670BDEC
:10A0300000180240000C024001460020024601299F
:10A040000DDB08290BDC481EC2B215480068104120
:10A0500000F0010008B1012070470020FCE7102942
:10A060000CDCA1F10900C2B20D484068104100F0BB
:10A07000010008B10120EFE70020EDE718290CDC12
:10A08000A1F11100C2B206488068104100F0010041
:10A0900008B10120E0E70020DEE700BFDCE70000B8
:10A0A000380F0120F0B503460C4615460022002665
:10A0B000012B01D1174911E0022B01D116490DE006
:10A0C000032B01D1154909E0042B01D1144905E006
:10A0D000062B01D1134901E00020F0BD002213E05E
:10A0E000B1F80008B1F80278B84200D10EE0761C51
:10A0F000B1F80208085CA054B1F80208401CC0F393
:10A100000900A1F80208521CAA42E9D300BF304658
:10A11000E3E70000ACE50020B4ED0020BCF5002032
:10A12000C4FD0020CC05012010B5C8223F49012004
:10A13000FFF7B8FF3E49087008460078002874DD34
:10A1400000203C4908702DE038483A490978405CC5
:10A15000AA2822D1354937480078401C085CAA2833
:10A160001BD134480078801C085CBB2815D13148CD
:10A170000078C01C085CBB280FD12E480078001D59
:10A18000085CCC2809D12B480078401D085CCC28FD
:10A1900003D10120284908700AE026480078401CB5
:10A1A0002449087023480078214909788842CBDB8C
:10A1B00000BF21480078C0B30020204908701AE091
:10A1C0001A481C490978405C1D491C4A1278885479
:10A1D00018480078401C1749087019481749097831
:10A1E000405C1849097808441649087013480078FB
:10A1F000401C12490870114800786328E0DB0B48C6
:10A200000C490978405C0E4981F8630008460078E3
:10A21000AA2807D1084690F86300EE2802D1012051
:10A220000949087000200449087010BD2E22022040
:10A23000142C0020102C0020152C0020112C0020A4
:10A2400098210220122C0020132C002010B500248D
:10A250000DE004EB8400074A02EBC0010648F6F764
:10A260008BFB10B9002005490855601CC4B2312C85
:10A27000EFDB10BD5C180120EC7A0120946C01200A
:10A28000002101280BDB082809DC421ED1B2114A4B
:10A29000126801238B401A430E4B1A6018E01028F5
:10A2A0000ADCA0F10902D1B20A4A536801228A40AD
:10A2B0001343084A53600BE0182809DCA0F111028F
:10A2C000D1B2044A926801238B401A43014B9A6031
:10A2D00070470000440F01200349D1F8C8108143A2
:10A2E000014AC2F8C8107047641F022010B52DED56
:10A2F0000C8BFE48B0F8720000EE100AB8EE400A6F
:10A30000DFEDFB0A80EE201AFA4890ED000A31EEEC
:10A31000000AB0EE408AF848807D01286CD0F648EB
:10A32000807D022868D0F5480078002842D1EF48A7
:10A3300090ED0C0AB5EEC00AF1EE10FA3AD090F8A2
:10A340002000032809D1E948807C30B10420EA4983
:10A3500088750120E94908704EE0E44890F8200033
:10A36000042809D1E148807C30B10320E249887596
:10A370000120E24908703FE0DC48407C032803D01C
:10A38000DA48007C032806D10420DB4988750120C7
:10A39000DA49087030E0D548407C042803D0D3481F
:10A3A000007C042828D10320D34988750120D34993
:10A3B000087021E0D048807DF0B9CC4890F82000AA
:10A3C000042819D0C94890F82000032814D0C748A1
:10A3D000407C042810D0C548407C03280CD0C348DA
:10A3E000007C042808D0C148007C032804D0002049
:10A3F000C2490870BD498874BC4890ED0C0AB5EE9E
:10A40000C00AF1EE10FA02D10020BB498875BA48A3
:10A4100090ED030ABA48D0ED000A30EE600AB94860
:10A4200080ED000A90ED000ADFEDB70AB4EEE00A15
:10A43000F1EE10FA07DD90ED000ADFEDAD0A30EE27
:10A44000600A80ED000AAF4890ED000ADFEDAF0A28
:10A45000B4EEE00AF1EE10FA07D290ED000ADFED5B
:10A46000A40A30EE200A80ED000AA04890ED0C0A04
:10A4700010EE101A08460AF02BFE41EC1B0BA14807
:10A4800000680AF025FE41EC1D0BB0EE4D0AF0EE1F
:10A490006D0A02F095FDB0EE40CAF0EE60CA53ECD2
:10A4A0001B2B51EC1C0B0AF029FD41EC1A0BB0EEF2
:10A4B0004A0AF0EE6A0A02F083FDB0EE409AF0EE2E
:10A4C000609A51EC190B09F0F5FF914908608A4830
:10A4D000807D01280BD08848807D022807D08648DF
:10A4E000807D032803D08448807D042841D188489A
:10A4F00090ED000AF3EE0E0AB4EEE00AF1EE10FA67
:10A5000003DD844880ED008A21E0814890ED000A57
:10A51000F0EE080AB4EEE00AF1EE10FA11DDB0EE4A
:10A52000482A7D48D0ED001AB3EE0E1AF0EE080A64
:10A53000774890ED000A07F0CDF9764880ED000AE3
:10A5400005E0754890ED000A724880ED000A7148F8
:10A5500000680AF0BDFD41EC1A0B9FED700B53EC47
:10A56000102B0AF0BFFA41EC190B09F0A3FF69495F
:10A5700008606148807D05287CD2DFE800F0030E8A
:10A580004685F6009FED670A5B4880ED010A90ED75
:10A59000030A5B4880ED000A67E15E4800680AF044
:10A5A00097FD41EC1A0B9FED600B53EC102B0AF05A
:10A5B00099FA41EC190B09F07DFF4F4948605C485E
:10A5C00000680AF085FD41EC190B514800680AF05B
:10A5D0007FFD41EC1B0BB0EE4B0AF0EE6B0A02F074
:10A5E000EFFCB0EE40AAF0EE60AA53EC192B51EC50
:10A5F0001A0B0AF03BFA07D89FED4A0A3E4880ED55
:10A60000010A00203C4988752FE1424890ED000A7C
:10A61000B1EE400A10EE100A0AF05AFD41EC190B97
:10A620009FED410B53EC102B0AF05CFA41EC1A0B36
:10A6300009F040FF304948603D4800680AF048FD95
:10A6400041EC190B324800680AF042FD41EC1B0B4B
:10A65000B0EE4B0AF0EE6B0A02F0B2FCB0EE40AA8C
:10A66000F0EE60AA53EC192B51EC1A0B0AF0FEF92C
:10A6700009D800E0F8E09FED2B0A1F4880ED010AA1
:10A6800000201D498875F0E0224800680AF020FD8E
:10A6900041EC1A0B9FED240B53EC102B0AF022FA1D
:10A6A00041EC190B09F006FF13494860184890ED7A
:10A6B000000AF1EE040AB4EEE00AF1EE10FA55D207
:10A6C000084690ED030AFAEE040AB4EEE00AF1EE51
:10A6D00010FA4BDD90ED030AF2EE040AB4EEE00A44
:10A6E000F1EE10FA42D2012024E00000641F0220A3
:10A6F0000000B443582100200C18012094210020B0
:10A70000842100208C21002000003443000034C349
:10A7100088210020642100205C210020A4703D0AD3
:10A72000D7A3D83F00000000CDCCCCAC6A6E594115
:10A7300060210020FFF780FC04460220FFF77CFC2C
:10A7400004404CB31FED090A514880ED010A002076
:10A750004F4988751FED0D0A084680ED030A1FED6D
:10A760000F0A4C4880ED000A16E016E04A4890EDCA
:10A77000000AF2EE040AB4EEE00AF1EE10FA0BD28F
:10A780000220FFF759FC38B11FED1A0A404880ED4E
:10A79000010A00203E49887567E0404890ED000AB4
:10A7A000B1EE400A10EE100A0AF092FC41EC190BCF
:10A7B0001FED230B53EC102B0AF094F941EC1A0B0C
:10A7C00009F078FE32494860334890ED000AF1EE16
:10A7D000040AB4EEE00AF1EE10FA2ED2084690ED2B
:10A7E000030AFAEE040AB4EEE00AF1EE10FA24DDF0
:10A7F00090ED030AF2EE040AB4EEE00AF1EE10FA6C
:10A800001BD20120FFF718FC04460220FFF714FCBE
:10A81000044044B31FED3D0A1D4880ED010A0020AD
:10A820001B4988751FED410A084680ED030A1FED9C
:10A83000430A184880ED000A15E0174890ED000A19
:10A84000F2EE040AB4EEE00AF1EE10FA0BD20220A6
:10A85000FFF7F2FB38B11FED4D0A0D4880ED010AFC
:10A8600000200B49887500E000BF00BF0C4890F83D
:10A87000DD0048B10648807D18B900200449886190
:10A8800002E0012002498861BDEC0C8B10BD000084
:10A890000C18012084210020882100206421002040
:10A8A000641F022021B1028842F04002028004E0CD
:10A8B00002884FF6BF731A4002807047024600209C
:10A8C00013890B400BB1012000E0002070470146C6
:10A8D000888970478181704710B50022028802F490
:10A8E00041520B884C8823438C882343CC882343D4
:10A8F0000C8923434C8923438C892343CC892343EC
:10A900001A430280838B4FF2FF74234083830B8AA8
:10A91000038210BD7047000000B52DED048B99B087
:10A92000AA208DF8000000208DF80100DA4890F888
:10A9300010018DF80200D84890F826008DF80B0021
:10A94000D548807E8DF80C00D34890F820008DF813
:10A950000D00D14890F8C8008DF80E00CE4890ED5B
:10A960003F0ABDEEC00A10EE100AC0B28DF80F000B
:10A97000C94890F8F9008DF81000C74890F8100108
:10A980008DF81100C448007E8DF8120000208DF86B
:10A9900013008DF814008DF815008DF816008DF851
:10A9A00017008DF81800BC48B0F86400000A8DF854
:10A9B0001900B94890F864008DF81A00B74890ED76
:10A9C000040ABDEEC00A10EE100A000A8DF81B0042
:10A9D000B24890ED040ABDEEC00A10EE100AC0B2F3
:10A9E0008DF81C00AD4890ED070ABDEEC00A10EED0
:10A9F000100A000A8DF81D00A84890ED070ABDEE68
:10AA0000C00A10EE100AC0B28DF81E0000208DF8AA
:10AA10001F008DF820008DF821008DF822009E483F
:10AA200090ED3F0ABDEEC00A10EE100AC0B28DF8DC
:10AA3000230000208DF824008DF825008DF82600D5
:10AA40008DF8270001208DF828009348B0F8C80041
:10AA5000000A8DF82900904890F8C8008DF82A0067
:10AA60008D48D0F8C800000E8DF82B008A48D0F829
:10AA7000C800000C8DF82C00874890ED420A10EEBB
:10AA8000101A08460AF024FB41EC190B9FED840BC9
:10AA900053EC102B0AF026F841EC180B09F00AFDD4
:10AAA0008149086008460088000A8DF82D00084694
:10AAB00000788DF82E0008464088000A8DF82F0097
:10AAC000084680788DF83000734890ED400A0846BB
:10AAD00080ED000A0088000A8DF8310008460078F1
:10AAE0008DF8320008464088000A8DF83300084689
:10AAF00080788DF83400684890ED410A084680ED72
:10AB0000000A0088000A8DF83500084600788DF8A4
:10AB1000360008464088000A8DF8370008468078DD
:10AB20008DF83800614890ED000A084680ED000A73
:10AB30000088000A8DF83900084600788DF83A0040
:10AB400008464088000A8DF83B00084680788DF85A
:10AB50003C00564890ED010A084680ED000A008846
:10AB6000000A8DF83D00084600788DF83E00084642
:10AB70004088000A8DF83F00084680788DF8400034
:10AB80004B4890ED000A084680ED000A0088000A54
:10AB90008DF84100084600788DF84200084640884C
:10ABA000000A8DF84300084680788DF8440040483C
:10ABB00090ED010A084680ED000A0088000A8DF831
:10ABC0004500084600788DF8460008464088000A8F
:10ABD0008DF84700084680788DF848002F4890EDA2
:10ABE000010A084680ED000A0088000A8DF8490035
:10ABF000084600788DF84A0008464088000A8DF81B
:10AC00004B00084680788DF84C00244890ED000AEF
:10AC1000084680ED000A0088000A8DF84D000846BD
:10AC200000788DF84E0008464088000A8DF84F00E5
:10AC3000084680788DF850001E480088000A8DF87C
:10AC400051001C4800788DF852001A480068000E28
:10AC50008DF8530017480068000C8DF85400154813
:10AC60008088000A8DF85500124800798DF856004A
:10AC700010484068000E8DF857000E484068000CE0
:10AC80008DF8580064226946012001F085FB19B057
:10AC9000BDEC048B00BD0000641F02209420022044
:10ACA0006666666666A64C40FC1100202C210220D8
:10ACB000382102202816012010B5124890F83C0EC9
:10ACC00080B1012819D11048FBF700F800B110BD80
:10ACD00014210E48F5F752FF0D4A0EA10B48F5F767
:10ACE00067FB0BE00848FAF7F1FF00B1EFE70A480D
:10ACF000007908B1F8F766FE00E000BF00BF00BFB2
:10AD0000E5E70000D002022020B00120EC7A01200B
:10AD100068B8012025730000641F022070B5044646
:10AD20000D46012D04D0022D05D0032D09D105E0DB
:10AD300000F0CEF808E000F0DBF805E000F0E8F8FD
:10AD400002E000F0C5F800BF00BF04F0010028B128
:10AD50004FF480513C48FAF749FE04E04FF480512B
:10AD60003948FAF741FE04F0020028B14FF40051CF
:10AD70003548FAF73BFE04E04FF400513248FAF749
:10AD800033FE04F0040028B14FF480412E48FAF756
:10AD90002DFE04E04FF480412B48FAF725FE04F025
:10ADA000080028B14FF400412748FAF71FFE04E0DD
:10ADB0004FF400412448FAF717FE04F0100020B1C8
:10ADC00001212248FAF712FE03E001211F48FAF799
:10ADD0000BFE04F0200020B102211C48FAF706FE09
:10ADE00003E002211948FAF7FFFD04F0400020B10A
:10ADF00080211748FAF7FAFD03E080211448FAF79A
:10AE0000F3FD04F0800028B14FF480711048FAF788
:10AE1000EDFD04E04FF480710D48FAF7E5FD012DDA
:10AE200004D0022D05D0032D09D105E000F058F81B
:10AE300008E000F065F805E000F074F802E000F0CA
:10AE40004FF800BF00BF70BD001402400018024060
:10AE5000001002400349D1F8C8100143014AC2F86A
:10AE6000C8107047641F022010B502210148FAF78C
:10AE7000BDFD10BD0010024010B502210148FAF7D7
:10AE8000B3FD10BD0010024010B501210148FAF7D2
:10AE9000ADFD10BD0010024010B501210148FAF7C8
:10AEA000A3FD10BD0010024010B54FF40071024820
:10AEB000FAF79CFD10BD00000004024010B54FF4ED
:10AEC00000710248FAF790FD10BD00000004024036
:10AED00010B501210148FAF789FD10BD00040240B8
:10AEE00010B501210148FAF77FFD10BD00040240B2
:10AEF00010B502210148FAF779FD10BD00040240A7
:10AF000010B502210148FAF76FFD10BD00040240A0
:10AF100010B54FF400610248FAF768FD10BD00005B
:10AF20000014024010B54FF400610248FAF75CFDCE
:10AF300010BD000000140240002101280BDB08288E
:10AF400009DC421ED1B2114A126801238B409A4398
:10AF50000E4B1A6018E010280ADCA0F10902D1B2E9
:10AF60000A4A536801228A409343084A53600BE01F
:10AF7000182809DCA0F11102D1B2044A9268012319
:10AF80008B409A43014B9A6070470000440F0120A8
:10AF900010B54FF480710248FAF726FD10BD00008D
:10AFA0000008024010B54FF480710248FAF71EFD08
:10AFB00010BD0000000802400CB500200190009078
:10AFC0003448006840F480303249086000BF31489E
:10AFD000006800F4003000900198401C0190009837
:10AFE00018B90198B0F5A04FF1D12A48006800F4D3
:10AFF000003010B10120009001E000200090009886
:10B00000012846D123484030006840F08050214953
:10B01000403108602048006840F440401E49086004
:10B020001C48083000681B49083108600846006861
:10B0300040F4004008600846006840F4A0500860F2
:10B040001648091F0860081F006840F08070091F3B
:10B05000086000BF0F48006800F000700028F9D0B9
:10B0600040F205700E4908600A480830006820F078
:10B0700003000849083108600846006840F00200F3
:10B08000086000BF03480830006800F00C00082882
:10B09000F8D10CBD00380240007000400854400751
:10B0A000003C024010B500F03BFEFEF71BFE10BD59
:10B0B00010B507F00FFF08F0A7FD08F00BFE0949D7
:10B0C000094807F0F7FD0949094807F0DFFD07F0D7
:10B0D00021FF08F071FB08F0BFFB0649064809F0A4
:10B0E000CAF810BDA13C01086D3C010841FD0008F3
:10B0F00051FD0008060B0020020B00209FED0A0AFC
:10B100000A4981ED010A9FED080A094981ED010A0A
:10B110009FED050A074981ED010A9FED030A0649E3
:10B1200081ED010A7047000000000000181701209F
:10B1300068170120EC1701200C180120DFED050A2B
:10B140000548C0ED010ADFED030A0448C0ED010A1D
:10B150007047000000000000181701206817012048
:10B1600010B51548006840F4700013490860134892
:10B17000006840F001001149086000200F490831C3
:10B1800008600E4800680E4908400C4908600D48E8
:10B19000091D0860081F006820F48020091F08604E
:10B1A000002006490C310860FFF706FF4FF00060F1
:10B1B00001498039086010BD88ED00E00038024088
:10B1C000FFFFF6FE1030002410B50121054800F005
:10B1D0004EF828B10121034800F046F807F0E4FBDF
:10B1E00010BD00000004004010B5002400BF00BFE7
:10B1F000F5F7B6F8044600BF00BFFCF767FE00BFD6
:10B2000000BF2046F5F7B0F800BF00BF0121054898
:10B2100000F02DF818B10121024800F025F8FCF7E4
:10B220006BFE10BD0008004010B5002400BF00BF39
:10B23000F5F796F8044600BF00BFFCF747FE00BFD5
:10B2400000BF2046F5F790F800BF00BF0121054878
:10B2500000F00DF818B10121024800F005F8FCF7E4
:10B260004BFE10BD00140040CA430282704730B547
:10B270000246002000230024158A05EA010395896F
:10B2800005EA010413B10CB1012000E0002030BD3B
:10B2900010B52DED060B2DED0A8B9DED0B0ADDEDA6
:10B2A0000E0A30EE600A10EE101A084609F010FF80
:10B2B00041EC1C0B9FED201BB0EE4C0AF0EE6C0A2B
:10B2C00001F0F2FEB0EE40AAF0EE60AA9DED0A0A8F
:10B2D000DDED0D0A30EE600A10EE101A084609F096
:10B2E000F7FE41EC1C0B9FED141BB0EE4C0AF0EE88
:10B2F0006C0A01F0D9FEB0EE40BAF0EE60BA53EC41
:10B300001A2B51EC1B0B09F007F941EC190BB0EEAD
:10B31000490AF0EE690A02F053FDB0EE408AF0EE01
:10B32000608A51EC180B09F0C5F800EE100ABDEC6C
:10B330000A8B06B010BD00000000000000000040B5
:10B3400008B5014608880090BDF8000008BD014618
:10B35000086870472DE9F0410026002700BF00BFB4
:10B36000F4F7FEFF074600BF00BFFCF7AFFD00BFCC
:10B3700000BF3846F4F7F8FF00BF00BF40F2255188
:10B38000694800F009FCE0B10126674800F0BEFC06
:10B39000C4B26648B0F80008401CC0F30900634915
:10B3A000B1F8021888420CD06048B0F800085F4934
:10B3B0000C540846B0F80008401CC0F30900A1F87E
:10B3C000000840F22771584800F0E6FB38B35748B0
:10B3D000B0F804085549B1F80618884212D053480D
:10B3E000B0F80658B0F80608401CC0F309004F49F1
:10B3F000A1F8060801F58060445D21464A4800F046
:10B400008AFC51E0002240F22771474800F0EEFB31
:10B41000012240F22661444800F0E8FB44E040F29B
:10B420002661414800F0B8FB08B34048B0F8040872
:10B430003E49B1F80618884212D03C48B0F8065888
:10B44000B0F80608401CC0F309003849A1F8060806
:10B4500001F58060445D2146334800F05CFC23E048
:10B46000002240F22661304800F0C0FB1CE0DEB94B
:10B470002D4800F04BFCC4B22C48B0F80008401C2A
:10B48000C0F309002949B1F8021888420CD02748B6
:10B49000B0F8000825490C540846B0F80008401CD4
:10B4A000C0F30900A1F800083C2C06D10020204977
:10B4B000086001201F49086008E03E2C06D11D48A5
:10B4C0000068012802D102201A4908601848006863
:10B4D0006E2804DD002017490860154908601548EA
:10B4E0000068012808D1124801680068401C104A11
:10B4F00010601148445413E00E48006802280FD130
:10B500000B4801680068401C094A10600A4844540E
:10B51000002008490860012008494877642088779E
:10B52000FCF7EAFCBDE8F081004C0040C4FD0020BF
:10B53000B80E0020B40E0020780E01204C16012019
:10B540002DE9F041002640F22551564800F024FB39
:10B55000074600BF00BFF4F703FF064600BF00BF69
:10B56000FCF7B4FC00BF00BF3046F4F7FDFE00BF9F
:10B5700000BF40F225514B4800F00EFBD8B14948BE
:10B5800000F0C4FBC5B24848B0F80008401CC0F346
:10B5900009004549B1F8021888420CD04248B0F879
:10B5A000000841490D540846B0F80008401CC0F39B
:10B5B0000900A1F8000840F227713A4800F0ECFABF
:10B5C00038B33948B0F804083749B1F8061888424A
:10B5D00012D03548B0F80648B0F80608401CC0F351
:10B5E00009003149A1F8060801F58060055D29468A
:10B5F0002C4800F090FB50E0002240F227712948CF
:10B6000000F0F4FA012240F22661264800F0EEFA3A
:10B6100043E040F22661234800F0BEFA08B3224816
:10B62000B0F804082049B1F80618884212D01E4824
:10B63000B0F80648B0F80608401CC0F309001A49E3
:10B64000A1F8060801F58060055D2946154800F05F
:10B6500062FB22E0002240F22661124800F0C6FAA6
:10B660001BE0104800F052FBC5B20F48B0F80008CC
:10B67000401CC0F309000C49B1F8021888420CD0F4
:10B680000948B0F8000808490D540846B0F8000809
:10B69000401CC0F30900A1F80008FCF72DFCBDE830
:10B6A000F081000000100140ACE500202DE9F041E0
:10B6B0000026002700BF00BFF4F752FE064600BF79
:10B6C00000BFFCF703FC00BF00BF3046F4F74CFEA0
:10B6D00000BF00BF40F225514E4800F05DFAE0B1D6
:10B6E00001274C4800F012FBC5B24B48B0F80008E7
:10B6F000401CC0F309004849B1F8021888420CD038
:10B700004548B0F8000844490D540846B0F8000810
:10B71000401CC0F30900A1F8000840F227713D4821
:10B7200000F03AFA38B33C48B0F804083A49B1F8A6
:10B730000618884212D03848B0F80648B0F8060813
:10B74000401CC0F309003449A1F8060801F58060E7
:10B75000055D29462F4800F0DEFA51E0002240F254
:10B7600027712C4800F042FA012240F22661294854
:10B7700000F03CFA44E040F22661264800F00CFA62
:10B7800008B32548B0F804082349B1F806188842E0
:10B7900012D02148B0F80648B0F80608401CC0F3A3
:10B7A00009001D49A1F8060801F58060055D2946DC
:10B7B000184800F0B0FA23E0002240F22661154854
:10B7C00000F014FA1CE0DFB9124800F09FFAC5B28D
:10B7D0001148B0F80008401CC0F309000E49B1F848
:10B7E000021888420CD00C48B0F800080A490D54E1
:10B7F0000846B0F80008401CC0F30900A1F8000892
:10B800002946064803F008FF05490870FCF774FB59
:10B81000BDE8F08100440040B4ED0020500F01204D
:10B820003C1500202DE9F0410026002700BF00BF95
:10B83000F4F796FD074600BF00BFFCF747FB00BFCB
:10B8400000BF3846F4F790FD00BF00BF40F225511D
:10B85000694800F0A1F9E0B10126674800F056FA06
:10B86000C4B26648B0F80008401CC0F30900634940
:10B87000B1F8021888420CD06048B0F800085F495F
:10B880000C540846B0F80008401CC0F30900A1F8A9
:10B89000000840F22771584800F07EF938B3574845
:10B8A000B0F804085549B1F80618884212D0534838
:10B8B000B0F80658B0F80608401CC0F309004F491C
:10B8C000A1F8060801F58060445D21464A4800F071
:10B8D00022FA51E0002240F22771474800F086F931
:10B8E000012240F22661444800F080F944E040F231
:10B8F0002661414800F050F908B34048B0F8040808
:10B900003E49B1F80618884212D03C48B0F80658B3
:10B91000B0F80608401CC0F309003849A1F8060831
:10B9200001F58060445D2146334800F0F4F923E0DE
:10B93000002240F22661304800F058F91CE0DEB9E0
:10B940002D4800F0E3F9C4B22C48B0F80008401CC0
:10B95000C0F309002949B1F8021888420CD02748E1
:10B96000B0F8000825490C540846B0F80008401CFF
:10B97000C0F30900A1F800083C2C06D100202049A2
:10B98000086001201F49086008E03E2C06D11D48D0
:10B990000068012802D102201A490860184800688E
:10B9A0006E2804DD00201749086015490860154815
:10B9B0000068012808D1124801680068401C104A3C
:10B9C00010601148445413E00E48006802280FD15B
:10B9D0000B4801680068401C094A10600A4844543A
:10B9E00000200849086001200849487764208877CA
:10B9F000FCF782FABDE8F08100480040BCF5002069
:10BA0000AC0E0020A80E0020000E012028160120F8
:10BA10002DE9F0410026002700BF00BFF4F7A0FC8D
:10BA2000074600BF00BFFCF751FA00BF00BF384611
:10BA3000F4F79AFC00BF00BF40F225514E4800F0D9
:10BA4000ABF8E0B101264C4800F060F9C5B24B48B4
:10BA5000B0F80008401CC0F309004849B1F80218CA
:10BA600088420CD04548B0F8000844490D540846B7
:10BA7000B0F80008401CC0F30900A1F8000840F22B
:10BA800027713D4800F088F848B33C48B0F80408F6
:10BA90003A49B1F80618884214D03848B0F8064838
:10BAA000B0F80608401CC0F309003449A1F80608A4
:10BAB00001F58060055DFFF775FA29462E4800F014
:10BAC0002AF955E0002240F227712B4800F08EF849
:10BAD000012240F22661284800F088F848E040F250
:10BAE0002661254800F058F828B32448B0F8040827
:10BAF0002249B1F80618884214D02048B0F8064808
:10BB0000B0F80608401CC0F309001C49A1F806085B
:10BB100001F58060055DFFF745FA2946164800F0FB
:10BB2000FAF825E0002240F22661134800F05EF8A2
:10BB3000FFF72EFA1CE0DEB90F4800F0E7F8C5B2B7
:10BB40000E48B0F80008401CC0F309000B49B1F8DA
:10BB5000021888420CD00948B0F8000807490D5473
:10BB60000846B0F80008401CC0F30900A1F800081E
:10BB7000FCF7C2F9BDE8F08100140140CC050120BA
:10BB800021B1828942F40052828104E082894DF61B
:10BB9000FF731A408281704770B50246002400236B
:10BBA0000025002040F66A16B14200D100BFC1F363
:10BBB000421501F01F03012606FA03F3012D02D1FD
:10BBC0009689334006E0022D02D1168A334001E007
:10BBD000968A33400C12012606FA04F41688344083
:10BBE00013B10CB1012000E0002070BDF0B5034698
:10BBF000002400260025002040F66A17B94200D133
:10BC000000BF1846C1F3421401F01F06012707FACE
:10BC100006F5012C01D10C3004E0022C01D11030CA
:10BC200000E014301AB107682F43076002E007688C
:10BC3000AF430760F0BD00002DE9FF4705460E4603
:10BC40000024A14600BFA046B08900B100BF2C8AE5
:10BC500024F44054F08804432C82AC8941F20C60F7
:10BC60008443B08831890843718908430443AC8117
:10BC7000AC8A24F44074B0890443AC826846FEF771
:10BC8000C9F82048854202D01F48854202D1DDF81C
:10BC90000C9001E0DDF80890A88900F4004040B164
:10BCA00009EBC90000EB091031684900B0FBF1F75E
:10BCB00007E009EBC90000EB091031688900B0FB0F
:10BCC000F1F76420B7FBF0F004012009642101FBC7
:10BCD0001078A88900F4004040B1322000EBC80081
:10BCE000B0FBF1F000F00700044308E0322000EB65
:10BCF00008106421B0FBF1F000F00F0004432C8128
:10BD0000BDE8FF870010014000140140014688880B
:10BD1000C0F308007047C1F308028280704700003A
:10BD200010B5E4B04FF4C8716846F4F727FF6846D1
:10BD3000FDF790FA04460A48D0F814010949096849
:10BD4000401A0C2809D30648D0F8140105490860A8
:10BD500022466946022000F01FFB64B010BD0000BF
:10BD6000641F02204C1A00207047000010B501200B
:10BD7000FEF7D4F8064908600220FEF7CFF8044920
:10BD800048600320FEF7CAF80149886010BD000032
:10BD9000380F012010B532240A4908780121FEF736
:10BDA000BDFF084908790221FEF7B8FF0549087A66
:10BDB0000321FEF7B3FF00BF201EA4F10104FBD155
:10BDC00010BD0000440F012000BFFEE770B504461F
:10BDD0000F49C86880470E49486980470C48016A86
:10BDE0000F2088470A48016AC4F307208847E0B259
:10BDF000074A116A88470649C869804705460449C9
:10BE000088698047024908698047284670BD00005C
:10BE10003C0B00202DE9F04105460E461746002454
:10BE20001349C86880471249486980471048016A29
:10BE30000F2088472A19C2F307200D4A116A884744
:10BE40002A19D0B20A4A116A884700BF05E008499A
:10BE5000C86980473055601C84B2BC42F7DB044996
:10BE600088698047024908698047BDE8F081000081
:10BE70003C0B002070B504460D460F49C86880474A
:10BE80000D49486980470C48016AF02088470A48F4
:10BE9000016AC4F307208847E0B2074A116A88475D
:10BEA0000548016A2846884703498869804702494E
:10BEB0000869804770BD00003C0B00202DE9F0416F
:10BEC00005460E46174600241349C86880471249A4
:10BED000486980471048016AF02088472A19C2F350
:10BEE00007200D4A116A88472A19D0B20A4A116AF6
:10BEF000884700BF05E0305D074A116A8847601C2B
:10BF000084B2BC42F7DB044988698047024908696A
:10BF10008047BDE8F08100003C0B00200020014973
:10BF200008607047082C004040F08001014A116011
:10BF300070470000002C0040012001490860704754
:10BF4000A4800542F8B506460C4615460121C802F4
:10BF5000FDF740FF1048007830400F490870284630
:10BF600000F024F8204600F02DF80B480078FFF789
:10BF7000DBFF00208DF800008DF801008DF8020035
:10BF800001208DF803006846FBF7CEFEFFF7C6FFE1
:10BF9000FFF7D2FFF8BD00006010002000F07F0125
:10BFA000014A116070470000002C00400021044A43
:10BFB000126822F4C0710143014A11607047000009
:10BFC000042C004008B5002100910749096821F0C0
:10BFD0007F01009100F07F01009A11430091024A15
:10BFE0000099116008BD0000042C004010B52DED33
:10BFF000048B0446E27A217B42EA0122617B42EA19
:10C000000142217B42EA01614FF4B47201FB02F06C
:10C0100008F001FD9FED060B53EC102B08F038FBE8
:10C0200008F0CAFC04490862BDEC048B10BD000096
:10C0300000000000009870404017012010B52DED61
:10C04000048B0446E27A217B42EA0122617B42EAC8
:10C050000142217B42EA01614FF4B47201FB02F01C
:10C0600008F0D9FC9FED060B53EC102B08F010FBE9
:10C0700008F0A2FC04490862BDEC048B10BD00006E
:10C08000000000000098704090170120C17B027CE6
:10C090001143427C1143827C0AB9012200E0002254
:10C0A000114311B101210D4A1170C17A01F00F0144
:10C0B000012901D1094A9161C17A01F00F010329D7
:10C0C00002D10221054A9161C17A01F00F010729CD
:10C0D00002D10321014A9161704700001817012025
:10C0E000C17B027C1143427C1143827C0AB901224C
:10C0F00000E00022114311B101211C4A1170C17AE4
:10C1000001F00F01012901D1184A9161C17A01F0B2
:10C110000F01032902D10221144A9161C17A01F071
:10C120000F01072908D11249097829B10021104AC5
:10C13000117003210D4A91610C498969032914D1B9
:10C140000C49097839B9017B0122B2EBE11F02D118
:10C150000421064A9161017BC911064A11701146FA
:10C16000097811B90021044A117070474017012065
:10C170007D0500207C05002060050020C17B027C3D
:10C180001143427C1143827C0AB9012200E0002263
:10C19000114311B101210D4A1170C17A01F00F0153
:10C1A000012901D1094A9161C17A01F00F010329E6
:10C1B00002D10221054A9161C17A01F00F010729DC
:10C1C00002D10321014A91617047000068170120E4
:10C1D000C17B027C1143427C1143827C0AB901225B
:10C1E00000E00022114311B101211C4A1170C17AF3
:10C1F00001F00F01012901D1184A9161C17A01F0C2
:10C200000F01032902D10221144A9161C17A01F080
:10C210000F01072908D11249097829B10021104AD4
:10C22000117003210D4A91610C498969032914D1C8
:10C230000C49097839B9017B0122B2EBE11F02D127
:10C240000421064A9161017BC911064A1170114609
:10C25000097811B90021044A117070479017012024
:10C260007F0500207E05002061050020C17B027C47
:10C270001143427C1143827C0AB9012200E0002272
:10C28000114311B101210D4A1170C17A01F00F0162
:10C29000012901D1094A9161C17A01F00F010329F5
:10C2A00002D10221054A9161C17A01F00F010729EB
:10C2B00002D10321014A916170470000B8170120A3
:10C2C000C27A017B42EA0122417B42EA0142017BC0
:10C2D00042EA0161494200EE101AB8EEC00A9FED31
:10C2E0000E1AC0EE010AB2EE040A80EE801ADFEDEB
:10C2F0000B0A81EE200AB3EE041AC0EE010A9FED8C
:10C30000080A20EE800ADFED070A20EE200A06491F
:10C3100081ED020A7047000000FF7F470000704275
:10C32000DA0F49400000204318170120C27A017B30
:10C3300042EA0122417B42EA0142017B42EA016179
:10C34000494200EE101AB8EEC00A9FED0E1AC0EE78
:10C35000010AB2EE040A80EE801ADFED0B0A81EECC
:10C36000200AB3EE041AC0EE010A9FED080A20EE7F
:10C37000800ADFED070A20EE200A064981ED020A55
:10C380007047000000FF7F4700007042DA0F49400D
:10C3900000002043681701202DE9F0470546894633
:10C3A0009246012D02D1274C274E15E0022D02D1D5
:10C3B000264C274E10E0032D02D1264C264E0BE0D2
:10C3C000042D02D1254C264E06E0062D02D1254C27
:10C3D000254E01E0BDE8F087B4F80408B4F806186B
:10C3E000884202D14FF0010801E04FF00008002719
:10C3F00019E0B4F80408401CC0F30900B4F80618AA
:10C4000088420ED019F80710B4F8042804F58060AB
:10C410008154B4F80408401CC0F30900A4F80408CF
:10C4200000E002E07F1C5745E3D300BFB8F1000FE6
:10C4300005D0012240F227713046FFF7D7FB00BF3D
:10C44000C8E70000ACE5002000100140B4ED00207A
:10C4500000440040BCF5002000480040C4FD00201E
:10C46000004C0040CC050120001401401CB5012106
:10C470005A20FDF79FFC4FF4FE70009002208DF8CB
:10C48000050001208DF8070000208DF806008DF8CA
:10C49000040069461148F9F733FA4FF40040009060
:10C4A00069460F48F9F72CFA0320009002208DF816
:10C4B000050001208DF8070000208DF806000120FE
:10C4C0008DF8040069460748F9F71AFA4FF400702E
:10C4D000009069460448F9F713FA1CBD00180240A1
:10C4E000000C0240001002400004024010B515206C
:10C4F000FDF7A2FDA2490870A24981F89C00162010
:10C50000FDF79AFD9E4948709E4981F89D001720CD
:10C51000FDF792FD9A4988709A4981F89E0006209D
:10C52000FDF78AFD80F0010095498871954981F8F1
:10C5300098001120FDF780FD934908701020FDF749
:10C540007BFD924908700820FDF776FD30B99048D0
:10C55000007818B101218B4880F8AB100820FDF756
:10C560006BFD8B490870874890F8AB0028B3002119
:10C57000844880F8AB100420FDF7AEFE814890F8A7
:10C5800020000B280AD101217E48807E401EC0EB8E
:10C59000C002804800EB8200C1810EE0794890F82B
:10C5A00020000C2809D102217648807E401EC0EB75
:10C5B000C002784800EB8200C1817748007858B902
:10C5C00071480078012807D16E48007908B9012028
:10C5D00000E000206B4908716B4800786E490870D4
:10C5E0006848007900286DD10D20FDF725FD6549CB
:10C5F00081F8A2000E20FDF71FFD624981F8A3001B
:10C6000062480078012810D16448007868B908466B
:10C6100090F8AC0048B9084690F8AD0008B901217F
:10C6200000E00021574880F8AD10584800785B4979
:10C630000870544890F8A20018B10120514988713F
:10C640000AE0504890F8A30018B102204D498871C3
:10C6500002E000204B4988710920FDF7EDFC4949B3
:10C6600081F8A4000A20FDF7E7FC464981F8A500FF
:10C670000B20FDF7E1FC434981F8A6000C20FDF7F3
:10C68000DBFC404981F8A7000F20FDF7D5FC3D49B0
:10C6900081F8A8001220FDF7CFFC3A4981F8A900E3
:10C6A0001820FDF7C9FC374981F8AA000220FDF7E0
:10C6B000C3FC344981F8CD00084690F8A40010B1BD
:10C6C0000120487132E02F4890F8A50018B10220EF
:10C6D0002C4948712AE02B4890F8A60018B1032095
:10C6E0002849487122E0274890F8A70018B1042093
:10C6F000244948711AE0234890F8A80018B1052091
:10C700002049487112E01F4890F8A90018B106208E
:10C710001C4948710AE01B4890F8AA0018B107208C
:10C720001849487102E00020164948710520FDF7BC
:10C7300083FC1349C871134981F89B000420FDF75D
:10C740007BFC0F4908730F4981F8B2000320FDF705
:10C7500073FC0B4948730B4981F8B300084690F805
:10C76000990018B10121074880F8CC10054890F8CD
:10C77000B30020B19FED0A0A0A4880ED030A10BDFC
:10C780003C1F0220641F02209621002099210020D6
:10C7900095210020CC6D0120972100209B210020B5
:10C7A00000000000EC1701201CB501217220FDF7EC
:10C7B00001FB4FF47040009002208DF8050001202D
:10C7C0008DF8070000208DF8060001208DF8040088
:10C7D00069460F48F9F794F80320009069460D4820
:10C7E000F9F78EF84FF4C070009069460A48F9F7DF
:10C7F00087F80320009069460848F9F781F84FF45C
:10C800000060009069460248F9F77AF81CBD000004
:10C8100000140240001802400010024000040240D0
:10C8200008B5244800782449097808402349097844
:10C83000084023490978084030B9002302222149E1
:10C840001846F7F787FA1DE006F0E2FC6A46082171
:10C850000220FBF7E1FD06F09FFD6A460821022059
:10C86000FBF7DAFD06F05CFE6A4608210220FBF7C2
:10C87000D3FD06F0FBFE6A4608210220FBF7CCFD43
:10C8800006F060FC1048007970B90F4890F8AC00D1
:10C890000D4991F8AD10084318B12B200A49487290
:10C8A00002E0012008494872074A117B507AFBF7E1
:10C8B00007FA08BD1817012040170120681701204A
:10C8C0009017012062050020641F022010B5FEF7BA
:10C8D000E9FB05F051FF0A49098888B206F004FA1D
:10C8E000FEF71AF8FDF720FC0649087EFAF7EAFA87
:10C8F0000449087EFAF7D0F9F6F758FC10BD00009D
:10C9000044030020641F022003B4019841000098F2
:10C9100050EAC12018BF04204A0D18BF40F00100A2
:10C9200040F2FF72B2EB515F08BF40F002000128F5
:10C9300008BF052002B0704730B52DED048B81B0E3
:10C94000B0EE408AF0EE608A6A4651EC180B03F0B4
:10C950008FFE00989FED329B7E300090002821DCF6
:10C9600053EC192B51EC180B07F0EAFF1AD00021F9
:10C9700040F608004FF00000044651EC180B07F099
:10C9800099FD08EE100A40F6080004EA00014FF095
:10C990000000B5EEC08AF1EE10FA04BF0220F4F7F1
:10C9A00028F92DE00098FF2830DB002108464FF0E1
:10C9B000000000F4400553EC192B51EC180B08F063
:10C9C0008FF98CBF002401240220F4F712F99FEDA7
:10C9D000168A4DB1002C0CBF4FF400004FF48000BC
:10C9E000A84218BF9FED118A042108464FF00000AD
:10C9F000002C01BFB1EE480A01B0BDEC048B30BD84
:10CA0000B0EE480A01B0BDEC048B30BD51EC180B00
:10CA100007F050FD01B000EE100ABDEC048B30BDF4
:10CA200000000000000000000000807FFFFF7F7F0B
:10CA300070B59B482DED020B2DED068B079D25F063
:10CA40000044A04218DC9748844202DC0AD10698D0
:10CA500040B19DED060BBDEC068B02B0BDE8704009
:10CA600001F0D6BF002DCCBF9FED8F0B9FED900B3B
:10CA7000BDEC068B02B070BD8F48A04215DD8F481B
:10CA8000A042D8BF4FF0FF3458DD9DED060B51ECAE
:10CA9000100BFFF739FF042808BF01F0EDFF9DEDF3
:10CAA000060BBDEC068B02B070BD9DED060B51EC84
:10CAB000100B03F0D1FDCDE9060181489FED828B7B
:10CAC000A0423CDD8248A0421FDD00249FED82ABE6
:10CAD0009DED060B53EC1A2B51EC100B07F01CFDCF
:10CAE0009DED060B41EC190B53EC1A2B51EC100B7E
:10CAF00007F0F8FF53EC182B08F000FA53EC192B51
:10CB000007F0C6FDCDE9060149E09DED060B0124C5
:10CB100053EC182B51EC100B07F0FEFC9DED060BAF
:10CB200041EC190B53EC182B51EC100B08F0E6F903
:10CB300053EC192B07F0ACFDCDE906012FE0684856
:10CB4000A0421FDD02249FED689B9DED060B53EC78
:10CB5000192B51EC100B07F0C5FF53EC182B07F005
:10CB6000DBFC9DED060B41EC180B53EC192B51EC43
:10CB7000100B08F0C3F953EC182B07F089FDCDE931
:10CB800006010CE09DED060B032453EC102B9FEDEA
:10CB9000580B51EC100B07F07BFDCDE906019DED24
:10CBA000060B53EC102B51EC100B07F09BFF41ECE4
:10CBB000180B53EC182B07F095FF41EC190B4E485E
:10CBC0000621B0EE490AF0EE690A784401F04CFC07
:10CBD00053EC182B51EC100B07F084FF41EC180BB1
:10CBE0004648B0EE490AF0EE690A0521784401F0A2
:10CBF0003BFC53EC192B51EC100B07F073FF41EC8D
:10CC0000100B51EC180B53EC102B002C0EDA07F024
:10CC100083FC9DED061B53EC112B07F063FF9DED8C
:10CC2000061B53EC112B08F091F835E007F074FC6B
:10CC30009DED061B53EC112B07F054FF41EC100B3C
:10CC40002F48784400EBC40090ED001B51EC100B12
:10CC500053EC112B08F052F99DED061B53EC112BF0
:10CC600008F04CF941EC100B2648784400EBC40066
:10CC700090ED001B51EC100B53EC112B08F066F8F3
:10CC800041EC100B002DA2BFBDEC068B02B070BDB5
:10CC900051EC100B07F002FC41EC100B01E7000017
:10CCA000000010440000F07F182D4454FB21F93F90
:10CCB000182D4454FB21F9BF0000DC3F0000203E4A
:10CCC0000000F33F00000000000000000000F03F03
:10CCD0000000E63F000000000000000000000040EF
:10CCE0000080034000000000000000000000F83F4A
:10CCF000000000000000F0BF4A880000008800002B
:10CD00008A8700004287000070B56B4E2DED040B42
:10CD10002DED028B82B0DDF81CC0DDE905235C42FD
:10CD20002CF000411C4341EAD474049D22F00040E1
:10CD3000B44205D86C422C4340EAD474B4420BD9B7
:10CD40009DED061B9DED040B02B0BDEC028B04B003
:10CD5000BDE8704001F066BEACF14054A4F17F64C0
:10CD60001C430BD0022404EAAC7444EAD274054399
:10CD70009FED538B9FED542B07D015E09DED040BD9
:10CD800051EC100B01F096FF42E0002C11BF012C7A
:10CD90009DED040B02B0BDEC028B04BF04B070BD6E
:10CDA000022C38D0032C3BD00B439FED491B9FED49
:10CDB0004A0B0AD0B14218D1B04209D121F08041CA
:10CDC00020F08040079105900FE0002A15DA10E06E
:10CDD000434B7B44002C08BF93ED000B0DD0012C7E
:10CDE00010D0022C17D0032C1AD0B0421DD1002A2B
:10CDF00003DAB0EE410AF0EE610A02B0BDEC028B3C
:10CE000004B070BD93ED000B51EC100B07F046FB26
:10CE100041EC100BF1E7B0EE480AF0EE680AECE7DF
:10CE2000B0EE420AF0EE620AE7E7401A00153C282D
:10CE3000C8BF8DED000B19DCBCF1000FBEBF10F1B7
:10CE40003C0F9FED290B8DED000B0FDB9DED060BCD
:10CE500053EC102B9DED040B51EC100B07F018FC5C
:10CE600003F0FAFB01F026FFCDE90001002C08BF1A
:10CE70009DED000BC1D0012C10D0022C9FED1C0B9E
:10CE800053EC102B9DED000B51EC100B0DD008F066
:10CE900035F853EC182B08F031F8B9E7019880F019
:10CEA000004001909DED000BA7E708F027F853EC38
:10CEB000182B07F04BFFABE70000F07F00000000ED
:10CEC000182D4454FB210940182D4454FB2109C05E
:10CED000182D4454FB21F9BF182D4454FB21F93F70
:10CEE0003287000000000000000000000000000089
:10CEF000075C143326A6A13C10B52F499FED2C1BCF
:10CF00002DED020B84B0059820F000408842D8BF78
:10CF10009DED040B2DDD2949884209D1049840B9C3
:10CF20004FF00100F3F765FE01F086FD06B010BD7D
:10CF300005DB9DED040B01F06BFD06B010BD6846EE
:10CF40009DED040B00F0BCFF10F0030004BF9DED4D
:10CF5000021B9DED000B0CD001280ED09DED021B95
:10CF60009DED000B022817D0012001F0F9FA06B060
:10CF700010BD01F0C1F906B010BD9DED021B9DED85
:10CF8000000B012001F0ECFA51EC100B07F086FACF
:10CF900006B041EC100B10BD01F0AEF951EC100BD6
:10CFA00007F07CFA06B041EC100B10BD0000000049
:10CFB0000000000000000000FB21E93F0000F07FBE
:10CFC0002DED020B019820F0004001909DED000B2B
:10CFD00002B070470000000030B540F2FF742DED44
:10CFE000048BF0EE608A18EE901A85B0B0EE408A9D
:10CFF0009FED2B9B05468DED008B34EA115147D0F8
:10D0000053EC192B51EC180B07F09AFC40D02A4630
:10D0100051EC180B08F010F941EC180B18EE900ABF
:10D020008DED008B34EA10501CD053EC192B51ECD1
:10D03000180B07F085FC2BD10220F3F7DAFD01F085
:10D040001BFD10EE901A18EE900A8DED020B8DED7F
:10D05000008B61F31E0003909DED020B05B0BDEC4B
:10D06000048B30BD0220F3F7C4FD01F0F5FC10EE97
:10D07000901A18EE900A8DED020B8DED008B61F386
:10D080001E0003909DED020B05B0BDEC048B30BD7E
:10D0900005B0B0EE480AF0EE680ABDEC048B30BD76
:10D0A00000000000000000002DE9F04D2DED040B04
:10D0B0002DED0E8B96B0DDE92550279CDDF890A074
:10D0C00025F0004624F00048BAF1000F14BF0121FA
:10D0D000002101EB4502FC4953184A1093422AD320
:10D0E000002814BF0123002303EB44030B44F7493A
:10D0F0008B4220D358EA00019FEDF59B76D0DFF8F4
:10D10000D8B35D4503D1BAF1000F05D188E0BAF17B
:10D11000000F08BF002100D0012101EB450111F5EE
:10D12000001F08D8002814BF0121002101EB440191
:10D1300011F5001F0BD99DED261B9DED240B16B09C
:10D14000BDEC0E8B04B0BDE8F04D01F06BBC0027C8
:10D15000002DBCBFE149884521DAE1498845A8BFD7
:10D1600002271CDAC3451ADCDE4901EB28511429D9
:10D1700008DDC1F1340220FA02F101FA02F2824222
:10D180000DD108E058B9C1F1140228FA02F101FAF0
:10D1900002F2424503D101F00101C1F1020756EA52
:10D1A0000A0124D1002C22DA002D18BF022F01D051
:10D1B000012F0AD00220F3F71CFD16B0BDEC0E8B38
:10D1C00004B0BDE8F04D01F00BBC0220F3F711FDF7
:10D1D00001F006FC51EC100B07F060F941EC100B6C
:10D1E00016B0BDEC0E8B04B0BDE8F08D18E09FEDDD
:10D1F000BEAB9FEDBF8B002871D1B848804522D1CE
:10D2000005F1804010F5801008BFBAF1000F07D07B
:10D21000B3450ADC002CA8BF9DED260BE0DA0DE03B
:10D22000B0EE490AF0EE690ADAE7002C06DA9DED65
:10D23000260B51EC100B07F031F96FE0AE48784443
:10D2400090ED000BCCE7D8454DD1002C48DA2EB13B
:10D2500086423AD1BAF1000F42D126E0BAF1000F6E
:10D2600013D00220F3F7C5FC01F0F6FB8DED020BA5
:10D270009DED240B8DED000B10EE900A039961F3E8
:10D280001E0003909DED020BAAE78DED02AB9DED14
:10D29000240B1AEE901A10EE900A8DED000B61F33C
:10D2A0001E0003909DED020B9AE78DED028B9DED24
:10D2B000240B18EE901A10EE900A8DED000B61F31E
:10D2C0001E0003909DED020B8AE709DA9DED240B09
:10D2D00051EC190B53EC102B07F0DAF91EE020E0AB
:10D2E0009DED240B7CE786421BDAB4F1804F0DD014
:10D2F000A4F10050B0F1FF5013D1002D11DB9DEDD2
:10D30000240B51EC100B06F013FD07E09DED240BF0
:10D3100053EC102B51EC100B00F0C2BC41EC100B85
:10D320005EE79DED240B51EC100B03F095F9BAF17B
:10D33000000FCDE90E0142D19FED710B46B3A6F16E
:10D34000E040B0F17F600CD05E4538D1002D00DAAE
:10D35000A7B3022F0CBF01204FF0FF3007F05BFB9B
:10D36000DCE7002D01DD002C0DDA002D01DD002CA5
:10D370001FDB002D16DA002C14DB012F08BF9FEDF8
:10D38000620B3FF42DAFB0EE4A0AF0EE6A0A27E7CF
:10D39000022F18BF002D0CD0012F0AD1002DFFF64F
:10D3A0001FAF06E0002DB8BF002C08DA012F3FF4B4
:10D3B00017AFB0EE480AF0EE680A11E71BE0012053
:10D3C00000EBE57050EA070115D0791EB0EE498AEE
:10D3D000F0EE698A084308BF9FED4D8B4E4800254B
:10D3E000804570DD4D494E48884514DDB0420DDB67
:10D3F000002C19DB2FE00120F3F7FBFB16B0BDEC8E
:10D400000E8B04B0BDE8F04D01F016BBB34502DC55
:10D41000002C09DC1FE0864202DA002C1BDA03E054
:10D420005E452BDD002C16DD0220F3F7E2FB01F058
:10D4300013FB8DED020B53EC1A2B51EC180B07F07C
:10D4400051FBCDE900010399019861F31E0003909F
:10D450009DED020BC4E60220F3F7CBFB01F00CFBC1
:10D4600010EE901A18EE900A8DED020B8DED008BE8
:10D4700061F31E0003909DED020BB1E69DED0E0BD6
:10D4800053EC192B51EC100B07F038FD9FED260BD8
:10D49000CDE9080153EC102B9DED080B51EC100B5E
:10D4A00007F020FB9FED221B53EC112B07F04EFCE5
:10D4B0009DED081B53EC112B07F014FB9FED1E1B79
:10D4C00053EC112B3CE08CE0FFFF1F00FFFF0F002F
:10D4D000000000000000F03F0000F03F0000F07F7F
:10D4E0000000404301FCFFFF000000000000F07F4F
:10D4F0000000000000000000C682000000000000E4
:10D500000000000000000080000000000000F0FFAC
:10D51000000000000000F0BF0000E0410000F04308
:10D52000FFFFEF3F00000000000000000000D03FC0
:10D53000555555555555D53F000000000000E03FBA
:10D5400007F004FC9DED080B41EC1A0B53EC102B7B
:10D5500051EC100B07F0C6FA53EC1A2B07F0C2FA85
:10D5600041EC1A0B9FEDFE0B53EC102B9DED080BBD
:10D5700051EC100B07F0B6FA41EC1B0B9FEDFA0BC8
:10D5800051EC1A0B53EC102B07F0ACFA41EC1A0BD0
:10D590009FEDF70B53EC102B9DED080B51EC100B8E
:10D5A00007F0A0FA53EC1A2B07F0A8FC41EC1A0B79
:10D5B00051EC1B0B53EC1A2B06F0AEFF0690CDE995
:10D5C00006519DED060B53EC1B2B51EC100B07F095
:10D5D00095FC53EC1A2B07F0B9FB41EC100B00F053
:10D5E000A1B90020B6F5801F0EDA9FEDE30B53ECD6
:10D5F000102B9DED0E0B51EC100B07F073FACDE9DB
:10D600000E016FF034000E4600EB2650A0F2FF37FB
:10D61000C6F31300DA4940F07F6646F04056884270
:10D62000D8BF002408DDD7498142C8BF012403DCEC
:10D630000024A6F580167F1CD348784400EBC40074
:10D640000F9690ED00CB9DED0E0B53EC1C2B51EC87
:10D65000100B07F053FC9DED0E0B41EC1B0B53EC34
:10D660001C2B51EC100B06F057FF41EC100B51EC4A
:10D67000190B53EC102B07F00BF841EC1D0B51EC80
:10D680001B0B53EC1D2B07F02DFA41EC1A0BBF4876
:10D690008DED10AB7844109590ED000B4FF00050DD
:10D6A00040EA660000EB84408DED080B00F5002099
:10D6B00009909DED080B53EC1C2B51EC100B07F05F
:10D6C0001DFC9DED0E1B53EC112B07F03FFB41ECB5
:10D6D000100B53EC102B9DED100B51EC100B07F0C1
:10D6E00001FA9DED080B41EC1C0B53EC102B9DED4A
:10D6F000100B51EC100B07F0F5F953EC1B2B07F056
:10D7000025FB53EC1C2B07F0F9FB53EC1D2B07F00A
:10D71000E9F941EC1C0B53EC1A2B51EC1A0B07F0F6
:10D72000E1F941EC1B0B9A480621B0EE4B0AF0EEF2
:10D730006B0A784400F098FEB0EE401AF0EE601AE2
:10D74000B0EE41DAF0EE61DA53EC1B2B51EC1B0B1F
:10D7500007F0C8F953EC1D2B07F0C4F99DED100B31
:10D7600041EC1B0B53EC1A2B51EC100B06F0D4FEC2
:10D7700053EC1C2B07F0B6F953EC1B2B06F0CCFE38
:10D780009DED100B41EC1B0B53EC102B51EC100BCF
:10D7900007F0A8F941EC1D0B9FED7FEB53EC1E2B1E
:10D7A00006F0BAFE53EC1B2B06F0B6FE0890CDE94E
:10D7B00008519DED080B53EC1E2B51EC100B07F09C
:10D7C0009DFB53EC1D2B07F099FB53EC1B2B07F033
:10D7D000BDFA9DED080B41EC1D0B53EC102B9DED9C
:10D7E000100B51EC100B07F07DF941EC1B0B53ECC7
:10D7F0001A2B51EC1D0B07F075F99DED080B41EC50
:10D800001A0B53EC102B51EC1C0B07F06BF953EC7B
:10D810001A2B06F081FE41EC1A0B51EC1B0B53EC5A
:10D820001A2B06F079FE0C90CDE90C519DED0C0BF6
:10D8300053EC1B2B51EC100B07F060FB53EC1A2B35
:10D8400007F084FA41EC1B0B9FED550B53EC102BAA
:10D850009DED0C0B51EC100B07F044F941EC1A0B49
:10D860009FED510B51EC1B0B53EC102B07F03AF9C9
:10D8700041EC1B0B9FED4E0B53EC102B9DED0C0B55
:10D8800051EC100B07F02EF953EC1B2B06F044FE65
:10D8900041EC100B4848784400EBC40090ED001BAD
:10D8A00051EC100B53EC112B06F036FE41EC1B0B28
:10D8B000384607F0B0F8CDE9080153EC1B2B51ECCA
:10D8C0001A0B06F029FE41EC100B3C48784400EBA3
:10D8D000C40090ED00CB51EC100B53EC1C2B06F068
:10D8E0001BFE9DED081B53EC112B06F015FE069058
:10D8F000CDE906519DED080B53EC102B9DED060B69
:10D9000051EC100B07F0FAFA53EC1C2B07F0F6FA67
:10D9100053EC1A2B07F0F2FA53EC1B2B07F016FA14
:10D9200041EC100B9DED261B53EC102B8DED001BD5
:10D9300000959DED260B51EC100B07F0D3F89DEDF3
:10D94000000B41EC1A0B53EC102B9DED260B51EC08
:10D95000100B07F0D3FA9DED061B53EC112B2FE0B3
:10D96000000000604715F73FFE822B654715F73F23
:10D9700044DF5DF80BAE543E000000000000404361
:10D980008E9803007AB60B000A7E0000707E0000BD
:10D99000427D000000000000000000000000084080
:10D9A000000000E009C7EE3FFD033ADC09C7EE3F87
:10D9B000F5015B14E02F3EBECE7B0000887B0000AB
:10D9C00007F090F853EC1A2B06F0A6FD9DED060B20
:10D9D00041EC1A0B53EC102B9DED000B51EC100B8E
:10D9E00007F080F8CDE90C019DED0C0B51EC1A0B02
:10D9F00053EC102B06F090FDCDE902010C46AA492C
:10DA00008C422FDB611A084318D19DED0C0B53ECAF
:10DA1000102B9DED020B51EC100B07F06FFA41EC4F
:10DA20001B0B9FEDA30B51EC1A0B53EC102B06F0C4
:10DA300073FD53EC1B2B07F053F92DD20220F3F7A3
:10DA4000D8F801F009F810EE901A18EE900A8DED52
:10DA5000020B8DED008B61F31E0003909DED020B18
:10DA6000FFF7BEBB944A24F00041914214D393497E
:10DA7000214408437FF4EFAC9DED0C0B53EC102BCD
:10DA80009DED020B51EC100B07F038FA53EC1A2BFA
:10DA900007F026F97FF6DFAC24F000408849894A78
:10DAA000002601EB205182422BDA481C4FF48011F2
:10DAB00021FA00F02044844AC0F30A517A44A1F2CA
:10DAC000FF3192ED000B814A8DED080BCA4020EA30
:10DAD0000202C0F3130040F48010C1F1140120FAD7
:10DAE00001F60992002CB8BF76429DED080B53EC6D
:10DAF000102B9DED0C0B51EC100B07F0FFF9CDE94D
:10DB00000C019DED0C0B51EC1A0B53EC102B06F095
:10DB100003FD9FED6F0B0890CDE9085153EC102BDE
:10DB20009DED080B51EC100B06F0DCFF41EC1B0BDC
:10DB30009FED690B53EC102B9DED080B51EC100B76
:10DB400006F0D0FF9DED0C0B41EC1C0B53EC102BA1
:10DB50009DED080B51EC100B07F0D0F953EC1A2B8C
:10DB600007F0F4F89FED5E1B53EC112B06F0BAFFA3
:10DB700053EC1C2B06F0D0FC41EC1A0B51EC1B0BA8
:10DB800053EC1A2B06F0C8FCCDE902019DED020B07
:10DB900053EC1B2B51EC100B07F0B0F953EC1A2B84
:10DBA00007F0D4F89DED020B41EC1A0B53EC102B4F
:10DBB00051EC100B06F096FFCDE908014A489DEDA7
:10DBC000080B0521784400F04FFC9DED081B51EC3B
:10DBD000100B53EC112B06F085FF9DED021B53EC4F
:10DBE000112B07F0B3F8CDE906019DED020B53ECC4
:10DBF0001A2B51EC100B06F075FF53EC1A2B06F0A4
:10DC00008BFC9FED3B0B41EC1A0B53EC102B9DED65
:10DC1000060B51EC100B07F071F99DED060B41EC72
:10DC20001B0B53EC102B9DED020B51EC100B06F06F
:10DC300059FF53EC1B2B06F02BFD53EC1A2B07F06E
:10DC40005DF99DED021B53EC112B07F057F953ECD6
:10DC5000192B07F07BF8CDE9020101EB0650011505
:10DC60000029C8BF039015DC9DED020B324651EC34
:10DC7000100B07F0E1FAFEF747FE042808BF00F09A
:10DC8000FBFE32469DED020B51EC100B07F0D4FA6F
:10DC9000CDE902019DED020B51EC180B53EC102B5A
:10DCA00006F020FFFFF73ABB0000904000000000A4
:10DCB000FE822B654715973C00CC904000346F3FA7
:10DCC00001FCFFFF0000E03F487A0000FFFF0F006B
:10DCD00000000000432EE63F396CA80C615C20BEBA
:10DCE000EF39FAFE422EE63FE07800000000000027
:10DCF000000000000000004010B52F499FED2C1BD4
:10DD00002DED020B84B0059820F000408842DCBF66
:10DD100000209DED040B32DD2849884209D104988A
:10DD200040B94FF00100F2F764FF00F085FE06B045
:10DD300010BD05DB9DED040B00F06AFE06B010BDC2
:10DD400068469DED040B00F0BBF810F0030011D005
:10DD5000012818D09DED021B9DED000B02281AD062
:10DD600000F0CAFA51EC100B06F098FB06B041EC3B
:10DD7000100B10BD9DED021B9DED000B012000F06E
:10DD8000EFFB06B010BD9DED021B9DED000B00F0FA
:10DD9000B3FA06B010BD012000F0E2FB51EC100B0D
:10DDA00006F07CFB06B041EC100B10BD000000003B
:10DDB0000000000000000000FB21E93F0000F07FB0
:10DDC00000B52DED048BB0EE409AF0EE609A83B072
:10DDD00051EC190B06F0C6FF41EC180B18EE100AB7
:10DDE00018EE901A8DED008B002818BF0120084313
:10DDF00020F00040C0F17F6000F1E040C00F14D07F
:10DE000019EE101A19EE900A8DED009B002918BF2B
:10DE10000121084320F00040C0F17F6000F1E040A4
:10DE2000C00F04BF0120F2F7E4FEB0EE480A03B0D1
:10DE3000F0EE680ABDEC048B00BD0000000000009D
:10DE400010B51D499FED1A1B2DED020B84B00598EE
:10DE500020F000408842DCBF01209DED040B21DD55
:10DE60001649884209D1049840B94FF00100F2F7F1
:10DE7000C0FE00F0E1FD06B010BD05DB9DED040B1A
:10DE800000F0C6FD06B010BD68469DED040B00F025
:10DE900017F800F001000121A1EB40009DED021BED
:10DEA0009DED000B00F0F4FB06B010BD000000007B
:10DEB0000000000000000000FB21E93F0000F07FAF
:10DEC0002DE9F14F04462DED020B2DED088B8AB0A4
:10DED0009FEDE70B80ED020B139EE74826F000450F
:10DEE00085420ADC9DED120B002084ED000B0AB088
:10DEF000BDEC088B03B0BDE8F08FE0489FEDE0ABD0
:10DF00009FEDE1BBA84247DDE14F9FEDE39B9FED15
:10DF1000E48B9DED120B53EC1A2B51EC100B002EE1
:10DF20001CDD06F0EBFF41EC100BBD4208D053ECBA
:10DF30001B2B51EC100B06F0E1FFC4E900010BE0D4
:10DF400053EC192B51EC100B06F0D8FF53EC182BA7
:10DF500006F0D4FFC4E900010120C8E706F0DCFAAE
:10DF600041EC100BBD4208D053EC1B2B51EC100BB5
:10DF700006F0D2FAC4E900010BE053EC192B51EC86
:10DF8000100B06F0C9FA53EC182B06F0C5FAC4E9D9
:10DF900000014FF0FF30AAE7C348A84279DB9DEDAE
:10DFA000120B51EC100B02F057FB41EC180B9FEDDC
:10DFB000C00B53EC102B06F095FD9FEDBF1B53ECEF
:10DFC000112B06F0A9FA06F0F7FC074606F023FD30
:10DFD00041EC190B53EC1A2B06F084FD53EC182B73
:10DFE00006F0B4FE41EC180B53EC1B2B51EC190B53
:10DFF00006F078FDDFF8C8A241EC100B4FEA155887
:10E000000125FA4453EC102B51EC180B06F076FF67
:10E01000032DC4E900013DD0C1F30A5005EB4511C1
:10E02000A8EB00001139814234DA0AEB051BB0EE8F
:10E0300048AA9BED000BF0EE68AA53EC102B51ECB4
:10E04000190B06F04FFD41EC1B0B51EC1A0B53EC76
:10E050001B2B06F053FF41EC180B51EC1A0B53EC41
:10E06000182B06F04BFF53EC1B2B06F047FF9BEDE4
:10E07000020B41EC1A0B53EC102B51EC190B06F070
:10E0800031FD53EC1A2B06F039FF41EC100B6D1CDF
:10E09000B8E70EE0002EA8BF3846BFF628AF94EDD3
:10E0A000000B51EC100B06F0F9F9C4E900017842BD
:10E0B0001DE7C6F3130040F4801EC6F30A50A0F219
:10E0C000F530471100F01F05C5F12000DDF848B01C
:10E0D00008900020069007900520EC467949002D15
:10E0E00007EB0002794408BF51F8221009D051F81B
:10E0F000223001EB8201AB404A68089922FA01F113
:10E100001943A1FB0E26A1FB0B131A449A4234BFFC
:10E110000123002303EB06080CEB8003D3E901A6DF
:10E120000E448E4234BF0121002192448A4411B131
:10E13000924502D903E0924501D2012100E000217D
:10E14000C3E901A641444CF82010011EA0F10100D2
:10E15000C4DC029800F10050850F0298DDE90367E6
:10E160008000DDF8148006F056FC41EC1A0B3046B6
:10E1700006F068FC9FED541B53EC112B06F0B2FC2B
:10E1800041EC1B0B384606F05DFC9FED511B53EC38
:10E19000112B06F0A7FC41EC180B404606F052FC90
:10E1A0009FED4D1B53EC112B06F09CFC41EC190B21
:10E1B00051EC180B53EC192B06F0AEF953EC1B2B5A
:10E1C00006F0AAF953EC1A2B06F0A6F9CDE90801DE
:10E1D000002008909DED080B53EC1A2B51EC100B0E
:10E1E00006F08CFE53EC1B2B06F088FE53EC182B2C
:10E1F00006F084FE53EC192B06F0A8FD9FED381BAA
:10E2000053EC112B06F06EFC9FED370B41EC180B15
:10E2100053EC102B9DED080B51EC100B06F062FC3B
:10E2200053EC182B06F078F99FED310B41EC180BED
:10E2300053EC102B9DED080B51EC100B06F052FC2B
:10E2400053EC182B06F068F941EC100B139810F002
:10E25000004F06D06D4251EC100B06F01FF941EC57
:10E26000100B284684ED000B41E600000000000082
:10E270000000000000000000FB21E93F7CD90240C3
:10E2800000004054FB21F93F3163621A61B4D03D74
:10E29000FB21F93F000000000000601A61B4D03D8E
:10E2A0007370032E8A19A33BFB2139410000000043
:10E2B00083C8C96D305FE43F000000000000E03F0C
:10E2C0000A75000058740000000000000000103EB5
:10E2D000000000000000103C000000000000103AA8
:10E2E000182D4454FB21F93D3326A611460B113C51
:10E2F00000000054FB21F93D10B52DED040B2DED70
:10E30000088B82B0B0EE419AF0EE619A0B9820F043
:10E3100000449FED4BABB4F1795F11DA9DED0A0B30
:10E3200051EC100B06F048FB002801BFB0EE4A0A82
:10E33000F0EE6A0A02B0BDEC088B04BF04B010BD59
:10E340009DED0A0B53EC102B51EC100B06F0CAFBA1
:10E3500041EC180B3C480621B0EE480AF0EE680A82
:10E36000784400F081F853EC182B51EC100B06F0B8
:10E37000B9FB9DED0A0B41EC1B0B53EC192B51EC37
:10E38000100B06F0AFFB41EC190B53EC1B2B51ECBF
:10E39000180B06F0A7FB53EC192B06F0AFFD9FED11
:10E3A0002C0B41EC190B53EC102B51EC180B06F015
:10E3B00099FB41EC100B2848844210DA53EC192BDE
:10E3C00051EC100B06F09AFD53EC1A2B06F0BEFC34
:10E3D00041EC100B02B0BDEC088B04B010BD1F481F
:10E3E000A042BCBF9FED1E1B8DED001B06DBA4F5FC
:10E3F00000100190002000909DED001B51EC100BCF
:10E4000053EC112B06F07AFD9DED000B41EC180B3F
:10E4100053EC102B51EC1A0B06F070FD41EC1A0B6B
:10E4200053EC192B51EC180B06F068FD53EC1A2B2A
:10E4300006F08CFC41EC100BCCE700000000000063
:10E44000000000000000F03F7471000000000000B8
:10E45000000000000000E03F3333D33F0000E93FFD
:10E46000000000000000D23F70B504462DED028B85
:10E470004D1E00EBC500B0EE408AF0EE608A90EDD4
:10E48000000B35F0060017D053EC182B51EC100B95
:10E4900006F028FB41EC100B6D1E04EBC50090ED5F
:10E4A000001B51EC100B53EC112B06F035F841EC2E
:10E4B000100B35F00600E7D1022D36D0042D1CD00C
:10E4C000062D1CBFBDEC028B70BD53EC182B51EC1C
:10E4D000100B06F007FB94ED0A1B53EC112B06F012
:10E4E0001BF853EC182B06F0FDFA94ED081B53ECC7
:10E4F000112B06F011F841EC100B53EC182B51ECDA
:10E50000100B06F0EFFA94ED061B53EC112B06F0FE
:10E5100003F853EC182B06F0E5FA94ED040B53ECDA
:10E52000102B05F0F9FF41EC100B53EC182B51ECBC
:10E53000100B06F0D7FA94ED021B53EC112B05F0EB
:10E54000EBFF53EC182B06F0CDFA94ED001B53ECC7
:10E55000112B05F0E1FFBDEC028B41EC100B70BDFF
:10E5600031B504462DED040B2DED0A8BB0EE41BA0A
:10E57000F0EE61BA0B989DED0A0B20F00040B0F16F
:10E58000795F0DDA51EC100BFEF7BEF9042808BFD5
:10E5900000F072FA9DED0A0BBDEC0A8B05B030BDA0
:10E5A00053EC102B51EC100B06F09CFA41EC180BBD
:10E5B0009DED0A0B53EC182B51EC100B06F092FA60
:10E5C00041EC190B2C48B0EE480AF0EE680A052120
:10E5D0007844FFF749FF9FED2ACBB0EE40AAF0EE5A
:10E5E00060AA9CB353EC1C2B51EC190B06F07AFA81
:10E5F00041EC1C0B53EC1A2B51EC190B06F072FA80
:10E600009FED210B41EC190B53EC102B51EC1B0B24
:10E6100006F068FA53EC192B06F070FC53EC182B3B
:10E6200006F060FA53EC1B2B06F068FC53EC1C2B35
:10E6300006F064FC9DED0A1B53EC112B06F086FBE3
:10E64000BDEC0A8B05B041EC100B30BDFFE753EC7D
:10E650001A2B51EC180B06F045FA53EC1C2B05F065
:10E660005BFF53EC192B06F03DFA9DED0A1B53ECB2
:10E67000112B05F051FFE3E70470000000000000DB
:10E68000495555555555C5BF000000000000E03FF5
:10E69000F1B506462DED040BBD482DED0C8B8AB06F
:10E6A000B0EE418AF0EE618A179D25F000449FED9F
:10E6B000BABB9FEDBBCB844208DA9DED160B51EC43
:10E6C000100B06F079F9002800F0E980B64FA74258
:10E6D00031DC002D0DDA9DED160B51EC100B05F021
:10E6E000DDFECDE9160151EC180B05F0D7FE41EC2B
:10E6F000180B9FEDAF0B53EC102B9DED160B51EC4F
:10E70000100B06F023FB53EC182B9FEDAB0BCDE960
:10E71000040151EC100B06F0F1FB41EC100B53EC33
:10E72000102B9DED040B51EC100B05F0F5FE9FED49
:10E73000A48BCDE916019DED160B53EC102B51EC7B
:10E74000100B06F0CFF9CDE904019DED040B53EC5D
:10E75000102B51EC100B06F0C5F941EC190B9A483F
:10E760000621B0EE490AF0EE690A7844FFF77CFE14
:10E770009648B0EE40DAF0EE60DAB0EE490AF0EE1C
:10E78000690A06217844FFF76FFE9DED041B51ECEA
:10E79000100B53EC112B06F0A5F99DED040B41EC89
:10E7A0001A0B53EC102B9DED160B51EC100B06F0D1
:10E7B00099F941EC190B53EC1A2B51EC1D0B05F098
:10E7C000ABFE53EC192B06F08DF953EC182B05F02A
:10E7D000A3FE9DED041B53EC112B06F083F953ECC3
:10E7E000182B05F099FE41EC180B9FED790B51ECBD
:10E7F000190B53EC102B06F075F953EC182B05F0A0
:10E800008BFE41EC190B9DED160B53EC192B51ECC3
:10E81000100B05F081FE41EC180BA74269DC304675
:10E8200006F0F9F841EC1A0B51EC180B53EC1A2BCB
:10E8300005F072FE41EC1B0B53EC182B51EC180B3E
:10E8400006F050F953EC1B2B05F022FF53EC192B6B
:10E8500006F054FB9DED161B53EC112B06F076FAD7
:10E860009FED5D1B53EC112B06F03CF953EC1A2B7A
:10E8700006F06CFA41EC180B022000EAA570C0F11A
:10E88000010006F0C8F853EC182B06F02BF900BF76
:10E8900041EC100B0AB0BDEC0C8B05B0F0BD711C47
:10E8A0001698214308430CD09DED160B012E1CBF7A
:10E8B00053EC102B51EC1C0B10D000BF05F0E8FE00
:10E8C000E6E79DED160B51EC100B01F0C5FE41EC97
:10E8D000100B51EC1B0B53EC102BEFE751EC100B12
:10E8E000FEF712F8042808BF00F0C6F89DED160BDD
:10E8F000D0E7012E04BFB0EE480AF0EE680AC9D096
:10E900008DED048B002404949DED040B53EC102B2F
:10E910009DED160B51EC100B06F018FA53EC192B69
:10E9200006F014FA41EC190B53EC182B51EC1C0BAC
:10E9300005F0AEFE41EC180B8DED008B00949DEDC3
:10E94000040B53EC102B9DED000B51EC100B06F05B
:10E95000C9F853EC1B2B05F0DFFD9DED000B41ECDE
:10E960001A0B53EC192B51EC100B06F0BBF853ECBF
:10E970001A2B05F0D1FD53EC182B06F0B3F89DEDE2
:10E98000001B53EC112B05F0C7FD81E700000000D0
:10E990000000303E00000000000000000000F03FDA
:10E9A000000000000000F0BF2894E53F00000000D8
:10E9B000182D4454FB21E93F075C143326A6813C03
:10E9C0000000000000000000926E0000A86E000031
:10E9D000635555555555D53F0000000000000040D7
:10E9E0009FED070B10B553EC102B9FED070B51EC6F
:10E9F000100B05F04DFE41EC100B10BD00000000A7
:10EA00000000000000000000000000000000F03FD7
:10EA100010B553EC102B51EC100B05F07DFD41ECC3
:10EA2000100B10BD10B553EC112B51EC100B05F071
:10EA300073FD41EC100B10BD9FED050B10B553ECB1
:10EA4000102B51EC100B05F023FE41EC100B10BD08
:10EA500000000000000000009FED050B10B553EC16
:10EA6000102B51EC100B06F03DF841EC100B10BDD3
:10EA700000000000000000709FED050B10B553EC86
:10EA8000102B51EC100B06F02DF841EC100B10BDC3
:10EA9000000000000000001010B5044691ED000BCE
:10EAA000FDF74AFF84ED000A10BD10B5044690ED55
:10EAB000000B0846FEF790FA84ED000B10BD3038CD
:10EAC0000A2801D2012070470020704700BF70471C
:10EAD00010B5044641F69A702040002868D004F42E
:10EAE000805040B14FF47A710320F8F76DF804209C
:10EAF0006E49487257E004F4807038B10021032059
:10EB0000F8F762F80320694948724CE004F4806029
:10EB100040B14FF47A710320F8F756F8102063499A
:10EB2000487240E004F4007060B14FF47A71012043
:10EB3000F8F74AF80B205D494872B2EE040AFCF778
:10EB4000FDFA30E004F0080040B14FF47A7104207F
:10EB5000F8F73AF804205549487224E004F08000A0
:10EB600028B14FF47A710420F8F72EF81BE004F472
:10EB7000006040B14FF47A710320F8F725F80720C0
:10EB80004A4948720FE004F0020038B10021062023
:10EB9000F8F71AF80A204549487204E04FF4FA7170
:10EBA0000320F8F711F83220FCF7A8FA002010BD76
:10EBB00046F2E7002040002866D004F4804040B1CF
:10EBC0004FF47A710720F7F7FFFF062037494872A4
:10EBD00055E004F0800028B14FF47A710620F7F771
:10EBE000F3FF4CE004F0200028B14FF47A710620C6
:10EBF000F7F7EAFF43E004F0400080B10021022073
:10EC0000F7F7E2FF0020294948720121274880F8E0
:10EC1000DD10B2EE040AFCF791FA0120C7E704F018
:10EC2000040080B12248407F20B164210220F7F720
:10EC3000CBFF04E04FF47A710220F7F7C5FF022002
:10EC40001A4948721BE004F0010038B10021052088
:10EC5000F7F7BAFF05201549487210E004F4005098
:10EC600040B14FF47A710420F7F7AEFF00200F494E
:10EC7000487204E04FF4FA710320F7F7A5FF05206E
:10EC8000FCF73CFA002092E70948407F20B164215C
:10EC90000120F7F799FF04E04FF47A710120F7F7AC
:10ECA00093FF082001494872012080E7641F022079
:10ECB0002816012010B541EC100BFDF7B9FE51EC00
:10ECC000100B10BD10B504464FF47A7104FB01F02F
:10ECD00000F002F810BD00002DE9F0410446F5F700
:10ECE00003FE07460025074800680749B0FBF1F01E
:10ECF00000FB04F602E0F5F7F7FDC51BB542FAD3B9
:10ED0000BDE8F0817807002040420F0008B5684652
:10ED1000F9F7DAFB08BD10B54FF47A70FFF7D2FFB0
:10ED20004FF44070F9F73CF84FF4E13005F046F845
:10ED3000FDF79CFBFDF738FD00210420F5F794F862
:10ED400000210420F4F7D0FEF7F738FF02F048FC6A
:10ED50006420FFF7B7FF10BD10B54FF4C0727E21DD
:10ED60007F20FDF7EFF810BD10B50446072C05D045
:10ED7000082C03D0092C01D00A2C2FD17A4890ED11
:10ED8000024AD0ED013A90ED003A7848D0ED022ADF
:10ED900090ED012AD0ED001A754890ED021AD0EDE1
:10EDA000010A90ED000AF6F723FE724880ED000A92
:10EDB000C0ED010A80ED021AD0ED022A90ED012A81
:10EDC000D0ED001A6C4890ED021AD0ED010A90EDDA
:10EDD000000AFCF75DFA694880ED080A072C74D236
:10EDE000DFE804F0040574A2A9B0B700B9E06049F7
:10EDF00008316248001D01F09BFE6148D0ED022AF7
:10EE000090ED012AD0ED001A5E4890ED021AD0ED87
:10EE1000010A90ED000AF6F7C3FA584880ED090A96
:10EE200090ED091AF0EE410A514890ED021AB0EE49
:10EE3000410AF6F787FA514880ED000A524890EDF2
:10EE4000000ADFED520AB4EEE00AF1EE10FA06DB3A
:10EE500018224A4938314E48F1F75EFE1FE04A4811
:10EE600090ED000ADFED490AB4EEE00AF1EE10FA87
:10EE70000FD290ED000ADFED470AB4EEE00AF1EEA2
:10EE800010FA06DB18223D4950314148F1F744FEA3
:10EE900005E01822394968313D48F1F73DFE374811
:10EEA000D0ED040A3848B0F86A0000EE100AB8EE57
:10EEB000400AF4EEC00AF1EE10FA05D218222F49EA
:10EEC00080313348F1F728FE4BE049E0284908310A
:10EED0002A48001D01F02CFE2948D0ED022A90EDB1
:10EEE000012AD0ED001A274890ED021AD0ED010A50
:10EEF00090ED000AF6F754FA204880ED090A90EDEB
:10EF0000091AF0EE410A1A4890ED021AB0EE410AD1
:10EF1000F6F718FA194880ED000A182200F150019E
:10EF20001B48F1F7F9FD1CE0114908311348001D99
:10EF300001F0FEFD15E00E4908311048001D01F0FA
:10EF4000F7FD0EE00A4908310C48001D01F0F0FD04
:10EF500007E0074908310948001D01F0E9FD00E01C
:10EF600000BF00BF10BD00007421022068210220F4
:10EF700044210220802102205C21022094200220D2
:10EF8000382102202C210220641F02200000FA43B5
:10EF90007C2002200000484310B52DED048B044670
:10EFA0000B2C6FD2DFE804F00607F8F7F6F5F4F360
:10EFB000F2F1F0001FE3F848D0ED022A90ED012AAB
:10EFC000D0ED001AF54890ED021AD0ED010A90ED4F
:10EFD000000AF6F7E5F9F24880ED090A90ED091A02
:10EFE000F0EE410AEF4890ED021AB0EE410AF6F752
:10EFF000A9F9EB4880ED000AE74890ED024AD0ED10
:10F00000013A90ED003AE548D0ED022A90ED012A50
:10F01000D0ED001AE34890ED021AD0ED010A90ED10
:10F02000000AF5F767FCB0EE409AF0EE609A51ECFA
:10F03000190B05F033FA41EC180B05F03BFAD849EF
:10F040004860084690ED010A10EE101A084606F0D6
:10F050003FF841EC190BB0EE490AF0EE690AFDF7F2
:10F06000AFFFB0EE408AF0EE608A9FEDCF0B53EC1D
:10F07000102B51EC180B05F033FE04D20520CC49BF
:10F08000087003E0B6E20320C9490870C44890ED57
:10F09000000A10EE101A084606F01AF841EC180B98
:10F0A0009FEDC40B53EC102B05F01AFE0AD29FED16
:10F0B000C30AC34880ED090A9FEDC20AC24880ED29
:10F0C000090A25E0B64890ED000A10EE101A08462D
:10F0D00005F0FEFF41EC180B9FEDBC0B53EC102B21
:10F0E00005F0C4FC0AD29FEDB70AB54880ED090AC5
:10F0F0009FEDB20AB44880ED090A09E0B7EE000AB4
:10F10000AF4880ED090AB7EE000AAF4880ED090A62
:10F11000A34890ED010AF0EE080AB4EEE00AF1EE21
:10F1200010FA12DDA248007800EE100AB8EE400A8C
:10F13000A84880ED070A9E48007800EE100AB8EE55
:10F14000400AA54880ED070A31E0954890ED010A94
:10F15000F8EE080AB4EEE00AF1EE10FA1DD2944877
:10F160000078404200EE100AB8EEC00A994880EDDF
:10F17000070A8F480078404200EE100AB8EEC00A35
:10F18000954880ED070A12E0F1E1ADE16DE12DE176
:10F190002BE129E127E125E10AE09FED900A8D4866
:10F1A00080ED070A9FED8D0A8B4880ED070A22E269
:10F1B0007948D0ED022A90ED012AD0ED001A774867
:10F1C00090ED021AD0ED010A90ED000AF6F7E8F88A
:10F1D000734880ED090A90ED091AF0EE410A714872
:10F1E00090ED021ADFED7E1A31EE211AB0EE410ADF
:10F1F000F6F7A8F86A4880ED000A674890ED024AE1
:10F20000D0ED013A90ED003A6448D0ED022A90ED3D
:10F21000012AD0ED001A634890ED021AD0ED010AE0
:10F2200090ED000AF5F766FBB0EE408AF0EE608ADA
:10F2300051EC180B05F03EF959494860084690ED2D
:10F24000010A10EE101A084605F042FF41EC190BB6
:10F25000B0EE490AF0EE690AFDF7B2FEB0EE408A60
:10F26000F0EE608A9FED500B53EC102B51EC180B15
:10F2700005F036FD03D205204D49087002E0032059
:10F280004B490870464890ED000A10EE101A0846E7
:10F2900005F01EFF41EC180B9FED460B53EC102BB5
:10F2A00005F01EFD0AD29FED470A454880ED090A88
:10F2B0009FED420A444880ED090A25E0384890ED68
:10F2C000000A10EE101A084605F002FF41EC180B78
:10F2D0009FED3E0B53EC102B05F0C8FB0AD29FEDBF
:10F2E000370A374880ED090A9FED360A364880ED27
:10F2F000090A09E0B7EE000A314880ED090AB7EEC5
:10F30000000A314880ED090A254890ED010AF0EE27
:10F31000080AB4EEE00AF1EE10FA14DD2448007891
:10F32000404200EE100AB8EEC00A2A4880ED070AF3
:10F330001F480078404200EE100AB8EEC00A264886
:10F3400080ED070A26E0164890ED010AF8EE080A5B
:10F35000B4EEE00AF1EE10FA12D21548007800EE91
:10F36000100AB8EE400A1B4880ED070A10480078E2
:10F3700000EE100AB8EE400A174880ED070A09E0CF
:10F380009FED160A134880ED070A9FED140A1248F4
:10F3900080ED070A2FE10000382102202C210220F5
:10F3A00094200220442102200000000000002E4092
:10F3B000F01D00209CC420B07268913FCDCC8C3FE2
:10F3C000181701206666663F681701209CC420B0AC
:10F3D000726891BF401701209017012000000000C3
:10F3E000DA0F494007E106E105E104E18448D0ED88
:10F3F000022A90ED012AD0ED001A824890ED021AFF
:10F40000D0ED010A90ED000AF5F7CAFF7E4880EDC5
:10F41000090A90ED091AF0EE410A7C4890ED021AB3
:10F42000B0EE410AF5F78EFF774880ED000A784884
:10F43000D0ED022A90ED012AD0ED001A734890ED2C
:10F44000021AD0ED010A90ED000AFBF721FF6E4889
:10F45000D0ED080A30EE600A80ED010A182200F1B2
:10F4600068016C48F1F758FBC5E06548D0ED022A09
:10F4700090ED012AD0ED001A624890ED021AD0ED0D
:10F48000010A90ED000AF5F78BFF5F4880ED090A4D
:10F4900090ED091AF0EE410A5C4890ED021AB0EEC8
:10F4A000410AF5F74FFF584880ED000A5848D0ED63
:10F4B000022A90ED012AD0ED001A544890ED021A6C
:10F4C000D0ED010A90ED000AFBF7E2FE4E48D0EDC8
:10F4D000080A30EE600A80ED010A182200F1680186
:10F4E0004C48F1F719FB86E04548D0ED022A90ED33
:10F4F000012AD0ED001A434890ED021AD0ED010A1E
:10F5000090ED000AF5F74CFF3F4880ED090A90EDB9
:10F51000091AF0EE410A3D4890ED021A5FED501ACB
:10F5200031EE211AB0EE410AF5F70CFF364880EDB6
:10F53000000A3748D0ED022A90ED012AD0ED001ADA
:10F54000324890ED021AD0ED010A90ED000AFBF767
:10F550009FFE2D48D0ED080A30EE600A80ED010ACA
:10F56000182200F168012B48F1F7D6FA43E024484D
:10F57000D0ED022A90ED012AD0ED001A214890ED3D
:10F58000021AD0ED010A90ED000AF5F709FF1E48B6
:10F5900080ED090A90ED091AF0EE410A1B4890ED42
:10F5A000021A5FED711A31EE211AB0EE410AF5F739
:10F5B000C9FE154880ED000A1548D0ED022A90EDED
:10F5C000012AD0ED001A114890ED021AD0ED010A7F
:10F5D00090ED000AFBF75CFE0B48D0ED080A30EE18
:10F5E000600A80ED010A182200F168010948F1F76C
:10F5F00093FA00E000BF00BFBDEC048B10BD00001B
:10F60000742102206821022094200220442102203B
:10F61000802102207C20022070B504460D4620681F
:10F6200058B9294604F1080004F0B9FB08B90020D4
:10F6300070BD022020600020FAE72168481C20608D
:10F6400004F108004554206806280BD104F10A0093
:10F65000FBF776FE6060B0F5FD7F03DD00202060E3
:10F66000401EE5E7D4E90010801D814201DA002048
:10F67000DEE700202060204600F072FBD8E70A4653
:10F680000271130A4371130C8371130EC371704717
:10F690000A460270130A4370130C8370130EC37072
:10F6A000704700005C4890F82000072879D2DFE816
:10F6B00000F004194169798897009FED580A58486D
:10F6C00080ED010A9FED550A564880ED010A9FED35
:10F6D000560A564880ED010A9FED530A544880EDC2
:10F6E000010A97E04C4890ED000AB5EEC00AF1EE31
:10F6F00010FA0AD19FED490A494880ED010A9FEDB1
:10F70000470A484880ED010A13E0434890ED000A9B
:10F710004348D0ED090A20EE200A80ED010A3E4858
:10F7200090ED000A3F48D0ED090A20EE200A80ED56
:10F73000010A6FE0384890ED000AB5EEC00AF1EE1C
:10F7400010FA0AD19FED350A354880ED010A9FED88
:10F75000330A344880ED010A13E02F4890ED000A87
:10F760002F48D0ED090A20EE600A80ED010A2A48F0
:10F7700090ED000A2B48D0ED090A20EE600A80EDDA
:10F78000010A47E0244890ED000AB1EE400A2448FF
:10F7900080ED010A204890ED000A224880ED010A20
:10F7A00038E02CE01C4890ED000A1D4880ED010A6D
:10F7B000194890ED000AB1EE400A1A4880ED010A9E
:10F7C00028E0154890ED000AB1EE400A144880ED9B
:10F7D000010A114890ED000A124880ED010A19E073
:10F7E0000D4890ED000A0E4880ED010A0A4890EDA0
:10F7F000000AB1EE400A0B4880ED010A0AE09FEDD5
:10F80000070A074880ED010A9FED040A054880EDCC
:10F81000010A00BF00BF7047641F02200000000003
:10F82000181701206817012000409C45401701204F
:10F830009017012010B54848407908287ED2DFE8AB
:10F8400000F004192E45505B66729FED440A44484F
:10F8500080ED010A9FED410A424880ED010A9FEDCB
:10F86000420A424880ED010A9FED3F0A404880ED80
:10F87000010A64E03848B0F86C0000EE100AB8EEF7
:10F88000400A374880ED010A3348B0F86C0000EEBA
:10F89000100AB8EE400A334880ED010A4FE02E48C6
:10F8A000B0F86C00404200EE100AB8EEC00A2C48D6
:10F8B00080ED010A2848B0F86C00404200EE100AC2
:10F8C000B8EEC00A274880ED010A38E09FED290A0A
:10F8D000264880ED070A9FED270A254880ED070A94
:10F8E0002DE09FED1E0A214880ED070A9FED1B0ABF
:10F8F0001F4880ED070A22E09FED1F0A1B4880ED9C
:10F90000070A9FED1D0A1A4880ED070A17E09FEDD0
:10F910001B0A134880ED010A9FED190A114880ED7A
:10F92000010A0CE00AE09FED160A0D4880ED010A7D
:10F930009FED120A0B4880ED010A00E000BF00BFF6
:10F940000548B0F86E0000EE900AF8EE600AB0EEDE
:10F95000600A03F0EBFB10BD641F022000000000F2
:10F96000181701206817012000409C45401701200E
:10F97000901701200000B442000060420000C8421D
:10F980000000C8C210B504462078012802D02078B3
:10F99000022802D1F6F726FF29E02078032808D0B4
:10F9A0002078042805D02078052802D02078062861
:10F9B00002D1F6F76FFB1AE02078072808D02078EC
:10F9C000082805D02078092802D020780A2802D1FA
:10F9D000F6F792FE0BE020780B2802D020780C2856
:10F9E00005D10348007810B10420FBF733FA10BDAD
:10F9F000B81F002010B501201049887601210F485A
:10FA000080F8DD104FF4D560FAF766FC00210B4852
:10FA100080F8DB1080F8DA1040F2B4710848F1F792
:10FA2000ADF84020FBF716FA9FED060A064880ED78
:10FA3000030A00200549087010BD0000641F022061
:10FA4000C06D01200000000094200220901F0020C3
:10FA500010B5044600BF042C02DD4FF0FF3010BD8E
:10FA600000BF210201F201401021FCF703FA00BFA0
:10FA7000210201F20140FCF7A9F90028F8D1210286
:10FA800001F20240FF21FCF7F5F90120A0400E49E8
:10FA9000098881430C4801800120A0400B49098856
:10FAA00081430A4801800020094921F814000949CE
:10FAB000085500BF210201F20340FCF787F9002836
:10FAC000F8D10120CBE7000056090020580900209A
:10FAD0005A0900206209002070B52DED048B0546FF
:10FAE0000C46082D07D2DFE805F0810407121D330C
:10FAF000537340490C7479E001203F49887500EE4A
:10FB0000104AB8EEC00A3D4880ED0C0A6EE00220B3
:10FB10003949887500EE104AB8EEC00A374880EDC2
:10FB20000C0A63E014B1012C10D107E00021082079
:10FB3000F9F7E4FA00203249487007E00121082073
:10FB4000F9F7DCFA01202E49487000BF00BF4DE0F4
:10FB50002A494D7100EE104AB8EEC00A10EE100AA4
:10FB600005F0B6FA41EC190B9FED260B53EC102B68
:10FB700004F08EFD41EC180B04F09CFC1F49486317
:10FB800000EE104AB8EEC00A084680ED0C0A2DE0DF
:10FB90001A494D7100EE104AB8EEC00A10EE100A74
:10FBA00005F096FA41EC190B9FED160B53EC102B58
:10FBB00004F06EFD41EC180B04F07CFC0F49486327
:10FBC00000EE104AB8EEC00A084680ED0C0A0DE0BF
:10FBD00014B1012C08D103E00420FAF77DFB03E007
:10FBE0000420FBF737F900BF00BF00BF00BFBDEC2A
:10FBF000048B70BDEC1701200C180120641F02203B
:10FC0000C06D01206666666666A64C403A4A127967
:10FC100022B9394AD2F81421384B1A60082868D220
:10FC2000DFE800F0670413212F3D4B5911B1012982
:10FC300009D104E00022304B1A71DA6203E001229C
:10FC40002D4B1A7100BF00BF53E011B1012908D13B
:10FC500003E00022284B5A7103E00122264B5A711F
:10FC600000BF00BF45E011B1012908D103E0002227
:10FC7000214B5A7103E002221F4B5A7100BF00BF93
:10FC800037E011B1012908D103E000221A4B5A7163
:10FC900003E00322184B5A7100BF00BF29E011B1E5
:10FCA000012908D103E00022134B5A7103E004221A
:10FCB000114B5A7100BF00BF1BE011B1012908D1DF
:10FCC00003E000220E4B1A7403E001220C4B1A745D
:10FCD00000BF00BF0DE011B1012908D103E00022EF
:10FCE000074B1A7403E00222054B1A7400BF00BFD1
:10FCF00000BF00BF70470000641F02208021002069
:10FD0000EC170120F0B503460C461888002113E0DB
:10FD1000675C80EA072000250BE0460000F4004CF9
:10FD2000BCF1000F03D041F2210C86EA0C063046EC
:10FD30006D1C082DF1D3491C9142E9D31880F0BD08
:10FD400010B510210148F5F751FE10BD000002402A
:10FD500010B510210148F5F747FE10BD0000024024
:10FD600038B5044600200090042204F108016846DA
:10FD7000FFF7C8FF04F10E0168466268FFF7C2FF93
:10FD800004F10C00FBF7DCFABDF80010884202D049
:10FD90004FF0FF3038BD204601F066FEFAE7000064
:10FDA00030B5ADF2D47D40F20360FCF70FF810B12E
:10FDB00022283DD107E000233A4802880221084664
:10FDC00003F076FE34E040F20260FBF7FFFF00F044
:10FDD000040020B1042140F20260FCF74BF802203D
:10FDE00001F066F83049088000280BDD2F48304BC1
:10FDF00000900846028801A9022002F0DDFD0120E2
:10FE00002C4908702C4890F8280080B12B48F0F756
:10FE1000C8FD85B225480088254B2A462749009011
:10FE2000022003F08BF80020234981F8280000BF4E
:10FE300000BF20480078012830D100201E4981F8F9
:10FE400028001C490870002424E01D4890F8900404
:10FE500050B901A9085D1B49F5F762FB042803D1DD
:10FE60000121174880F89014154890F8900480B14B
:10FE7000F5F736FC08B9FAF71FFF0021104880F8A3
:10FE80009014A0F5805090F83C0E012801D1FAF7AB
:10FE9000DDF9641C044800888442D6D30DF2D47D79
:10FEA00030BD0000200B0020080D00202A0B002090
:10FEB000260B00200A0D0020641F02206C17022070
:10FEC000D012022020B001202DE9F05F06460D4639
:10FED0004FF0000B2888052848D170784FEA002998
:10FEE000B07840EA090909F101001FFA80F9F078B9
:10FEF000040230790443012C35DBB4F5FA6F32DAB1
:10FF0000374600202880012007F8010B2888401C74
:10FF1000288004F0070040B12046E11704EB51713E
:10FF2000C910491C01F0FF0805E02046E11704EB69
:10FF30005171C1F3C70807F8018B2888401C28803D
:10FF4000002322464946384600F04EFA8246BAF16E
:10FF5000000F04D0504602F015FD834608E02888C3
:10FF60004044288004E04FF0030B01E04FF0030B06
:10FF70005846BDE8F09F2DE9F05F06460D464FF06C
:10FF8000000B2888052847D170784FEA0029B078FF
:10FF900040EA090909F101001FFA80F9F07804022A
:10FFA00030790443012C34DBB4F5FA6F31DA37468B
:10FFB00000202880022007F8010B2888401C288098
:10FFC00004F0070040B12046E11704EB5171C9105D
:10FFD000491C01F0FF0805E02046E11704EB5171D0
:10FFE000C1F3C70807F8018B2888401C28802246E7
:10FFF0004946384600F07CFA8246BAF1000F04D038
:020000040801F1
:10000000504602F0BFFC834608E028884044288020
:1000100004E04FF0030B01E04FF0030B5846BDE83E
:10002000F09F2DE9F04705460C464FF0000A208866
:10003000052837D168784FEA0028A87840EA0808F0
:1000400008F101001FFA80F8E87806022E79012EE7
:1000500025DB7D2E23DC2F4600202080032007F89F
:10006000010B2088401C20807006000E07F8010B51
:100070002088401C2080002332464146384600F04C
:1000800089FA8146B9F1000F04D0484602F07AFCA3
:10009000824609E0208800EB4600208004E04FF013
:1000A000030A01E04FF0030A5046BDE8F0872DE94E
:1000B000F04705460C464FF0000A2088052837D146
:1000C00068784FEA0028A87840EA080808F101009B
:1000D0001FFA80F8E878060228790643012E24DB0F
:1000E0007D2E22DA2F4600202080042007F8010B05
:1000F0002088401C20807006000E07F8010B208825
:10010000401C208032464146384600F081FA814644
:10011000B9F1000F04D0484602F034FC824609E0F1
:10012000208800EB4600208004E04FF0030A01E045
:100130004FF0030A5046BDE8F0872DE9FC5F044606
:100140000D460020009028880A285DDB60784FEA81
:10015000002AA07840EA0A0A0AF101001FFA80FA90
:10016000E07806022079064360794FEA002BA079F7
:1001700040EA0B0B0BF101001FFA80FBE07907024C
:10018000207A0743607A0190012E3BDB7D2E39DC1B
:10019000012F37DB792F35DC79000198814231D18D
:1001A00001233A46594604F10A0000F0F3F981466A
:1001B000B9F1000F1ED1A04600202880172008F8B2
:1001C000010B2888401C28807006000E08F8010BDF
:1001D0002888401C2880002332465146404600F0C3
:1001E000D9F98146B9F1000F04D12888022101FB19
:1001F00006002880B9F1000F06D0484602F0C2FB85
:10020000009001E0032000900098BDE8FC9F0000F2
:1002100070B505460C46064802880649681CF0F78A
:1002200036FC03480088401C2080002070BD000080
:10023000E22C0020662502202DE9F84304460F46F3
:100240004FF000083888052829D160780502A07889
:100250000543681C85B22079F0B9E078FF2801D009
:10026000E078C8B900208DF80100E078FF2803D1BC
:1002700001208DF8000002E000208DF8000001232D
:100280001A462946684600F0AFF806464EB1304699
:1002900002F078FB804604E04FF0030801E04FF0E5
:1002A00003084046BDE8F8832DE9F04104460F46B7
:1002B0004FF000083888052812D160780502A07830
:1002C0000543681C85B201231A462946E01C00F04C
:1002D00061F9064636B1304602F054FB804601E033
:1002E0004FF003084046BDE8F0812DE9F05F054678
:1002F0000E464FF0000B3088052839DD687807027C
:10030000A8780743781C87B2E87804022879044368
:1003100095F805A004F0070040B12046E11704EB72
:100320005171C910491C01F0FF0805E02046E11792
:1003300004EB5171C1F3C708012C16DBB4F5F66F5D
:1003400013DCD04511D1012322463946A81D00F007
:100350004BF88146B9F1000F04D0484602F012FB79
:10036000834607E00520308004E04FF0030B01E0F6
:100370004FF0030B5846BDE8F09F2DE9F0470446C7
:100380000E464FF0000A3088062828DB6078070206
:10039000A0780743781C87B2E078050220790543EE
:1003A00094F80590012D17DB782D15DC6806000EFA
:1003B000484511D101232A463946A01D00F0EAF82C
:1003C0008046B8F1000F04D0404602F0DBFA8246C6
:1003D00007E00520308004E04FF0030A01E04FF011
:1003E000030A5046BDE8F0872DE9F05F05460E464A
:1003F00014469A464FF0000B2046E11704EB51716A
:10040000C91001F10109012E68DB3019612865DC92
:1004100035490988701AC11700EB5171CF10324964
:100420000988701AC11700EB5171C910A0EBC108FF
:10043000BAF1000F03D0BAF1010F4ED124E00CE065
:100440001FFA88F13A467F1C284BD018082203F087
:10045000B4FF05F8010BA9F10109B9F1000FEFDCB8
:100460006D1E2046E11704EB5171C910A4EBC101C8
:100470008CB22878C4F10801884028702878C4F12B
:1004800008010841287028E00EE015F8013B1FFA2A
:1004900088F13A467F1CDFF854C002EB0C000822BA
:1004A00003F0A0FFA9F10109B9F1010FEDDC20462D
:1004B000E11704EB5171C910A4EBC1018CB215F81E
:1004C000013BE2B21FFA88F1BC467F1CDFF81CE05A
:1004D0000CEB0E0003F086FF00BF01E04FF0010BB4
:1004E0005846BDE8F09F0000262C00200223022081
:1004F0002DE9F04705460E4614464FF0000A204607
:10050000E11704EB5171C91001F10109012E37DB2C
:100510003019612834DC1D490988701AC11700EBB5
:100520005171CF1019490988701AC11700EB517128
:10053000C910A0EBC1080CE01FFA88F13A467F1CF5
:10054000134BD018082203F038FF05F8010BA9F16E
:100550000109B9F1000FEFDC6D1E2046E11704EB35
:100560005171C910A4EBC1018CB22878C4F1080103
:10057000884028702878C4F108010841287001E0FB
:100580004FF0010A5046BDE8F0870000242C0020FF
:10059000F6220220F0B504460D460020012D31DB85
:1005A000AE18652E2EDC184E3688A91B13B1012B10
:1005B00027D111E00DE0154E36F81160360A04F827
:1005C000016B124E16F8116004F8016B491C561E9F
:1005D000B2B2002AEFDC14E011E014F8017B3E0215
:1005E00036B20A4F27F8116014F8016B37F9117011
:1005F0003E43064F27F81160491C561EB2B2002A2E
:10060000EBDC00E00120F0BD2A2C0020D6230220E4
:1006100030B503460020012917DB8D18652D14DC49
:100620000B4D2D884C1B0DE00A4D35F814502D0A4A
:1006300003F8015B074D15F8145003F8015B641CC7
:10064000551EAAB2002AEFDC00E0012030BD0000F8
:10065000282C00200E23022082B0CDE9000121F0D9
:10066000004001909DED000B02B051EC100B704763
:1006700010B582B01446CDE900010023009A236032
:10068000194B21F0004098422ADA024328D0B0F5F5
:10069000801FA8BF226810DA9FED150B53EC102BBA
:1006A0009DED000B51EC100B04F01CFACDE900019C
:1006B0006FF0350221F0004022600F4B6FF31E51A6
:1006C00003EB20501044206041F0FF5040F00050F8
:1006D00001909DED000B00BF02B051EC100B10BD5E
:1006E0009DED000BF8E700000000F07F0000000027
:1006F000000000000000504302FCFFFF30B52DED6C
:10070000068B83B004460D46A069012828D194EDDC
:10071000000A8DED000A9DED000A10EE101A084641
:1007200004F0D6FC41EC1A0B95ED081BB0EE410A23
:10073000F0EE610A53EC102B04F0D4F941EC190BE4
:1007400095ED0A1BB0EE410AF0EE610A53EC102B56
:1007500003F0E2FE41EC180B03F0ACFE0190F0E078
:10076000A869012828D195ED000A8DED000A9DEDBC
:10077000000A10EE101A084604F0AAFC41EC1A0B0D
:1007800094ED081BB0EE410AF0EE610A53EC102B19
:1007900004F0A8F941EC190B94ED0A1BB0EE410AE4
:1007A000F0EE610A53EC102B03F0B6FE41EC180B8F
:1007B00003F080FE0190C4E094ED081BB0EE410A06
:1007C000F0EE610A9FED641B53EC112B51EC100B02
:1007D00004F0B6F828D194ED010A8DED010A9DEDE3
:1007E000010A10EE101A084604F072FC41EC1A0BD4
:1007F00095ED0A1BB0EE410AF0EE610A53EC102BA6
:1008000004F07CFB41EC190B95ED081BB0EE410A9E
:10081000F0EE610A53EC102B03F03AFF41EC180B99
:1008200003F048FE00908CE095ED081BB0EE410A05
:10083000F0EE610A9FED481B53EC112B51EC100BAD
:1008400004F07EF828D195ED010A8DED010A9DEDA9
:10085000010A10EE101A084604F03AFC41EC1A0B9B
:1008600094ED0A1BB0EE410AF0EE610A53EC102B36
:1008700004F044FB41EC190B94ED081BB0EE410A67
:10088000F0EE610A53EC102B03F002FF41EC180B61
:1008900003F010FE009054E095ED082BB0EE420AF4
:1008A000F0EE620A94ED082BB0EE421AF0EE621AF6
:1008B00053EC102B51EC110B04F020FB41EC180B06
:1008C00094ED0A2BB0EE420AF0EE620A95ED0A2B87
:1008D000B0EE421AF0EE621A53EC102B51EC110BF1
:1008E00004F00CFB41EC190B53EC182B03F0D0FE79
:1008F00041EC1A0B03F0DEFD00909DED000A10EEB6
:10090000101A084604F0E4FB41EC1A0B94ED081BA6
:10091000B0EE410AF0EE610A53EC102B04F0E2F85D
:1009200041EC190B94ED0A1BB0EE410AF0EE610A9E
:1009300053EC102B03F0F0FD41EC180B03F0BAFD63
:1009400001909DED000ADDED010A9DED021A03B054
:10095000BDEC068B30BD0000000000000000000070
:1009600011B52DED040B2DED088B8DB0044615A8A7
:1009700007C88DE807009DED170A10EE101A08460B
:1009800004F0A6FB41EC1B0BB0EE4B0AF0EE6B0A39
:10099000FCF716FBB0EE40AAF0EE60AA9FED300B1C
:1009A00053EC102B51EC1A0B04F0A8FA41EC190B84
:1009B000B0EE490AF0EE690AFCF702FBB0EE408A9D
:1009C000F0EE608A9FED280B53EC102B51EC180BC6
:1009D00004F04CF802D20120069036E00020069088
:1009E0009DED170A10EE101A084604F071FB41EC59
:1009F000180BB0EE480AF0EE680AFDF721FA8DED0B
:100A0000080B9DED150A10EE101A084604F060FB65
:100A100041EC1A0B9DED081BB0EE410AF0EE610AA5
:100A200053EC102B04F05EF841EC180B9DED160A08
:100A300010EE101A084604F04BFB41EC190B53EC76
:100A4000182B04F05BFACDE90A01302269462046F2
:100A5000F0F762F80DB0BDEC088B05B010BD0000DA
:100A600000000040FB21F93FFCA9F1D24D62503F4C
:100A700031B52DED060B2DED068B8CB0044612A87A
:100A800007C88DE8070015A807C803AB07C39DED8D
:100A9000000ADDED030AB4EE600AF1EE10FA02D1AD
:100AA000012006903AE0002006909DED010ADDED60
:100AB000040A30EE600ADDED000A9DED031A70EEC7
:100AC000C10A80EE201A11EE105A284604F000FBED
:100AD000CDE908019DED000A10EE101A084604F059
:100AE000F7FA41EC1A0B9DED081BB0EE410AF0EE4F
:100AF000610A53EC102B03F0F5FF41EC180B9DED50
:100B0000010A10EE101A084604F0E2FA41EC190B43
:100B100053EC182B04F0F2F9CDE90A0130226946B2
:100B20002046EFF7F9FF0CB0BDEC068B07B030BDE7
:100B300070B52DED108B94B005460C46CA4890ED6B
:100B4000010ACA48D0ED010A30EE200AF0EE000A90
:100B500080EE201AB7EE000A21EE000A10EE106AAD
:100B6000304604F0B5FA41EC180BC14890ED010A8B
:100B700084ED000A94ED000ADFEDBE0AB4EEE00A4F
:100B8000F1EE10FA08DD94ED000ADFEDBA0A30EE5E
:100B9000600A84ED000A10E094ED000ADFEDB60A69
:100BA000B4EEE00AF1EE10FA07D294ED000ADFEDA0
:100BB000B10A30EE200A84ED000AB048407F0128D7
:100BC0007ED1AE4890ED030AF7EE000A20EE200A2F
:100BD00085ED000AAA4801680068401CA84A106018
:100BE00014296EDD002011460860A64890ED040A25
:100BF00010EE101A084604F06BFA41EC190B9C48F1
:100C000090ED010A10EE101A084604F061FA41EC6A
:100C10001F0B9FED9D0B53EC102B03F063FF41EC7A
:100C20001A0B94ED000A10EE101A084604F050FA60
:100C300041EC1F0B9FED940B53EC102B03F052FF74
:100C400041EC1B0B95ED000A10EE101A084604F05B
:100C50003FFA41EC1C0B8B4890ED030A10EE101A82
:100C6000084604F035FA41EC1D0B814890ED000A6E
:100C700010EE101A084604F02BFA41EC1E0B7B48CC
:100C800090ED000A10EE101A084604F021FACDE9A2
:100C90001201754890ED000A10EE101A084604F093
:100CA00017FACDE910018DED0E9B8DED0CAB8DED9E
:100CB0000ABB8DED08CB8DED06DB8DED04EB01E07D
:100CC0000FE094E08DED028B9DED120B8DED000B8E
:100CD0009DED100B53EC102B6D490120FBF744F8F0
:100CE0009AE06C48D0F814016B490968401A14283E
:100CF0007DD36848D0F814016749086051EC180B9F
:100D000003F0D8FB09EE100A594890ED000AB0EE46
:100D1000401A224629460020DFED601ADFED600A06
:100D2000B0EE490AF4F776F9564890ED040A10EE51
:100D3000101A084604F0CCF941EC190B4C4890ED20
:100D4000010A10EE101A084604F0C2F941EC1F0B1C
:100D50009FED4D0B53EC102B03F0C4FE41EC1A0B2E
:100D600094ED000A10EE101A084604F0B1F941ECB7
:100D70001F0B9FED450B53EC102B03F0B3FE41EC22
:100D80001B0B95ED000A10EE101A084604F0A0F9AE
:100D900041EC1C0B3B4890ED030A10EE101A08467C
:100DA00004F096F941EC1D0B314890ED000A10EE6D
:100DB000101A084604F08CF9CDE912012B4890ED89
:100DC000000A10EE101A084604F082F9CDE910016D
:100DD000254890ED000A10EE101A084604F078F944
:100DE00041EC1E0B8DED0C9B8DED0AAB00E013E08A
:100DF0008DED08BB8DED06CB8DED04DB9DED120B6B
:100E00008DED020B9DED100B8DED000B53EC1E2BA9
:100E100024490120FAF7A8FF1E48D0F814012249FE
:100E20000968401A1E281BD31A48D0F814011E491D
:100E3000086051EC180B03F03DFB09EE100A0C485A
:100E400090ED000AB0EE401A224600210D480C3009
:100E5000DFED161ADFED120AB0EE490AF4F7DAF800
:100E600014B0BDEC108B70BDE816012000170120F6
:100E7000E0170120DA0FC940DA0FC9C02816012097
:100E8000301C0020942002206666666666A64C40F0
:100E900038580108641F0220281C00200AD7A33CF0
:100EA00000000000C45701082C1C00208FC2F53C34
:100EB00070B504460025002600BF210201F226403D
:100EC000FAF784FF0646210201F22740FAF77EFF77
:100ED00000EB062086B26EB1210201F22640FAF73D
:100EE00075FF0546210201F22740FAF76FFF00EB7C
:100EF000052085B2B542E0D1284670BD70B50546E3
:100F00004FF4C04600240FE01A20FAF75FFF62009A
:100F1000032191400840610008410121814088B2CD
:100F200006EB8026601C44B2AC42EDDB304670BD5F
:100F300070B504460025002600BF210201F584603B
:100F4000FAF744FF0646210201F22140FAF73EFF7C
:100F500000EB062086B26EB1210201F58460FAF73B
:100F600035FF0546210201F22140FAF72FFF00EB81
:100F7000052085B2B542E0D1284670BD70B5054662
:100F80004FF4804600240FE01B20FAF71FFF620099
:100F9000032191400840610008410121814088B24D
:100FA00006EB8026601C44B2AC42EDDB304670BDDF
:100FB000F0B52DED108B8FB005460C46B0EE408A93
:100FC00016461F46A86900287ED195ED081BB0EE95
:100FD000410AF0EE610A9FEDE71BFCF765F8B0EE01
:100FE00040CAF0EE60CA9FEDE50B53EC102B51ECBC
:100FF0001C0B03F091FA41EC190B94ED000A10EE72
:10100000101A084604F064F841EC1D0B94ED010A37
:1010100010EE101A084604F05BF841EC1F0B95ED3A
:101020000A1BB0EE410AF0EE610A53EC102B03F0FC
:101030008DFECDE9060195ED081BB0EE410AF0EEFC
:10104000610A53EC102B9DED061B51EC110B03F0C4
:1010500049FD41EC1E0B53EC1D2B03F04FFF41ECFF
:101060001C0B9FEDC40B53EC102B03F03BFD41EC2C
:101070001A0B18EE100A04F02BF841EC1E0B9FED32
:10108000BD1BB0EE4E0AF0EE6E0AFCF70DF8B0EEA6
:1010900040CAF0EE60CA94ED000A10EE101A08463D
:1010A00004F016F841EC1E0B9FEDB21BB0EE4E0A99
:1010B000F0EE6E0AFBF7F8FF8DED060B94ED010ADA
:1010C00010EE101A084600E021E104F001F841ECAE
:1010D0001F0B95ED0A1BB0EE410AF0EE610A53ECCE
:1010E000102B03F033FE41EC1E0B9FEDA21BB0EE64
:1010F0004E0AF0EE6E0AFBF7D7FF8DED040B9DED67
:10110000060B53EC102B9DED040B51EC100B03F070
:1011100003FA41EC1D0B53EC1C2B03F0EFFE41ECEA
:101120001B0B53EC192B9FED930B51EC100B03F0A1
:10113000D9FC41EC1C0B53EC192B9FED920B51EC9D
:10114000100B03F0CFFC41EC1F0B53EC1B2B03F0F7
:10115000C9FC9FED881BB0EE4A0AF0EE6A0ACDE9A1
:101160000201FBF7A1FF8DED000B9DED020B53EC8F
:10117000102B9DED000B51EC100B03F0BFFECDE9E1
:1011800004019DED040BFCF71BFEB0EE40EAF0EE0F
:1011900060EA51EC1A0B03F081F953EC1E2BCDE9F8
:1011A00006019DED060B51EC100B03F0B5F941EC77
:1011B0001D0B53EC1C2B03F06BFACDE90A0153EC29
:1011C000192B9FED6C0B51EC100B03F08BFC41ECD9
:1011D0001C0B53EC192B9FED6B0B51EC100B03F018
:1011E00081FC53EC1B2BCDE900019DED000B51EC74
:1011F000100B03F077FC9FED5F1BB0EE4A0AF0EE98
:101200006A0ACDE90201FBF74FFFB0EE40FAF0EEBB
:1012100060FA9DED020B53EC102B51EC1F0B03F009
:101220006DFECDE904019DED040BFCF7C9FD8DEDCC
:10123000060B51EC1A0B03F031F941EC1E0B9DED3E
:10124000060B53EC102B03F059FE41EC1D0B53EC35
:101250001C2B03F01DFACDE90801012E2BD19DEDC9
:101260000A0B51EC100B03F025F90C909DED0C0AC4
:1012700010EE101A084603F02BFF41EC1E0B95ED03
:10128000081BB0EE410AF0EE610A53EC102B03F09C
:1012900029FC41EC1D0B95ED0A1BB0EE410AF0EE66
:1012A000610A53EC102B03F037F941EC1C0B03F0EF
:1012B00001F90D902AE09DED080B51EC100B03F0A5
:1012C000F9F80C909DED0C0A10EE101A084603F088
:1012D000FFFE41EC1E0B95ED081BB0EE410AF0EE4F
:1012E000610A53EC102B03F0FDFB41EC1C0B95ED58
:1012F0000A1BB0EE410AF0EE610A53EC102B03F02A
:101300000BF941EC1D0B03F0D5F80D9028E0012EF0
:1013100013D194ED000A8DED0C0A781C30B994EDD0
:10132000010A30EE080A8DED0D0A19E094ED010A6C
:1013300030EE480A8DED0D0A12E094ED000A8DEDB5
:101340000C0A781C30B994ED010A30EE480A8DED94
:101350000D0A05E094ED010A30EE080A8DED0D0A44
:101360009DED0C0ADDED0D0A9DED0E1A0FB0BDECE2
:10137000108BF0BD000000000000004000000000E5
:101380000000F03F000000000000104070B52DED9F
:10139000068B8CB006460C46154695E807008DE88E
:1013A0000700A06901280FD1002006909FED2F0BA8
:1013B0008DED080B95ED010A10EE101A084603F0AA
:1013C00087FECDE90A0147E094ED081BB0EE410A23
:1013D000F0EE610A9FED251B53EC112B51EC100B25
:1013E00003F0AEFA02D10120069035E0002006900D
:1013F00094ED081BB0EE410AF0EE610A53EC102B9D
:101400009FED1C1B51EC110B03F042F9CDE90801D3
:101410009DED000A10EE101A084603F059FE41EC4B
:101420001A0B9DED081BB0EE410AF0EE610A53EC79
:10143000102B03F057FB41EC180B9DED010A10EE49
:10144000101A084603F044FE41EC190B53EC182B1C
:1014500003F054FDCDE90A01302269463046EFF72A
:101460005BFB0CB0BDEC068B70BD00000000000003
:1014700000000000000000000000F0BF10B550A107
:101480000120FAF771FC012051498876087100218A
:101490004F4880F8991080F89A10012180F8DD10EB
:1014A00000204B4981F820004A4908704A490870D9
:1014B0004FF496714648A0F86C106421A0F87210A1
:1014C0000121A0F86E100521A0F8701000204049FD
:1014D000C88140F2DC513E48A0F868106421A0F8B1
:1014E00066104FF4FA71A0F86A1042F21071A0F879
:1014F00074100120364988721F2088810120C8722B
:10150000002008834AF20100A1F864000846B0F800
:1015100064004AF20601884209D1B0EE080A2C485C
:1015200080ED1F0AB0EE000A80ED200A47E028484F
:10153000B0F864004AF20401884205D1B7EE080A07
:10154000234880ED1F0A3AE02148B0F864004AF2CF
:101550000101884208D1B0EE000A1D4880ED1F0A43
:1015600028201B49C8652AE01948B0F864004AF2EF
:101570000201884208D19FED190A154880ED1F0A23
:101580000421C0F888101AE01148B0F864004AF24B
:101590000301884209D1B0EE080A0D4880ED1F0A08
:1015A000B7EE000A80ED200A09E00948B0F86400AF
:1015B0004AF20501884202D128200549C86510BDBC
:1015C000B2CECAFDB3F5CABCBBAF0D0A0000000025
:1015D000641F0220EC1701200C18012066664640AB
:1015E00010B540F2B4710348EFF7C8FA4020F9F79C
:1015F00031FC10BDC06D0120B6EE000A2F4880ED11
:101600000E0A9FED2F0A80ED0F0A9FED2D0A80ED47
:10161000100AB7EE000A80ED110AB2EE080A80ED5A
:10162000120A9FED280A80ED130AB6EE000A80ED3B
:10163000140A9FED230A80ED150A9FED210A80ED23
:10164000160AB7EE000A80ED170AB2EE040A80ED22
:10165000180A9FED1C0A80ED190AB6EE000A80ED0B
:101660001A0A9FED170A80ED1B0A9FED150A80EDFF
:101670001C0AB7EE000A80ED1D0AB2EE0E0A80EDDC
:101680001E0A9FED100A80ED1F0A9FED0F0A80EDE4
:10169000200A9FED0B0A80ED210A9FED090A80EDDB
:1016A000220A9FED070A80ED230AB2EE0E0A80EDB2
:1016B000240A9FED040A80ED250A70479420022039
:1016C00000000000000020423333B33E0F4890ED8D
:1016D000400AD0ED0E0A30EE200A0D4880ED000AD7
:1016E0000A4890ED410AD0ED0F0A30EE200A084872
:1016F00080ED010A054890ED420AD0ED100A30EE67
:10170000200A034880ED020A70470000641F02208F
:1017100044210220074991F8C71019B1322801DD90
:10172000322006E0034991F8C61011B1642800DDAB
:1017300064207047641F02203348007C20B10128D8
:1017400008D002281DD110E09FED300A2E4880ED10
:10175000010A17E02E48B0F8740000EE100AB8EE47
:10176000400A294880ED010A0CE02948B0F87400CD
:10177000404200EE100AB8EEC00A234880ED010A8C
:1017800000E000BF00BF224890F8B30098B11E48A7
:1017900090ED010AB5EEC00AF1EE10FA0BD200206E
:1017A0001C4908709FED190A174880ED010A0020B6
:1017B0001549087412E0164890F8B20070B112484A
:1017C00090ED010AB5EEC00AF1EE10FA06DD9FEDCC
:1017D0000F0A80ED010A00200B4908740C4890F8AC
:1017E000B30020B14FF0FF30074948610AE00848D4
:1017F00090F8B20018B101200349486102E00020CE
:101800000149486170470000EC170120000000000A
:10181000641F0220542100202248807901280AD127
:101820002048B0F8740000EE100AB8EE400A1E48D6
:1018300080ED010A14E01B48807902280BD1194879
:10184000B0F87400404200EE100AB8EEC00A164824
:1018500080ED010A04E09FED150A134880ED010AAE
:10186000104890F8B30060B10F4890ED010AB5EE52
:10187000C00AF1EE10FA04D29FED0C0A80ED010AC5
:101880000FE0084890F8B20058B1074890ED010AFF
:10189000B5EEC00AF1EE10FA03DD9FED040A80ED0B
:1018A000010A7047641F0220EC17012000000000AD
:1018B00008B5F2F7CDFFFDF72EFAF2F74FF86846BC
:1018C000F6F798FA6846F1F7D5FD6846F6F7C0FBDB
:1018D000002008BDF0EE402AF4EEE02AF1EE10FA06
:1018E00002D2B0EE600A01E0B0EE620AF0EE402AE9
:1018F000F4EEC12AF1EE10FA02DDB0EE410A01E089
:10190000B0EE620AF0EE402A32EEE00A32EE613AC0
:1019100020EE030A71EE603A80EE233A33EE210A9C
:1019200070470000464991ED010A4649D1ED000A91
:10193000B4EE600AF1EE10FA0AD1414991ED000AC5
:101940004149D1ED000AB4EE600AF1EE10FA33D04D
:101950003B4991ED010A3B4981ED000A384991ED7F
:10196000000A394981ED000A354991ED000ADFEDA1
:10197000370A20EE200ADFED360A80EE201A90EDBD
:10198000040A21EE000AD1ED010A90ED031A00EEDF
:10199000810A304981ED000A91ED000A2E49D1ED0E
:1019A000000A30EE600A2D4981ED000A294991EDC7
:1019B000000A294981ED000A90ED000A2549D1ED80
:1019C000000A20EE200AD0ED010A254991ED001A07
:1019D00001EE200AD0ED020A204991ED001A01EE35
:1019E000200A174981ED0A0A91ED0A0AD0ED050A8D
:1019F000B4EEE00AF1EE10FA04DB90ED050A81ED99
:101A00000A0A11E00E4991ED0A0AD0ED050AF1EE3D
:101A1000600AB4EEE00AF1EE10FA05D890ED050A7E
:101A2000B1EE400A81ED0A0A0E490A680968491CAC
:101A30000C4B19600A2A02DD00211A46116070471A
:101A400094200220381C00203C1C0020000034435D
:101A5000DA0F4940401C0020481C0020441C002094
:101A60004C1C0020341C00202DE9F04104460025C8
:101A7000002704F10E0604F5D0600021C164016561
:101A8000002084F8D40606E3705DB02859D008DC45
:101A900062287DD090280DD091287AD0A02879D1C5
:101AA0001AE0C02877D0D02876D0D12875D0F02879
:101AB000F5D111E1012084F80902902194F8D4268F
:101AC000501C84F8D40604F2CC608154701940781C
:101AD000C4F80C02AD1CDDE2012084F80902A0214B
:101AE00094F8D426501C84F8D40604F2CC608154B7
:101AF0007019B0F9010000EE100AB8EEC00ADFED6F
:101B0000FE0A80EE201A84ED841A7019B0F90300E1
:101B100000EE100AB8EEC00ADFEDF70A80EE201AD8
:101B200084ED851A7019B0F9050000EE100AB8EEC0
:101B3000C00ADFEDF10A80EE201A84ED861AED1D51
:101B4000A8E2012084F80902B02194F8D426501CA0
:101B500084F8D40604F2CC6081547019B0F9010005
:101B600000EE100AB8EEC00AF2EE040A80EE201A67
:101B700084ED871A7019B0F9030000EE100AB8EE70
:101B8000C00AF2EE040A80EE201A84ED881A05E0FD
:101B900046E1B5E07CE210E044E075E07019B0F990
:101BA000050000EE100AB8EEC00AF2EE040A80EE5C
:101BB000201A84ED891AED1D6CE2012084F80902D7
:101BC000C02194F8D426501C84F8D40604F2CC60CA
:101BD00081547019B0F9010000EE100AB8EEC00A85
:101BE000F2EE040A80EE201A84ED8A1A7019B0F918
:101BF000030000EE100AB8EEC00AF2EE040A80EE0E
